:10000000B01E02200D0201081502010817020108A6
:10001000190201081B0201081D020108000000006E
:100020000000000000000000000000001F020108A6
:10003000210201080000000023020108CD85030809
:10004000472F040827020108270201082702010898
:100050002702010827020108270201081B360108B0
:1000600027020108270201082702010827020108C8
:1000700027020108270201082702010827020108B8
:1000800027020108270201082702010827020108A8
:100090002702010827020108270201082702010898
:1000A0002702010827020108270201082702010888
:1000B0003D8603082702010827020108213B0208A8
:1000C000193B02082702010827020108270201083C
:1000D00027020108A5A10308270201082702010839
:1000E0002702010827020108270201082702010848
:1000F0002702010827020108270201082702010838
:100100002702010827020108270201082702010827
:1001100027020108D99A03082702010827020108CB
:10012000452001084D200108270201082702010887
:1001300027020108270201082702010827020108F7
:1001400027020108270201082702010827020108E7
:10015000552001082702010827020108270201088B
:1001600027020108270201082702010827020108C7
:1001700027020108B9A002083D2001080000000084
:100180002702010827020108E19A03082702010853
:100190002702010827020108270201082702010897
:1001A000BD650208B565020827020108270201089B
:1001B0002702010827020108270201082702010877
:1001C00027020108270201083B2101082702010834
:1001D000270201082702010827020108DD5703084A
:1001E0002702010827020108270201082702010847
:1001F000B365020827020108DFF80CD000F058FAB6
:10020000004800473D610408B01E022006488047B0
:1002100006480047FEE7FEE7FEE7FEE7FEE7FEE7EB
:10022000FEE7FEE7FEE7FEE7D9850308F9010108CE
:1002300040EA01039B0703D009E008C9121F08C068
:10024000042AFAD203E011F8013B00F8013B521EE8
:10025000F9D27047D2B201E000F8012B491EFBD25F
:1002600070470022F6E710B513460A4604461946C1
:10027000FFF7F0FF204610BD10B5044604E00B78F0
:1002800000F8013B03B1491C521EF8D2204610BDB4
:10029000421C10F8011B0029FBD1801A704703464D
:1002A00011F8012B00F8012B002AF9D118467047EC
:1002B00030B50B46014600202022012409E021FA36
:1002C00002F59D4205D303FA02F5491B04FA02F533
:1002D0002844151EA2F10102F1DC30BD2DE9F05FCA
:1002E0000546002092469B468846064681464024A5
:1002F0001BE0284641464746224600F0FAF953469D
:100300005A46C01A914110D311461846224600F0B1
:10031000E1F92D1A67EB01084F4622460120002122
:1003200000F0D8F917EB00094E41201EA4F101049A
:10033000DFDC484631462A464346BDE8F09F2DE9BA
:10034000FE4F804681EA0300C00F0C46009021F06A
:10035000004123F00045B8EB0200A94105D2404618
:10036000214690461C460B46024623F000401043AF
:1003700047D0270DC7F30A00C3F30A510290401A71
:10038000019040286BDAC3F3130040F4801B0098FF
:10039000924620B10023D2EB030A63EB0B0B0198CA
:1003A0005946C0F14002504600F094F906460D4609
:1003B00050465946019A00F0ACF910EB0800614133
:1003C000002487EA115284EAE7731A4340D0009A66
:1003D00062B3019A012A4FEA075215DC001B61EB58
:1003E00002014FF0004202EA0752CDE90042001C30
:1003F00041F5801132462B4600F0ACF903B0BDE860
:10040000F08F40462146F9E7001B61EB0201001C1A
:1004100041F5801300185B412018A2F5001747EB47
:10042000030140EAD570B6196D4111E06D084FEA3D
:10043000360645EAC0754FEA0752001B61EB020120
:10044000001C41F5801149084FEA30000019514164
:1004500032462B4603B0BDE8F04F00F06CB900986F
:10046000012240000023D0EB020263EBE07300980E
:1004700021464FEAE074B8EB000061EB0401E9E7C4
:1004800083F000435BE781F0004158E72DE9FE4F20
:1004900081EA030404F0004421F0004100944FF08D
:1004A000000B23F0004350EA01045ED052EA03043B
:1004B0005BD0C3F30A54C1F30A552C44A4F2F334BD
:1004C0000194A0FB0254C1F3130141F48011C3F362
:1004D000130343F4801301FB024400FB034E840A20
:1004E000970A44EA815447EA8357A4FB07680295B8
:1004F0008D0A05FB07854FEA932C04FB0C54270556
:10050000029D4FEA065847EA1637B5EB08056EEB31
:10051000070C870E920E47EA811742EA8312A7FB67
:100520000201B6EB0B0164EB00042B0D43EA0C3324
:100530005E1844EB1C50DA465146E7FB0201C5F356
:1005400013044FEA0B3343EA14534FEA0432019C7D
:1005500043EA0603A4F10C040294009CCDE900B424
:1005600000F0F8F803B0BDE8F08F00200146F9E78D
:100570002DE9F04D81EA030404F0004B21F0004521
:1005800014464FF0000A23F0004150EA050220D043
:1005900054EA01021DD0C5F30A570246C5F31303FE
:1005A000C1F31300C1F30A5640F4801543F48013DD
:1005B000A7EB0608101BD64608F2FD3873EB0500C2
:1005C00002D308F1010801E092185B41B8F1000F75
:1005D00003DA00200146BDE8F08D00204FF48011C1
:1005E000064684460EE0171B73EB050705D3121B66
:1005F00063EB050306434CEA010C49084FEA30005F
:1006000092185B4150EA0107EDD152EA030012D083
:1006100082EA040083EA0501084305D0101BAB41C0
:1006200006D20122002306E000224FF0004302E040
:100630006FF0010253101AEB06004CEB085110EB5F
:100640000A0041EB0B01BDE8F04D00F074B8C1F3B6
:100650000A52C1F3130140F2FF3341F480119A4270
:1006600002DA00200146704740F233439A42A2F278
:10067000334202DC524200F03CB800F02BB80000DC
:1006800030B5041E71F1000404DB4FF00044404219
:1006900064EB0101141E73F1000405DB1C464FF0EE
:1006A0000043524263EB0403994208BF904230BDBD
:1006B000064C074D06E0E06840F0010394E80700AF
:1006C00098471034AC42F6D3FFF79AFDA8C40D0842
:1006D000C8C40D08202A04DB203A00FA02F10020E9
:1006E00070479140C2F1200320FA03F31943904070
:1006F0007047202A04DB203A21FA02F000217047DB
:1007000021FA02F3D040C2F1200291400843194679
:100710007047202A06DBCB17203A41FA02F043EA61
:10072000E07306E041FA02F3D040C2F120029140AA
:1007300008431946704710B5141E73F1000408DA17
:10074000401C41F1000192185B411A4301D120F095
:10075000010010BD2DE9F04D92469B4611B1B1FA52
:1007600081F202E0B0FA80F220329046FFF7B2FF49
:1007700004460F4640EA0A0041EA0B0153465A4636
:10078000084313D0114653EA010019D0C8F14002C2
:100790005046FFF7AEFF05460E46504659464246C4
:1007A000FFF798FF084305D0012004E020463946B2
:1007B000BDE8F08D0020054346EAE0762C43374340
:1007C0000A986305E40AA0EB08000022FD0A44EA47
:1007D00047540A3002D500200146E9E70105101907
:1007E0006941DDE9084500196941BDE8F04DA2E71E
:1007F00070B58C1810F8015B15F0070301D110F8E3
:10080000013B2A1106D110F8012B03E010F8016B0F
:1008100001F8016B5B1EF9D12B0705D40023521E92
:100820000DD401F8013BFAE710F8013BCB1A921CFA
:1008300003E013F8015B01F8015B521EF9D5A142F8
:10084000D8D3002070BD0000014800887047000028
:100850001400002010B51648164908604FF44030C7
:100860004860002113488160016181610162416239
:10087000C1628162C1600121C161002101634161E6
:100880000DF0F6FC10B16FF0010010BD11200A4907
:1008900008600120486000208860C86005480DF0AD
:1008A00025FC10B14FF0FF30EFE70020EDE700002E
:1008B0000020014034260020C426002000B5064850
:1008C0000DF042FD28B103200449086004200449CA
:1008D0000870002000BD000034260020680E0020B3
:1008E0005D0E0020014800887047000016000020BF
:1008F00010B51648164908604FF440304860002192
:10090000134881600161816101624162C16281625B
:10091000C1600121C1610021016341610DF0A8FCAA
:1009200010B16FF0010010BD08200A4908600120D5
:10093000486000208860C86005480DF0D7FB10B102
:100940004FF0FF30EFE70020EDE70000002201400C
:100950007C260020C426002000B505480DF0F4FCDC
:1009600020B104200349086003490870002000BD3D
:100970007C260020680E00205D0E002008B5694628
:10098000002011F01FFF40B1BDF90010002901DA6D
:1009900000210091BDF9000008BD0C48006842F23A
:1009A0001071484340F6FF71B0FBF1F00849096847
:1009B00048434FF47A71B0FBF1F040F654314843AC
:1009C00042F21071B0FBF1F0E6E70000600E00208B
:1009D000580E002008B56946012011F0F3FE40B121
:1009E000BDF90010002901DA00210091BDF90000D5
:1009F00008BD0C48006842F21071484340F6FF7190
:100A0000B0FBF1F00849096848434FF47A71B0FB34
:100A1000F1F040F65431484342F21071B0FBF1F06E
:100A2000E6E70000640E0020580E002043490968E4
:100A300021F44031424AC2F804131146D1F804139C
:100A4000426811433D4A11600168496821F4807190
:100A50000268516001684A68016942EA012102683E
:100A600051600168496821F0407102685160016875
:100A7000496882681143026851600168896821F4FD
:100A800000610268916001688968C2681143026868
:100A900091600168896821F0706102689160016865
:100AA0008968826A1143026891600168896821F04F
:100AB00040510268916001688968C26A1143026806
:100AC00091600168896821F0020102689160016803
:100AD0008A68816942EA4101026891600168496857
:100AE00021F40061026851600168C96A21F4700153
:100AF0000268D1620168CA6A818B491E42EA0151CB
:100B00000268D1620168896821F40071026891600D
:100B100001688A68016B42EA4121026891600168BC
:100B2000896821F480610268916001688A6841697E
:100B300042EA81210268916070470000042301406D
:100B40000020014010B5084822F098F804460748F4
:100B5000604340F6FF71B0FBF1F00549B1FBF0F0E6
:100B60000449086010BD000098090020A08601001B
:100B7000000E2707580E002010B54E4800780128B7
:100B800007D14D480068806840F080404A490968B4
:100B9000886048480078032807D148480068806882
:100BA00040F08040454909688860424800784449DF
:100BB00008700846007804287AD2DFE800F00209BD
:100BC000303701203B49087064203E4908806FE0BF
:100BD0003C480088002805DD3A480088401E394915
:100BE000088005E001203849086004203149087078
:100BF00031480068006800F0020002280ED16FF052
:100C000012002D49096808602B480068C06C2F4904
:100C10000880FFF797FF02202649087048E003206C
:100C20002449087064202749088041E0254800884D
:100C3000002805DD23480088401E2249088005E081
:100C400002202149086004201A4908701B480068E6
:100C5000006800F00200022829D16FF01200174945
:100C60000968086015480068C06C194908802CF0B4
:100C700069FC2CF0D1FC00200E490870052011F011
:100C8000C3FDA0B15B2029F0E9FBFFF7A3FE04B28E
:100C9000204629F027FC2C2029F0E0FBFFF76EFE10
:100CA00004B2204629F01EFC5D2029F0D7FB00BFCE
:100CB00000BF10BD5D0E0020342600207C260020E1
:100CC0005C0E00205E0E0020680E00201400002044
:100CD000160000207CB505460C4601208DF800006A
:100CE0000020ADF802000848446035F09BF8064843
:100CF0004068001B019000208DF80000DDE9000134
:100D0000C5E900017CBD0000D42600207CB5054665
:100D10000E46144601208DF800000020ADF80200B8
:100D200008484460084A314635F042F805484068B2
:100D3000001B019000208DF80000DDE90001C5E9ED
:100D400000017CBDD42600200053070070B586B09A
:100D500005460E46144601208DF810000020ADF81F
:100D600012000F210CA24FF4C873CDE90206CDE9A1
:100D700000211A4621460A4835F062F800208DF815
:100D8000100007484068001B0590DDE90401C5E933
:100D9000000106B070BD000000000000000000006F
:100DA000D42600200A6810700A68521C0A60704736
:100DB00070B505460C462DB904F10801C8B201F022
:100DC00021FA70BD04F11701C8B201F01BFAF8E76F
:100DD0001CB5002007490871088048800846016852
:100DE00000918088ADF80400DDE9000102F0B2FD59
:100DF0001CBD0000761700202DE9FC4106460F4679
:100E000015461C46B4F5C87F01DD002402E0C4F598
:100E1000C87084B2012008490871084605804480E2
:100E2000016800918088ADF80400DDE9000102F05E
:100E300091FDBDE8FC810000761700200FB410B5CD
:100E4000829C2046E31704EBD363C3F34F11E317EF
:100E500004EBD3635B11A4EB43139AB205A850F8DB
:100E6000210001239340184018B1012010BC5DF807
:100E700014FB0020FAE730B50C46CD1701EBD56521
:100E8000C5F34F12CD1701EBD5656D11A1EB4515DB
:100E9000ABB200F10C0454F8224001259D402C40D7
:100EA0005CB100F10C0454F8225001249C402D1B2D
:100EB00000F10C0444F822500AE000F10C0454F84C
:100EC000225001249C40254400F10C0444F8225097
:100ED00030BD000010B50648007838B118F0F6FCB7
:100EE000FF2001F068F900200149087010BD0000E2
:100EF000C11600202DE9F04704460D4616461F4650
:100F0000DDE9099ADDF8208026806780A4F8048056
:100F1000A4F806902846FFF7BBF9608732222946DD
:100F200004F10800FFF7A8F901213D200155002038
:100F300084F83C00A08FE087C4F840A0BDE8F087AB
:100F40002DE9F0410446884615461E46069FB8F135
:100F5000000F2AD00020B4F90010A94212DCB4F925
:100F60000010B4F904201144A9420BDBB4F90210BB
:100F7000B14207DCB4F90210B4F906201144B142C1
:100F800000DB012038B194F83C1069B9012184F8E4
:100F90003E10397008E094F83C10012904D100217A
:100FA00084F83E10012139700CE094F83C000128CF
:100FB00008D1002084F83E0001203870206C08B170
:100FC000206C8047BDE8F0812DE9F0410446884659
:100FD00015463F20015D3D20005D814201D001208A
:100FE000287094F83E103D20005D814201D0012020
:100FF0002870E08FA0873D20005D002850D094F835
:101000003C00022806D150231A461946FF200BF057
:1010100085FE10E094F83C00012806D1FF231A4613
:10102000194618460BF07AFE05E096231A46194633
:10103000FF200BF073FEB4F806C01FFA8CF3B4F86F
:1010400004C01FFA8CF2B4F802C01FFA8CF1B4F895
:1010500000C01FFA8CF00BF06DFDB4F9040000EB3A
:10106000D071228802EB6101628F02EB4202A1EB98
:1010700042010EB2B4F9060000EBD071628802EBB7
:101080006101C91F0FB200231A461946FF200BF059
:1010900045FEB9B2B0B204F1080207F0E5FF00BFA7
:1010A000BDE8F08102463F208154012070470000D6
:1010B0000148006870470000700E00200748007863
:1010C000012803D005480078022804D100200349F4
:1010D0000870012070470020FCE70000740E00201B
:1010E00005480078022804D1002003490870012037
:1010F00070470020FCE70000740E00202DE9FE433D
:101100000E48006840F001000C490860084600687D
:1011100000F0010900240025032601274FF00008F4
:101120002B462246012106488DE8C0010BF042FF04
:1011300004481FF001FABDE8FE8300003038024089
:1011400000000240780E002002200149087070471C
:10115000740E00207047000010B5064800681FF0AC
:10116000B3F90446642C04D902481FF0E5F900F0F5
:10117000FDFE10BD780E002010B52DED048B0E483D
:1011800000681FF0A1F908EE100AB8EE480BB0EEA7
:10119000409B9FED0A0B89EE001BB0EE419B094876
:1011A00090ED000B30EE090B80ED000B02481FF0B4
:1011B000C3F9BDEC048B10BD7415002000000000C5
:1011C0000088C3407815002000B513F0FBFB002811
:1011D00006DC00200C49088002200C49087012E04F
:1011E0000B4814F09DF830B96820074908800320A7
:1011F0000649087007E00020034908800549088077
:1012000001200249087000BDBE140020BA1400205D
:10121000BC140020C014002010B518481FF08CF931
:10122000002426E016480078012820D115480088BF
:10123000B0F57A7F06DB6920134908800320104946
:10124000087010BD1148008811490E4A128821F813
:1012500012000E4814F02EF928B10A480088401CEC
:101260000849088003E0022005490870E9E7601C8E
:1012700084B2C82CD6DB00BFE3E70000C414002012
:10128000BA140020C0140020BE140020BC1400209A
:10129000D451012010B5012026F060FF10BD0000E0
:1012A0000148007870470000E00E00200148006807
:1012B00070470000800E0020014800687047000061
:1012C000940E002001480068704700008C0E00203A
:1012D0000148006870470000880E0020014800683F
:1012E00070470000840E002001480068704700002D
:1012F000980E00200148006870470000900E002002
:1013000001480068704700009C0E002001480068FA
:1013100070470000A80E00200148006870470000D8
:10132000A40E00200148006870470000AC0E0020A9
:101330000148006870470000B00E002001480068B6
:1013400070470000A00E00200148006870470000B0
:10135000B40E00200148008870470000D40E002021
:101360000148006870470000CC0E0020014800785A
:1013700070470000B80E00202DE9FE4300F060FF2A
:101380007C49086000F060FF7B4908604FF4C8703A
:101390007A49086008460068C821484377490860D0
:1013A0000846006800EB40000860084600688008B6
:1013B00008607348006840F0010071490860084601
:1013C000006800F001006F4908606D48001F006868
:1013D00040F480006A49091F08600846006800F46C
:1013E0008000684908606648001F006840F00100FE
:1013F0006349091F08600846006800F00100614960
:1014000008605F48001F006840F002005C49091F47
:1014100008600846006800F002005A490860584811
:10142000001F006840F004005549091F0860084685
:10143000006800F00400534908605148001F00682C
:1014400040F008004E49091F08600846006800F097
:1014500008004C4908604A48001F006840F010002E
:101460004749091F08600846006800F01000454918
:10147000086002274FF00008032400250D2643468C
:101480003A46502140488DE870000BF093FD4346EA
:101490003A4680213D488DE870000BF08BFD4346B5
:1014A0003A464FF43C613A488DE870000BF082FDFB
:1014B00043463A46482137488DE870000BF07AFDE4
:1014C00043463A46602134488DE870000BF072FDC7
:1014D000E02132480170780331490860E02130484A
:1014E000083880F8391338064FF0E021C1F80401BC
:1014F0002C48006820F001002A49086004E02A48CE
:101500000068401C284908602648006800F0010077
:101510000028F4D1254823490860202021491431AE
:10152000086040201F49203908604FF4706008604F
:10153000E0201F4908600846C06840F01000C860FD
:101540000846C06840F00800C8600846C06840F01F
:101550000400C8600846C06840F00200C860084641
:10156000C06840F00100C860002012490870BDE862
:10157000FE830000BC0E0020C00E0020C40E002020
:1015800034380240DC0E002000000240000402401B
:1015900000080240000C0240001002404EE400E04F
:1015A00008E100E0286402407C0E0020005406029E
:1015B00000000550B80E0020014800787047000078
:1015C000E50E00200021304A1069304A1268521C92
:1015D0002E4B1A6000F00402042A0ED12C4A126825
:1015E000521C2B4B1A6001210422274B5A61294AB5
:1015F000126822F00102274B1A6000F00202022A50
:101600000ED10121244A1268521C234B1A60022277
:101610001D4B5A611F4A126822F001021D4B1A60CD
:1016200000F01002102A08D11C4A1268521C1B4BF1
:101630001A6001211022144B5A6100F00802082A96
:101640000CD1114A926A164B1A60164A1268521C43
:10165000144B1A60012108220B4B5A6100F0010261
:1016600052B1114A1268521C0F4B1A60012101221B
:101670000E4B1A70044B5A6121B90D4A1268521C64
:101680000B4B1A607047000000000550800E0020D0
:10169000840E002028640240880E00208C0E00205A
:1016A000F40E0020900E0020940E0020B90E0020B1
:1016B000980E00200021454A1268521C434B1A60C4
:1016C000434A106800F40072BAB1414A28321268E5
:1016D00002F004028AB13E4A2832126822F0040263
:1016E0003B4B28331A605A15394B08331A600121D5
:1016F000384A1268521C374B1A6000F040027AB127
:10170000334A3C32126802F080024AB14022304B28
:1017100008331A60304A1268521C2F4B1A6001219C
:1017200000F4807282B12A4A2832126802F0020262
:1017300052B14FF48072264B08331A60274A126860
:10174000521C264B1A60012100F480621AB3204A11
:101750002832126802F00802EAB1214A1268521CCB
:101760001F4B1A6001218A02194B08331A60184A6C
:101770002832126802F480226AB9154A28321268A7
:1017800002F480723AB9124A2832126822F0080232
:101790000F4B28331A6000F400627AB10C4A2832E9
:1017A000126802F010024AB10E4A1268521C0D4B28
:1017B0001A600121CA02064B08331A6021B90A4A8D
:1017C0001268521C084B1A60704700009C0E0020E3
:1017D00000640240A00E0020A40E0020A80E0020ED
:1017E000AC0E0020B00E0020B40E00200748007898
:1017F000022809D106480088401C054908800420B9
:1018000002490870012070470020FCE7E00E00202C
:10181000D40E00200348006840F001000149086030
:10182000704700000000055010B50F48007818B14F
:101830000D480078022815D10C480068401C0B495F
:1018400008604FF4FA700A490880012006490870C0
:1018500000200849087026F081FC07481EF06CFE45
:10186000012010BD0020FCE7B80E0020D00E0020A3
:10187000C80E0020B90E0020D80E002003480068D2
:1018800020F0010001490860704700000000055089
:1018900010B518F055FD10BD10B514F0D7FE134863
:1018A0000078012820D11248007850B1002010495A
:1018B000087014F087FE00200C49087003F0C6FA87
:1018C00012E00C4800681EF0FFFDB0F5FA6F0BD96E
:1018D00009480068401C0849086002200349087054
:1018E000FFF7CCFF14F074FE10BD0000B80E00200E
:1018F000B90E0020D80E0020CC0E0020074800783A
:10190000022803D103200549087006E00348007847
:10191000012802D10020014908707047E00E002024
:101920000748007818B901200549087006E0044806
:101930000078032802D10220014908707047000096
:10194000E00E002030B587B004461EF025FA85B2BF
:1019500001A9284613F054FCC8B19DF8060010B93F
:101960000B20207015E09DF80A0010B10A202070AD
:101970000FE0BDF812004FF6FF71884202D1072038
:10198000207006E000202070012007B030BD082044
:1019900020700020F9E70000002004E00021034A45
:1019A0001154411C88B20228F8DB70470014002053
:1019B000002004E00021034A1154411C88B20B2886
:1019C000F8DB7047C427012038B50446002000909A
:1019D0008DF801406B460222502111F06FFB402030
:1019E0000149086038BD00001804024010B54FF4EA
:1019F00000720448016801F500710348FEF718FC05
:101A000010BD0000981400207461012010B54FF43F
:101A1000007204490448006800F50070FEF708FCF5
:101A200010BD000074610120981400202DE9F04FD2
:101A30000E46DDE909450021DDF82CB0BBF1000FB1
:101A400009D0BBF1010F08D0BBF1020F07D0BBF1E9
:101A5000040F08D105E0042107E0032105E002217D
:101A600003E0022101E0BDE8F08F00BF0027D0F8BD
:101A700004B00BF4704BC0F804B0D0F808B00BF40D
:101A8000704BC0F808B004F10B0B1FFA8BFC9344A9
:101A9000ABF1010B1FFA8BF805F10B0B1FFA8BF959
:101AA0009B44ABF1010B1FFA8BFA4CEA084BC0F8D0
:101AB00004B049EA0A4BC0F808B0D0F810B02BF0D7
:101AC000070BC0F810B0DDF82CB0C0F810B0BB4662
:101AD000C0F818B0D0F814B02BF0FF0BC0F814B059
:101AE0004FF0FF0BC0F814B0D0F81CB040F2077EE6
:101AF0002BEA0E0BC0F81CB040F2076BC0F81CB00C
:101B0000D0F828B0BB46C0F828B086620F46D0F89F
:101B10002CB00BF0E02BC0F82CB093460BFB07FB6E
:101B20000BF1030B02FB07FE4BEA0E4BC0F82CB087
:101B3000D0F830B06FF30A0BC0F830B0036300BFC9
:101B400091E700002DE9F34F83B00C4625462B2D7D
:101B50002DDA04EB4400174951F8306004EB4400DF
:101B600001EBC000078904EB440001EBC000B0F8B2
:101B70000A8004EB440001EBC00080891FFA80F961
:101B800004EB440001EBC000B0F812A004EB4400E9
:101B900001EBC000B0F814B043463A463146CDE9F7
:101BA00000ABCDF808900398FFF740FF00BF05B0E9
:101BB000BDE8F08F040F00202DE9F84307460E46DC
:101BC00015469846DDF820902B4632460221C80182
:101BD000CDF8008002F046F800204B463A4602213C
:101BE0000090C80102F03EF848488488002108307F
:101BF00000EB441001704548083000EB441047806A
:101C00004248083000EB441006714048083000EBB1
:101C10004410C580284627F086FC3C49083101EB7A
:101C200044110881C8213948083000EB4410418133
:101C30002946304606F03EFE01463448083000EBA7
:101C40004410017329463046FFF7B2F82F49083196
:101C500001EB44110861384613F0B0FA2B49083102
:101C600001EB441108752948083000EB4410007D51
:101C7000A0B1384612F0DCFE00EE100AB8EE400BC0
:101C8000234890ED001B20EE010BBCEEC00B1F485B
:101C9000083000EB441080ED060A05E000211B48E7
:101CA000083000EB4410816101211848083000EB36
:101CB0004410017715488088401C14498880022010
:101CC000C6EB061101EB4101124A02EB810105EB63
:101CD000450201F82200C6EB061000EB40000D495A
:101CE00001EB800005EB450100EB81004760C6EB8E
:101CF000061000EB4000074901EB800005EB4501B1
:101D000000EB8100C0F80880BDE8F883347301203F
:101D10006016002064780120F8B506460D460020C4
:101D20002B463246032100904FF4807001F09AFF59
:101D30002F4884880121083000EB441001700021F5
:101D40002B48083000EB441041802948083000EB54
:101D5000441006712648083000EB4410C580284620
:101D600027F0E1FB2249083101EB44110881C82129
:101D70001F48083000EB4410418100211C48083006
:101D800000EB441001751A48083000EB44108161E3
:101D90001748083000EB4410017715488088401C34
:101DA000134988800120C6EB061101EB4101114A5D
:101DB00002EB810105EB450201F822000020C6EB91
:101DC000061101EB41010B4A02EB810105EB4502D3
:101DD00001EB82014860C6EB061101EB4101054AA7
:101DE00002EB810105EB450201EB82018860F8BD41
:101DF0003473012064780120F8B506460D460020B2
:101E00002B46324604210090880101F02BFF2F4819
:101E100084880221083000EB4410017000212B4817
:101E2000083000EB441041802848083000EB441093
:101E300006712648083000EB4410C580284627F07C
:101E400072FB2249083101EB44110881C8211F4867
:101E5000083000EB4410418100211C48083000EBA1
:101E6000441001751948083000EB4410816117488F
:101E7000083000EB4410017714488088401C134957
:101E800088800020C6EB061101EB4101104A02EBED
:101E9000810105EB450201F82200C6EB061101EBBA
:101EA00041010B4A02EB810105EB450201EB820186
:101EB0004860C6EB061101EB4101054A02EB8101C6
:101EC00005EB450201EB82018860F8BD3473012007
:101ED0006478012070B506460D46204884880021AC
:101EE000083000EB441001701C48083000EB44102F
:101EF000468002211948083000EB4410017100218E
:101F00001648083000EB4410C1801448083000EB3C
:101F1000441001811148083000EB441041810F4802
:101F2000083000EB441001730C48083000EB4410FB
:101F30000561304613F042F901460848083000EBCD
:101F40004410017500210548083000EB441001776A
:101F500002488088401C0149888070BD347301208C
:101F60000020014988807047347301202F48007891
:101F700020B1012825D0022856D142E02C48006922
:101F800000F0010028B92B480088401C294908802E
:101F900002E00020274908802648008803280FDD3A
:101FA0002548007818B124480078032802D1012080
:101FB0002149087000201F49088001201B49087032
:101FC00032E01B48006900F0010028B11948008880
:101FD000401C1849088002E0002016490880154876
:101FE000008803280CDD0020124908801248007880
:101FF000012802D102201049087002200B49087004
:1020000012E00C480088401C0A49088008460088F5
:102010001E2808DD0648006900F0010018B1002004
:1020200008800249087000BF00BF70476E0E002094
:10203000000002406C0E0020740E002010B5FFF767
:10204000C1FA10BD10B521F0FBF910BD10B5FFF7B6
:1020500031FB10BD10B521F0A9FA10BD014608787A
:1020600010381823B0FBF3F20848805CC865032AD7
:1020700005D908686FF30900001D886503E008684A
:102080006FF309008865886D704700007070040860
:10209000014600208A6A8B69CBB932B1012A0DD082
:1020A000022A03D0032A10D10EE000BFCB6A03F04E
:1020B0008073B3F1807F00D1012007E0CB6AB3F1D8
:1020C000C07F00D1012001E000E000BF34E08B6957
:1020D000B3F5005F1AD132B1012A07D0022A03D02A
:1020E000032A11D10AE000BF01200EE0CB6A03F001
:1020F0008073B3F1807F00D1012006E0CB6AB3F199
:10210000C07F00D1012000E000BF15E032B1012AFC
:1021100005D0022A04D0032A0CD103E000BF00BF7F
:10212000012008E0CB6A03F08073B3F1807F00D117
:10213000012000E000BF00BF704710B500F0AAFC0E
:1021400010BD0146002205E0002301F51F7040F894
:102150002230521C0F2AF7D3002204E0002301F1A1
:102160001C008354521CB2F5007FF7D30020087086
:102170004870012088700020C1F8B80201230B7656
:1021800040238B7100234B7681F81C32012381F8A8
:102190001D32704710B50548007828B9002000F0BE
:1021A0000AF801200149087010BD0000C116002086
:1021B00010B50A9C10BD10B50446234651221521C6
:1021C000002034F0A5FA10BD0348406820F0080054
:1021D00001494860704700000070014003484068B2
:1021E00040F008000149486070470000007001405D
:1021F00000487047C084AFC1014840687047000084
:10220000040F002001460A462B2A06DA01EB4100A2
:10221000034B03EBC000406870470020FCE7000060
:10222000040F00200148D0F894037047040F0020E9
:1022300000487047C084AFC100487047C0D7B6C1DE
:102240004FF04040704700000048704780A903C02D
:102250000148008870470000FA0E002001480088FD
:1022600070470000FE0E0020014800887047000003
:10227000FC0E00200148008870470000000F00207D
:1022800070B505460C4626462B2E09DA04EB4400B1
:10229000074A02EBC00118222846FDF7C9FF70BDAE
:1022A000182204492846FDF7C3FF00BFF7E70000E6
:1022B000040F0020D4270020014800687047000068
:1022C0001068014001480068704700000C68014038
:1022D0000148006870470000186801400148006824
:1022E000704700000868014001480068704700001E
:1022F000146801400148006870470000AC68014064
:102300000148006870470000846801400148006887
:102310007047000094680140014800687047000061
:102320008868014001480068704700008C680140DF
:1023300001480068704700002C69014001480068AE
:1023400070470000046901400148006870470000C0
:1023500014690140014800687047000008690140A5
:1023600001480068704700000C690140014800788E
:10237000704700000D1300200148007870470000EE
:10238000020F0020FEB5FE48006840F00100FC4945
:1023900008600846006800F00107FA48006820F469
:1023A0004030F84908600846006840F48030086012
:1023B0000846806820F4403088600846806840F411
:1023C000003088600846406820F480704860084605
:1023D000C06820F44030C860E948006840F480607C
:1023E000E74908600846006800F48067E64800682E
:1023F00020F44040E44908600846006840F480400A
:102400000860E1480830006840F44040DE49083187
:102410000860081F006820F08000091F0860DA4883
:102420000C30006820F44040D7490C310860084661
:10243000006840F480400860D3481830006840F4D9
:102440000000D14918310860142034F0F5F8CE4866
:102450001830006840F08000CB4918310860142023
:1024600034F0EAF8C6481430006840F08060C4498F
:10247000143108600846006800F08067C0480C38D6
:10248000006840F08060BE490C390860084600686A
:1024900020F080600860BA48006840F40000B84945
:1024A00008600846006800F40007B5482038006856
:1024B00040F40000B249203908600846006820F462
:1024C00000000860AE481430006840F00060AC497D
:1024D000143108600846006800F00067A8480C380E
:1024E000006840F00060A6490C39086008460068A2
:1024F00020F000600860F021A44801704FF0807067
:10250000A3490860F021A248083880F85A134FF018
:1025100080604FF0E021C1F80801F0219B480A30AB
:10252000017004204FF0E021C1F80C0194483038CC
:10253000006820F08050924930390860002400E0A3
:10254000641C8F4830380068C0F340700028F7D111
:1025500090488B4958310860081D006800F44030ED
:10256000091D086086483038006840F08050844972
:102570003039086000E0641C814830380068C0F3DE
:1025800040700028F7D08448406820F00800824955
:1025900048608248006820F00100804908607F4858
:1025A0009C30006820F006007C499C3108607A4825
:1025B000006B20F00100784908630846006B20F0AA
:1025C000807008630846006B40F08070086300E08C
:1025D000641C7148C06800F480500028F8D06E4830
:1025E000006B6F4908406C4908630846006B42F66F
:1025F00090110843684908630846006B40F00100E9
:10260000086300E0641C6448C06800F4807000281F
:10261000F8D062489C30006840F006005F499C3169
:1026200008605E489030006820F003005B499031FC
:1026300008600846006840F0010008605748A03074
:10264000006820F003005549A03108600846006882
:1026500008605248001D006820F0FF004F49091D26
:1026600008600846006840F00400086005254D48F1
:1026700068434D49B0FBF1F64748806920F03F00C0
:102680004549886108468069304388610020434994
:10269000C031086000214148C43001603F483030FB
:1026A000006840F001003D49303108603A48006858
:1026B00020F00100384908600846006840F0010039
:1026C000086036480830006820F0030033490831BC
:1026D000086008460068086030481030006820F044
:1026E00007002E4910310860084600680860081F7E
:1026F000006820F00F00091F08600846006840F0DD
:10270000050008602448006820F00E002249086097
:102710000846006840F00A00086020486030006801
:102720006FF30F001D49603108600846006840F4EF
:10273000C87008601848006820F0F000164908606A
:1027400008460068086015486430006820F0010001
:102750001249643108600846006840F001000860D2
:102760000D48806840F001000B4988600846806889
:1027700040F0020088600948643000680B4917E0A7
:1027800030380240000002400028024058E400E0D7
:1027900008E100E00060035300700140046C014058
:1027A0000386FCFF00093D00A0252600FF80F0FE07
:1027B0000840AD49086008460068AC490843AA498A
:1027C00008600846006820F00200086008460068BB
:1027D0000860A748006820F07040A54908600846D6
:1027E00000680860A24810380068A2490840A04963
:1027F000103908600846006840F005100860081DA0
:1028000000689C4908409A490C39086008460068ED
:1028100040F00A100860081D006896490840944975
:102820000839086008460068934908439049083908
:102830000860081D00688F4908408D49091F08601D
:10284000084600688D4908438949091F086088487F
:102850001430006800F07F40854914310860002082
:10286000086083481C30006840F0040080491C3137
:1028700008600846006840F0020008607C48006874
:1028800040F001007A49086077486438006840F0F9
:1028900001007549643908607948406840F00800D3
:1028A000774948600A2033F0C7FE0523FE22152130
:1028B000002033F02DFF002305221521184633F0A8
:1028C00027FF0723FE221521002033F021FF4F238D
:1028D00007221521002033F01BFF0A23FE221521B9
:1028E000002033F015FF1B231C221521002033F09C
:1028F0000FFF0023FE221521184633F009FF0023A5
:1029000035221521184633F003FF0023112205213B
:10291000184633F0FDFE00200346024629210090B0
:1029200033F098FE40F2311033F086FE0023292266
:102930000521184633F0ECFE002033F07DFE002028
:102940008DF808008DF8090001208DF80A008F200D
:102950008DF80B0000208DF804008DF80500012093
:102960008DF806008F208DF8070046483623012297
:1029700039210090002033F06DFE02A82A230422A2
:1029800039210090002033F065FE01A82B2304229A
:1029900039210090002033F05DFE3B483A230122AC
:1029A00039210090002033F055FE962033F044FE8C
:1029B0002D480068354908402B49086008460068E2
:1029C00008600846006820F00200086008460068B9
:1029D000086025483C38006820F01F0022493C3937
:1029E00008600846006840F0040008602448406819
:1029F00040F0040022494860002000F0E9F81C483B
:102A00006C30006840F0010019496C310860012009
:102A100000F0EEF81648EC30006840F00100144970
:102A2000EC310860012012490C310860000218499D
:102A30008861012033F000FE012012E04FF0807128
:102A4000134A9161002100E0491CA629FCDB4FF4E8
:102A500080710F4A9161002100E0491CA629FCDB2E
:102A6000401C1628EADBFEBD686C0140007F0F00A9
:102A70001868014000F800F09A019A019F019F0137
:102A800000700140F80E0020F90E0020FF80F0FEDB
:102A9000000002403CB53948C46800253848008829
:102AA000401C3749088004F00100A0B13548008877
:102AB000401C344908800125012030490861002369
:102AC00034221521184633F023FE2C48406840F08C
:102AD00004002A49486004F00200002847D02A4830
:102AE0000088401C284908800125022023490861EC
:102AF0000846406820F0080048602448007800EB51
:102B00004000234901EBC000406822490860224888
:102B1000007800EB40001E4901EBC00040681D49F1
:102B2000803108601B488838006840F0010019496E
:102B3000883908601148406840F008000F49486033
:102B400000208DF804008DF8050001208DF80600A6
:102B50008F208DF8070001A82A2304223921009034
:102B6000002033F077FD01200C49087000BF25B923
:102B70000B480088401C0A4908803CBD0070014099
:102B8000FA0E0020FC0E0020FE0E00200C13002088
:102B9000040F0020AC6801400D130020030F00203B
:102BA000000F0020704770470348006840F00100A4
:102BB000014908607047000024680140034800682C
:102BC00040F001000149086070470000246801409E
:102BD00030B5044625462B2D05DA034804702146FE
:102BE0000248FEF7AFFF30BD0C130020846801409F
:102BF00030B5044625462B2D05DA034804702146DE
:102C00000248FEF79FFF30BD0D130020046901400C
:102C100070B50B4600EB4004104D55F8341000EB36
:102C2000400405EBC4042489544300EB40050B4EDB
:102C300006EBC5052D7C04FB051100EB4004354671
:102C400005EBC404247C03FB041100EB400405EBFA
:102C5000C4046160024C216070BD0000040F0020BC
:102C6000AC68014010B500EB40020B4B03EBC20215
:102C7000138900EB4002084C04EBC202127C534360
:102C800000EB400204EBC202127C4A43D21C42EA2F
:102C90000342024B1A6010BD040F0020B0680140CF
:102CA0002DE9F04100F10B0C1FFA8CF49444ACF1C7
:102CB000010C1FFA8CF501F10B0C1FFA8CF69C44E9
:102CC000ACF1010C1FFA8CF744EA054CDFF81480D4
:102CD000C8F800C046EA074C08F10408C8F800C06C
:102CE000BDE8F0818868014070B50B4600EB4004F8
:102CF000104D55F8341000EB400405EBC404248952
:102D0000544300EB40050B4E06EBC5052D7C04FB40
:102D1000051100EB4004354605EBC404247C03FB9D
:102D2000041100EB400405EBC4046160024C216017
:102D300070BD0000040F00202C69014010B500EBAD
:102D400040020B4B03EBC202138900EB4002084C1C
:102D500004EBC202127C534300EB400204EBC202BC
:102D6000127C4A43D21C42EA0342024B1A6010BD55
:102D7000040F0020306901402DE9F04100F10B0CF7
:102D80001FFA8CF49444ACF1010C1FFA8CF501F19C
:102D90000B0C1FFA8CF69C44ACF1010C1FFA8CF75B
:102DA00044EA054CDFF81480C8F800C046EA074C36
:102DB00008F10408C8F800C0BDE8F08108690140C6
:102DC0000948007868B901200749087000200749C0
:102DD00008700748406840F0040005494860012039
:102DE00070470020FCE70000020F0020030F0020C6
:102DF0000070014005480078012805D1044800789A
:102E000010B100200149087070470000020F002037
:102E1000030F00207FB542233C223121FF2009F01F
:102E20007DFF09F06FFF054600EBD5704410B82315
:102E30001A4640F22B2120B209F000FE01A811F041
:102E40005FF940F28110B623009001A807C807F08F
:102E50008FF97FBD1FB5022009F082FF01A811F094
:102E60004FF94FF4C370B623009001A807C807F0CC
:102E70007FF91FBD7FB542233C223121FF2009F09D
:102E80004DFF09F03FFF054600EBD5704410B82315
:102E90001A4640F22B2120B209F0D0FD01A811F012
:102EA0002FF940F28110B623009001A807C807F05F
:102EB0005FF97FBD70B504460D4616463246B7EE43
:102EC000000B2946204600F001F870BD2DE9F74FB0
:102ED0002DED020B8FB005468A46B0EE403BB7EEB3
:102EE000004BB4EEC43BF1EE10FA0BDBFE48007869
:102EF000FF2807DB1FFA8AF1A8B209F05DFF14B0C2
:102F0000BDE8F08FF948008800287DD1F8480468B2
:102F1000F8480068800000FB0A4404EB850413981D
:102F200010B1012871D118E0F34890F800B0F348CF
:102F300000780E90F24800780D90EB4800780C90E5
:102F40009DED0C4AB8EE444B24EE034BBCEEC44B53
:102F500014EE100AC0B20C90AAE0E678A77894F8B4
:102F6000018094F80090E048007804EE100AB8EE72
:102F7000444BB0EE441B21EE034BB0EE441B04EE79
:102F8000106AB8EE444B81EE045BB0EE451BDA48A4
:102F9000007804EE100AB8EE444BB0EE440B20EE7D
:102FA000014BB0EE440B04EE107AB8EE444BB0EE99
:102FB000442BB7EE004B34EE414B24EE024BB0EE07
:102FC000442B30EE024BBCEEC44B14EE100A00F062
:102FD000FF0BCA48007804EE100AB8EE444BB0EE7E
:102FE000440B20EE014BB0EE440B04EE108AB8EE19
:102FF000444BB0EE442BB7EE004B34EE414B24EE85
:10300000024BB0EE442B01E05CE050E030EE024BAE
:10301000BCEEC44B14EE100AC0B20E90B848007853
:1030200004EE100AB8EE444BB0EE440B20EE014B18
:10303000B0EE440B04EE109AB8EE444BB0EE442BC5
:10304000B7EE004B34EE414B24EE024BB0EE442B76
:1030500030EE024BBCEEC44B14EE100AC0B20D9021
:10306000A148007804EE100AB8EE444BB0EE440BD1
:1030700020EE034BB0EE440BB7EE004B34EE404B6A
:10308000B0EE440BC6F1010004EE100AB8EEC44BDA
:10309000B0EE442BB7EE004B00EE424BB0EE440BCB
:1030A000BCEEC04B14EE100AC0B20C9027E726E726
:1030B00000BF0C98E07084F802B00E9860700D9814
:1030C0002070EEE18948008801287CD18848046896
:1030D0008848006800EB400000FB0A4405EB45000F
:1030E0000444139810B1012809D109E082480078FE
:1030F000A07082480078607081480078207088E075
:10310000A77894F8018094F80090FF26764800781C
:1031100004EE100AB8EE444BB0EE441B21EE034B14
:10312000B0EE441B04EE106AB8EE444B81EE045B33
:10313000B0EE451B7048007804EE100AB8EE444B20
:10314000B0EE440B20EE014BB0EE440B04EE107ACF
:10315000B8EE444BB0EE442BB7EE004B34EE414B8F
:1031600024EE024BB0EE442B30EE024BBCEEC44BCF
:1031700014EE100A00F0FF0B6048007804EE100A0D
:10318000B8EE444BB0EE440B20EE014BB0EE440BD6
:1031900004EE108AB8EE444BB0EE442BB7EE004B71
:1031A00034EE414B24EE024BB0EE442B30EE024B9A
:1031B000BCEEC44B14EE100AC0B20E90504800781A
:1031C00004EE100A00E025E0B8EE444BB0EE440BEC
:1031D00020EE014BB0EE440B04EE109AB8EE444BD7
:1031E000B0EE442BB7EE004B34EE414B24EE024BD5
:1031F000B0EE442B30EE024BBCEEC44B14EE100A82
:10320000C0B20D9084F802B00E9860700D982070D6
:1032100000BF46E1354800880428FAD1DFF8D0C065
:10322000DCF80040DFF8CCC0DCF800C04FEA4C0C02
:103230000CFB0A4404EB4504DDF84CC0BCF1000F64
:1032400003D0BCF1010F7CD123E0DFF8B8C09CF8BB
:1032500000C04FEA2C10DFF8ACC09CF800C00CF0A6
:103260000F0104EE100AB8EE444B24EE034BBCEE03
:10327000C44B14EE10CA0CF0FF0001EB001C0CF064
:10328000FF036370DFF880C09CF800C084F800C0C2
:1032900005E194F801C0CDF824C094F800C0CDF841
:1032A00020C0DDF824C04FEA2C12DDF824C00CF059
:1032B0000F0CCDF81CC0DDF820C04FEA2C1CCDF857
:1032C00018C0DDF820C00CF00F0CCDF814C0DFF8EA
:1032D00034C09CF800C04FEA2C10DFF828C09CF8DE
:1032E00000C00CF00F0111E0E6130020E4130020F1
:1032F000D8130020DC130020E7130020E81300207F
:10330000E9130020EA130020EB130020DFF898C136
:103310009CF800C04FEA2C1CCDF82CC0DFF888C107
:103320009CF800C00CF00F0CCDF828C004EE100A79
:10333000B8EE444BB0EE441B21EE034BB0EE441B01
:1033400000E0ABE004EE102AB8EE444B81EE045BE3
:10335000B0EE451B04EE101AB8EE444BB0EE440B31
:1033600020EE014BB0EE440B9DED074AB8EE444B06
:10337000B0EE442BB7EE004B34EE414B24EE024B43
:10338000B0EE442B30EE024BBCEEC44B14EE10CA30
:103390000CF0FF0CCDF80CC09DED0B4AB8EE444B81
:1033A000B0EE440B20EE014BB0EE440B9DED064A0F
:1033B000B8EE444BB0EE442BB7EE004B34EE414B2D
:1033C00024EE024BB0EE442B30EE024BBCEEC44B6D
:1033D00014EE10CA0CF0FF0ECDF808E09DED0A4A7D
:1033E000B8EE444BB0EE440B20EE014BB0EE440B74
:1033F0009DED054AB8EE444BB0EE442BB7EE004BC2
:1034000034EE414B24EE024BB0EE442B30EE024B37
:10341000BCEEC44B14EE10CA0CF0FF0CCDF804C087
:1034200004EE100AB8EE444BB0EE440B20EE034B12
:10343000B0EE440BB7EE004B34EE404BB0EE440B15
:10344000C2F1010C04EE10CAB8EEC44BB0EE442B2E
:10345000B7EE004B00EE424BB0EE440B9FED134B2A
:1034600020EE044BBCEEC44B14EE10CA0CF0FF0E61
:10347000CDF810E0DDE903CE0CEB0E1C0CF0FF03E1
:10348000DDE901CE0CEB0E1C0CF0FF0CCDF800C0FA
:103490006370DDF800C084F800C000E02FE500BFD5
:1034A00000BF00BF2BE50000EB1300200000000070
:1034B00000E06F402DE9F04104460D4616460A2C07
:1034C0006AD2DFE804F0050F19232D37414B555F11
:1034D0000AF05EFD074600233A463146284608F0CA
:1034E000CBFB59E00AF058FD074600233A46314627
:1034F000284608F0C1FB4FE00AF052FD07460023C2
:103500003A463146284608F0B7FB45E00AF04CFD44
:10351000074600233A463146284608F0ADFB3BE01B
:103520000AF046FD074600233A463146284608F091
:10353000A3FB31E00AF040FD074600233A4631463E
:10354000284608F099FB27E00AF03AFD07460023D9
:103550003A463146284608F08FFB1DE00AF034FD5C
:10356000074600233A463146284608F085FB13E01B
:103570000AF02EFD074600233A463146284608F059
:103580007BFB09E00AF028FD074600233A46314656
:10359000284608F071FB00BF00BFBDE8F0817FB591
:1035A00042233C223121FF2009F0B8FB09F0AAFB9D
:1035B000054600EBD5704410B8231A466FF09A0107
:1035C00020B209F03BFA01A810F09AFD0F20B623B3
:1035D000009001A807C806F0CBFD7FBD7FB5422350
:1035E0003C223121FF2009F099FB09F08BFB0546B5
:1035F00000EBD5704410B8231A466FF09A0120B240
:1036000009F01CFA01A810F07BFD0F20B6230090F2
:1036100001A807C806F0ACFD7FBD10B525F036FF48
:1036200010BD000010B500241FE011480078A04232
:1036300019DD1048007820B90F4850F824100020F8
:1036400088470C480078012804D10B4850F8241012
:103650000120884707480078022804D1064850F81E
:10366000241002208847601C84B20A2CDDDB10BDC8
:10367000A2170020A0170020E808022070B5054618
:103680000E4600240BE007480078A04205DD0648FE
:1036900050F82420314628469047601C84B2032C01
:1036A000F1DB70BDCE1400207463012070B50546B7
:1036B00000240AE006480078A04204DD054850F8DE
:1036C000241028468847601C84B2032CF2DB70BDAE
:1036D0004C180020A80B022070B5054600240AE013
:1036E00006480078A04204DD054850F8241028461A
:1036F0008847601C84B2032CF2DB70BDB21C002032
:10370000B40B022070B5054600240AE00648007894
:10371000A04204DD054850F8241028468847601C64
:1037200084B2032CF2DB70BDBD1C0020C00C022053
:1037300070B5054600240AE006480078A04204DD82
:10374000054850F8241028468847601C84B2032C92
:10375000F2DB70BD0A1D0020F40C022070B5054696
:1037600000240AE006480078A04204DD054850F82D
:10377000241028468847601C84B2032CF2DB70BDFD
:10378000801D0020640D022070B5054600240AE06B
:1037900006480078A04204DD054850F82410284669
:1037A0008847601C84B2032CF2DB70BDA51D00208D
:1037B000880D022070B5054600240AE0064800780E
:1037C000A04204DD054850F8241028468847601CB4
:1037D00084B2032CF2DB70BDB11D0020940D0220D9
:1037E00070B5054600240AE006480078A04204DDD2
:1037F000054850F8241028468847601C84B2032CE2
:10380000F2DB70BDB71D00203C0E022070B50546EE
:1038100000240AE006480078A04204DD054850F87C
:10382000241028468847601C84B2032CF2DB70BD4C
:10383000CD1D0020680E022070B5054600240AE068
:1038400006480078A04204DD054850F824102846B8
:103850008847601C84B2032CF2DB70BDD11D0020B0
:10386000980E02207FB500240BE007480078A042A4
:1038700005DD064850F824509DE80F00A847601C5D
:1038800084B2032CF1DB7FBDCD1300204023012047
:103890002DE9FC47044604EB4410294901EB0010D4
:1038A000B0F9009004EB441001EB0010468804EBE3
:1038B000441001EB001090F80C7204EB441001EB83
:1038C0000010B0F80E8204EB441001EB00100079F8
:1038D000012820D100251BE01A480078A84215DDF8
:1038E00004EB4410DFF858A00AEB001000F58473D5
:1038F00004EB44100AEB0010CDE90078B0F80A227E
:10390000B1B2114850F825C04846E047681C85B25E
:10391000032DE1DB11E000250DE00C480078A84202
:1039200007DDB1B20A4850F825C043463A4648463A
:10393000E047681C85B2032DEFDBBDE8FC87000083
:103940007C28012035140020C851012034140020A7
:10395000BC51012013B582B000200090BDF80A30A0
:10396000BDF808209DF80C104FF4805000F07AF953
:1039700000240BE007480078A04205DD064850F817
:103980002420DDE902019047601C84B2032CF1DBA6
:103990001FBD00008F170020687F012070B505460D
:1039A0000E4600240BE007480078A04205DD0648DB
:1039B00050F82420314628469047601C84B2032CDE
:1039C000F1DB70BD03170020EC7C012070B50546CB
:1039D0000E4600240BE007480078A04205DD0648AB
:1039E00050F82420314628469047601C84B2032CAE
:1039F000F1DB70BD02170020E07C01202DE9F047CB
:103A000011F0D2FB054629F0E7F8012800D100E0CB
:103A10000020074610F0B0FB044610F0C7FF8246B6
:103A200011F030F8824501DA012000E000208146E3
:103A300010F0C8FF002801DD012000E0002006464C
:103A400015F03EFE032801D0012000E00020804652
:103A5000B8F1000F04D0022017494873887314E0AE
:103A600027B901201449887348730EE025B9012055
:103A700011498873487308E000200F4988730CB11E
:103A8000487302E001200C4948736DB186F00100D3
:103A90000949887486F00100C87384F00100087435
:103AA00084F00100487405E0012003498874C8735C
:103AB00008744874BDE8F087CC0C022010B50023D0
:103AC0001A461946184609F029F91E23C8224FF450
:103AD000B971642009F02EF810BD70B504460D468A
:103AE00000231A461946184609F018F9B3EE0C2BB4
:103AF00005F10E0000EE100AB8EEC01B04F10E0036
:103B000000EE100AB8EEC00B07F07EF970BD10B5DC
:103B1000022009F025F942233C223121FF2009F03F
:103B2000FDF80A2332224FF4C371B62009F002F8DF
:103B300010BD10B500231A461946184609F0EEF8D4
:103B40002823C822B421642008F0F4FF10BD10B56A
:103B500000231A461946184609F0E0F81E23C82229
:103B60004FF4B971642008F0E5FF10BD10B50023D3
:103B70001A461946184609F0D1F81E23C82200211A
:103B8000642008F0D7FF10BD10B500231A4619466F
:103B9000184609F0C3F81E23C8220021642008F04B
:103BA000C9FF10BD70B506460C461546304609F0F3
:103BB000D7F800231A461946184609F0AFF86423CF
:103BC0008C222946204608F0B5FF70BD10B50320B1
:103BD00009F0C6F800231A461946184609F09EF85F
:103BE00078231A468C21084608F0A4FF10BD10B5B2
:103BF000022009F0B5F842233C223121FF2009F0D0
:103C00008DF82D234FF48272FF21502008F092FF8F
:103C100010BD70B57E24204604EBD0714910C1F16F
:103C2000C805022009F09CF842233C223121FF20E4
:103C300009F074F804F10C02A91F88B20E2340F2B7
:103C4000611108F077FF70BD10B500231A461946C0
:103C5000184609F063F846231A46A521084608F0DD
:103C600069FF10BD2DE9F04104460D4616461F467A
:103C7000DDF818802A480068204000284ED02948E6
:103C8000007800284AD0284800681CF01DFC27490D
:103C9000098801EB4101264A42F831002348008897
:103CA00000EB4000114601EBC00044601F48008853
:103CB00000EB400001EBC00085601C48008800EB71
:103CC000400001EBC000C6601848008800EB4000CF
:103CD00001EBC00007611548008800EB400001EBD4
:103CE000C000C0F8148013480068401C11490860E7
:103CF0000E480088401C0D49088008460088B0F531
:103D00007A7F01DB002008800B480088B0F57A7FBD
:103D100004DA09480088401C07490880BDE8F081A2
:103D20001C1300202413002020130020181300204F
:103D3000EC270020141300201013002000207047EF
:103D400010B505481CF0F8FB002004490880044920
:103D500008600449088010BD2013002010130020C3
:103D6000141300201813002010B5044602481CF05C
:103D7000E3FB0248047010BD201300202413002030
:103D80002DE9F043D3B028F027FF012803D001200C
:103D900053B0BDE8F08300270026002477E03020F0
:103DA0008DF818013A208DF819016C208DF81A0150
:103DB0006F208DF81B0167208DF81C01B4F5803F42
:103DC00001DA302009E020140F2190FBF1F201FB11
:103DD000120085B2284604F013FD8DF81D01B4F5DC
:103DE000805F01DA302009E020130F2190FBF1F20F
:103DF00001FB120085B2284604F002FD8DF81E0179
:103E0000FF2C01DC302009E020120F2190FBF1F2A1
:103E100001FB120085B2284604F0F2FC8DF81F0168
:103E20000F2C01DC302009E020110F2190FBF1F272
:103E300001FB120085B2284604F0E2FC8DF8200157
:103E40000F2094FBF0F100FB114085B2284604F0EE
:103E5000D7FC8DF821012E208DF8220174208DF8D9
:103E6000230178208DF8240174208DF8250100208D
:103E70008DF8260146A828F0CBFD38B1641C701CD3
:103E800086B2B6F5803F02DB022081E70127002FD2
:103E900085D046A828F04AFE80463148006831495E
:103EA0000968CDE90010304803883048028830A105
:103EB00006A82FF045F906A8FCF7EAF905462946B9
:103EC00006A828F04FFE002536E005EB45003649F0
:103ED00001EBC000406905EB4501334A02EBC1012B
:103EE000096905EB4502304B03EBC202D26805EBD2
:103EF0004503DFF8B4C00CEBC3039B68CDE9013286
:103F0000CDE9031005EB4500614601EBC0004068B8
:103F1000009005EB450051F830302A4623A106A851
:103F20002FF00EF906A8FCF7B3F98146494606A81A
:103F300028F018FE681C85B20C4800888542C4DB56
:103F400022A106A82FF0FCF806A8FCF7A1F9054667
:103F5000294606A828F006FE28F0D4FD002017E721
:103F60001C1300201413002018130020101300202D
:103F70004576656E74204C6F672028636F756E748C
:103F80003D25642C2077726964783D25642C207768
:103F900072697465733D25642C2066696C74657262
:103FA0003D2564290A000000EC27002025642C2010
:103FB00025642C2025642C2025642C2025642C20AD
:103FC00025642C202564200A00000000456E642032
:103FD0006F66206C6F670A0010B50248008800F019
:103FE0000FF810BD1013002010B5642000F008F881
:103FF00010BD10B54FF4FA7000F002F810BD0000CB
:1040000010B504462848007800284AD1274800887F
:10401000A04218DC2548008800B2254908802348C2
:10402000008800B22349088020480088B0F57A7FD4
:1040300005DB2148008800B2204908801CE00020F0
:104040001E49088018E020B21949088020B2194999
:1040500008801948008816490988401A00B2174993
:1040600008800846B0F90000002805DA08460088F4
:1040700000F57A7000B20880114800781149087084
:1040800000F0C4F80120084908700A48B0F900207F
:104090000DA112482FF054F8104826F025FB0120FE
:1040A00010BD0020FCE700002513002010130020A5
:1040B0002A1300202C13002018130020281300209E
:1040C00024130020261300205B4C6F6744756D702D
:1040D0005374617274696E6725645D00AC8500205D
:1040E00010B50948007860B10020074908700748FA
:1040F000007808B100F084F805A026F0F5FA012058
:1041000010BD0020FCE7000025130020261300202E
:104110005B4C6F6744756D70436F6D706C65746553
:104120005D00000000B58DB025480078012845D11C
:104130002448B0F90000002802DCFFF7D1FF3DE081
:104140002148B0F9000000EB4000204A02EBC0011A
:10415000182207A8FCF76CF8DDE90923DDE90B104C
:10416000CDE90223CDE90410DDE90701CDE9000125
:104170001748B0F900001349B1F90010421A144869
:10418000B0F9003013A11A482EF0DAFF184826F0D3
:10419000ABFA0D480088401C00B20B490880084665
:1041A000B0F90000B0F57A7F01DB002008800548F7
:1041B0000088401E00B20349088000BF0DB000BD5A
:1041C000251300202C13002028130020EC270020AA
:1041D0002A1300205B25642C25642C25642C25647F
:1041E0002C25642C25642C25642C25645D0000009E
:1041F000AC85002001490860704700001C130020B6
:104200000120014908707047241300200020014953
:10421000087070472413002010B5FFF783FF10BD0E
:104220000F4909784E3903EE101AB8EEC33BB0EED1
:10423000430B9FED0C3B80EE034BB0EE441B9FED18
:104240000B3B31EE033BB0EE432BB6EE003B32EEC0
:10425000033BBCEEC33B13EE101A88B2704700005C
:104260005C13002033333333333303C000000000CA
:1042700000405A4001480068704700005813002071
:1042800001480068704700005413002000B5002268
:1042900000BF1E48006840F002001C490860084644
:1042A000006800F002021A48006820F440501849E3
:1042B00008600846006840F480500860081D0068E7
:1042C00020F04000091D0860081D006820F44050DF
:1042D000091D08600846006840F400500860081D89
:1042E000006820F44050091D08600846006840F44A
:1042F0008050086006482030006820F07060044953
:104300002031086000F066F800BD0000303802403F
:104310000004024070B52DED068B0446A4F169003F
:1043200000EE100AB8EEC00BB0EE409B9FED180BEC
:1043300029EE000BB0EE40AB9FED170B3AEE000BF1
:10434000B0EE408BB3EE040BB4EEC08BF1EE10FA7E
:1043500003D2B3EE040BB0EE408B9FED110BB4EE25
:10436000C08BF1EE10FA03DD9FED0D0BB0EE408B2C
:10437000B6EE000B38EE000BBCEEC00B10EE100AD0
:1043800085B2E8B200F010F8BDEC068B70BD0000FD
:1043900033333333333303C0000000000080534015
:1043A0000000000000206B4010B50446142C00DA19
:1043B0001424D92C00DDD924044804700448007862
:1043C00018B102480078FDF7FFFA10BD5C13002019
:1043D000501300204FF48000024908600020024979
:1043E00008707047180402405013002010B50448AC
:1043F0000078FDF7E9FA01200249087010BD0000BD
:104400005C130020501300202DE9F84F82460C4623
:1044100016461F461648007808F0A2FC4FF0010827
:104420004FF00009E019801E05B21AE0721C91B22B
:10443000A8B26A4608F0FAFB9DF80000FF280CD1EC
:104440009DF80100E62808D19DF80200E62804D175
:104450009DF80300E62800D1C1444FEA4808681ED1
:1044600005B2601C8542E1DA4846BDE8F88F0000DD
:104470004817002001480078704700001E180020EF
:104480001CB5FE480078012806D0FD480068019060
:10449000BDF8041008461CBDFA480068002879D011
:1044A000002003460090F74804210268C801FFF786
:1044B000D9FBF5480068B0F80802C0F308000028EE
:1044C00069D1F1480068D0F8000290F80202401E5D
:1044D000ED490968D1F8081200EA5120EB4908704B
:1044E0000846007800287DD1E7480068D0F8080227
:1044F00090B9E5480068D0F81002E5490860084620
:10450000006828BBE0490968D1F80002002130F0BA
:10451000CDF8DF4908601BE0DB480068D0F82402D2
:1045200050B1D9480068D0F80812D748006830F078
:1045300085F8D74908600BE0D34A1268D2F8141204
:10454000D14A1268D2F8000230F0B0F8D0490860C1
:10455000CF48006838B90020CA4908600090BDF80B
:104560000010084697E7CA480068012814D10220C5
:10457000C549096881F807020120C6490880022060
:10458000BE490870BE48001D00680090BDF80010CC
:10459000084680E7AEE148E1BD480068401C88B9A4
:1045A0000120B949096881F807020220B949088049
:1045B000B2490870B248083000680090BDF8001099
:1045C000084668E7B2480068AF490968C1F81402B4
:1045D000AD480068D0F8100220B9AD480068AA497B
:1045E000096800E001E0C1F81002A748006890F8EF
:1045F000060200F0400070B3002003460246052189
:1046000000904FF40070FFF72DFB9F490968D1F827
:1046100018229D490968D1F8001291F8010201237E
:104620009949096830F0CAFB0446ACB101209649AB
:10463000096881F8070203209649088002208F4903
:1046400008708F480C30006800908DF80140BDF86C
:10465000001008461FE70AE08B48006890F8060241
:1046600020F040008849096881F8060200BF864AA8
:104670001268D2F81412844A1268D2F8000230F09C
:1046800005F8854908600846006890B902207E490F
:10469000096881F8070203207E49088002207749D3
:1046A00008707748103000680090BDF80010084688
:1046B000F1E6794800687549097808447649086048
:1046C00070480068400A754908600846006800287C
:1046D00071D06E480078096808446B490968D1F8C0
:1046E000001291F8021288420AD967480068D0F88F
:1046F000000290F8020265490978401A674908608B
:10470000002003460246062100904FF40070FFF798
:10471000A9FA5D490968D1F8001291F801025F49D0
:104720000B685D490A685E49096830F047FB04463A
:10473000A4B101205449096881F8070203205549B2
:10474000088002204D4908704D48143000680090E0
:104750008DF80140BDF8001008469CE64A48006804
:10476000D0F818024C490968401A4C490968884237
:104770001AD245480068D0F81802474A1268801AD1
:10478000474A126802EB40214FF400723E4800682D
:1047900031F01FFF3C48006890F8060220F040000E
:1047A0003949096881F806023C48006840023D49E1
:1047B000086080E0FFE734480068D0F81802364906
:1047C000096888422BD030480068D0F808022E498A
:1047D0000968D1F80C12884220D22B490968D1F817
:1047E000001291F8010201232B490A682649096841
:1047F00030F080FA90B101202349096881F807025E
:1048000003202449088002201C4908701C481830E5
:1048100000680090BDF8001008463CE600BF1E4846
:10482000006819490968C1F8180217480068B0F80B
:104830000802C0F30800C0F500701A490860084675
:10484000006810490968884203D90E480068154974
:1048500008600D490968B1F80812C1F308010A4A55
:10486000126888180F490A680D49096831F0B1FECD
:104870000548006890F8060216E000001E180020A7
:104880000871040824180020281800202C18002083
:104890003018002020180020341800203C18002078
:1048A000401800203818002040F0400028490968CE
:1048B00081F8060200BF27480068274909680844B4
:1048C0002449086022480068D0F808022249096893
:1048D00008441F490968C1F80802204800681E49B9
:1048E0000968401A1D49086000200190BDF80410B5
:1048F0000846D0E516480068D0F80802144909684F
:10490000D1F80C12884207D911480068D0F8080283
:104910000F490968C1F80C020D48006890F80602BA
:1049200040F020000A49096881F806020020034689
:104930000246032100904FF40070FFF793F9002026
:10494000074908700190BDF804100846A3E500006F
:1049500028180020401800203818002024180020B3
:104960001E1800202DE9FC4104460D4616461F4640
:104970003648007838B1364800680190BDF8041018
:104980000846BDE8FC8133480460334806600020D7
:10499000034600903048002102684FF40070FFF792
:1049A00061F92E4805602E48076000202C490968EF
:1049B00008602848006832F086F88046B8F1000F99
:1049C00009D02348001D006800908DF80180BDF8D3
:1049D00000100846D5E71F48006890F8070268B144
:1049E0001B480830006800901A48006890F80702D9
:1049F0008DF80100BDF800100846C2E715480068B0
:104A000090F8060200F0020038B911480C30006836
:104A10000090BDF800100846B3E70E480068D0F8D3
:104A200008020D49096808440A490968D1F80812C2
:104A3000884202D20020084908600120034908701A
:104A400000200190BDF8041008469AE71E180020C7
:104A5000F8700408281800202418002040180020AE
:104A60004418002010B50A48007880B10948006851
:104A7000382803D900200649087008E0054908785D
:104A800000F090FA03480068401C0249086010BD1D
:104A90003C130020381300200148008870470000B4
:104AA0004013002001480088704700004213002096
:104AB00001480088704700003E130020014800882C
:104AC00070470000441300202DE9FE43484B494A3B
:104AD0004FF40051484821F031FD484B484A4FF40B
:104AE0000051484821F018FD4FF000094648006881
:104AF00040F02000444908600846006800F02009A2
:104B000041486030006820F400503F49603108603F
:104B10000846006840F4805008603B481030006848
:104B200040F080403849103108600846006800F0C5
:104B3000804902240025032600274FF008082B4651
:104B40002246C02131488DE8C00108F033FA6004E4
:104B50002F4908602F48006820F001002D490860A7
:104B60004FF4D9602C4908602B480838006820F4BD
:104B700080402949083908600846006820F4006030
:104B80000860081D006820F02000091D0860084624
:104B9000006820F0080008600846006820F0020065
:104BA00008601D480C38006840F001001A490C39B3
:104BB00008600846006840F00C000860084600687D
:104BC00040F0400008600846006840F0200008609F
:104BD0000846006840F4807008600F48001F0068B5
:104BE00040F001000C49091F0860BDE8FE83000089
:104BF000CCA60020CC860020AC860020CCE600208D
:104C0000CCC60020BC860020303802400014024090
:104C100008E100E0005000400C78004070470000C0
:104C200038B52D480088401C2B4908802B48046863
:104C300004F0010040B101202849091D08602848FE
:104C40000088401C2649088004F0020040B1022080
:104C50002249091D086023480088401C214908801A
:104C600004F0040040B104201C49091D08601E48DE
:104C70000088401C1C49088004F0080040B108204E
:104C80001649091D086019480088401C174908800A
:104C900004F0200040B1114808300068C5B2294630
:104CA000134821F0A9FC00BF04F0400090B140205F
:104CB0000A49091D086069460E4821F06BFC28B1BD
:104CC0009DF8000005490C31086002E000200A4907
:104CD000087000BF38BD0000361300201C7800406B
:104CE00046130020481300204A1300204C130020D4
:104CF000AC860020BC8600203413002030B585B07F
:104D0000044622460BA168462EF01AFA6846FBF7C5
:104D1000BFFA0546A9B2684624F0FCFE7B2025F0C8
:104D20009DFBA9B2684625F0AFFB7D2025F096FBE0
:104D300005B030BD5220253032780D0001200349E6
:104D40000870002002490860704700003C130020F2
:104D5000381300203EB506A168462EF0F1F96846EA
:104D6000FBF796FA0446A1B2684624F0D3FE3EBD96
:104D7000572046462033310D000000003EB506A105
:104D800068462EF0DDF96846FBF782FA0446A1B2C8
:104D9000684624F0BFFE3EBD522030300D000000BA
:104DA0003EB506A168462EF0CBF96846FBF770FACF
:104DB0000446A1B2684624F0ADFE3EBD5720303710
:104DC0002032360D0000000070B586B004460D4656
:104DD0002B46224606A101A82EF0B2F901A8FBF746
:104DE00057FA0646B1B201A824F094FE06B070BD91
:104DF00057202530327820253032780D0000000011
:104E000070B586B004460D462B4622460BA101A87C
:104E10002EF096F901A8FBF73BFA0646B1B201A8BD
:104E200024F078FE7B2025F019FBB1B201A825F013
:104E30002BFB7D2025F012FB06B070BD57202530DE
:104E4000327820253032780D000000000120014921
:104E5000087070476D1300202DE9FE431348006869
:104E600040F00100114908600846006800F001099F
:104E700001240025032601274FF000082B46224677
:104E800006210B488DE8C00108F094F800F028F8DE
:104E900000F030F807481BF04FFB0020064908706F
:104EA000012006490870BDE8FE830000303802404A
:104EB00000000240641300206C13002060130020E7
:104EC00001200149087070476C13002003484069B5
:104ED00040F00200014948617047000000000240B4
:104EE0000348406920F00200014948617047000012
:104EF000000002400348406940F004000149486155
:104F000070470000000002400348406920F00400A0
:104F100001494861704700000000024010B51C487C
:104F20000078062832D2DFE800F003040B182230A4
:104F30002CE01848007810B102201549087025E0CF
:104F4000154800681BF0C0FAB0F57A7F04D9FFF766
:104F5000BDFF03200E49087018E01048007828B102
:104F60000F481BF0E9FA0420094908700EE00C48CC
:104F700000681BF0A9FA41F28831884204D9FFF792
:104F8000DDFE05200249087000E000BF00BF10BD33
:104F9000601300206C130020641300206D130020A8
:104FA0006813002010B50446392C6ED2DFE804F0F7
:104FB0001D22272C31363B40454A4F54595E6368C9
:104FC0006E73787D82878C91969BA0A5AAAFB4B9A9
:104FD000BEC3C8CDD2D7DCF3F8FDEFEEEDECEBEAC3
:104FE000E9E8E7E6E5E4E3E2E10031210020FFF74C
:104FF000EBFE2BE150210220FFF7E6FE26E16021C7
:105000000F20FFF7E1FE21E161211120FFF7DCFE17
:105010001CE162213220FFF7D7FE17E163217D20DA
:10502000FFF7D2FE12E164210846FFF7CDFE0DE145
:1050300065217D20FFF7C8FE08E16621E620FFF725
:10504000C3FE03E167210220FFF7BEFEFEE07021F0
:105050000120FFF7B9FEF9E071210120FFF7B4FE4E
:10506000F4E072210220FFF7AFFEEFE0732123206E
:10507000FFF7AAFEEAE000210846FFF7A5FEE5E0FB
:1050800001213220FFF7A0FEE0E0DEE00221072050
:10509000FFF79AFEDAE00321D020FFF795FED5E076
:1050A00004210520FFF790FED0E00521DC20FFF76A
:1050B0008BFECBE006210520FFF786FEC6E0072128
:1050C000DC20FFF781FEC1E008210520FFF77CFE10
:1050D000BCE00921DC20FFF777FEB7E00A210020C1
:1050E000FFF772FEB2E00B210420FFF76DFEADE08A
:1050F0000C210020FFF768FEA8E00D210020FFF73B
:1051000063FEA3E00E210020FFF75EFE9EE00F216C
:105110000020FFF759FE99E010210020FFF754FE10
:1051200094E011210020FFF74FFE8FE012210020B4
:10513000FFF74AFE8AE013210020FFF745FE85E0D5
:1051400014210020FFF740FE80E015210020FFF72A
:105150003BFE7BE016210020FFF736FE76E01721AC
:105160000020FFF731FE71E018210020FFF72CFE30
:105170006CE065E05FE059E053E04DE047E041E07E
:105180003BE035E02FE029E023E01DE017E011E0EF
:105190000BE005E0FFE719210020FFF715FE55E0C1
:1051A0001A210420FFF710FE50E01B210020FFF71A
:1051B0000BFE4BE01C210020FFF706FE46E01D2100
:1051C0000020FFF701FE41E01E210020FFF7FCFD5B
:1051D0003CE01F210020FFF7F7FD37E020210420ED
:1051E000FFF7F2FD32E021210020FFF7EDFD2DE079
:1051F00022210020FFF7E8FD28E023210020FFF70F
:10520000E3FD23E024210020FFF7DEFD1EE0252141
:105210000120FFF7D9FD19E026210520FFF7D4FD75
:1052200014E027210020FFF7CFFD0FE02821002008
:10523000FFF7CAFD0AE0FE214C20FFF7C5FD05E09F
:10524000FF210020FFF7C0FD00E000BF00BF10BD40
:1052500010B52A2001F06AFB10BD10B52C2001F01A
:1052600065FB10BD10B52B2001F060FB10BD10B523
:10527000252001F05BFB10BD10B5262001F056FB88
:1052800010BD10B5282001F051FB10BD10B504462B
:1052900002480480292001F049FB10BDB013002012
:1052A00010B5272001F042FB10BD00002DE9F041B0
:1052B0002DED028B8EB005460C462CB9FA482946D6
:1052C000026800200DF0B4FA44B9002003460090B3
:1052D000F548294602680120FEF7C4FC032C0AD1D8
:1052E000F248006840F28A21884204D2EF48006800
:1052F000401CEE490860284611F04CF9B8BB0FF08D
:10530000FBFB34280CD10FF057FB0B2101EB0020E5
:10531000E54908603D200EB0BDEC028BBDE8F08190
:1053200017F064F82E2808D117F05AF80C2101EB79
:105330000020DD4908603D20EDE71AF053FD3328D9
:1053400008D11AF01DFD0D2101EB0020D64908609F
:105350003D20E0E718F0C4F9192809D118F0A8F9A0
:105360000E2101EB0020D04908603D20D3E7FFE784
:10537000412D81F07682DFE815F041004700800082
:10538000A100DF00100132014D016401D201E601EC
:1053900012021C021D02540255028D0205034A032B
:1053A000FC030E042D045E0469048104F0019F04D3
:1053B000D404DD04EE041E0523054A0553056405E7
:1053C00094059E05D505C905F505730658075907C7
:1053D000DD07FD0760084A08AD08C808DD08F208C7
:1053E0000D090E0949098C09CF0980068106960628
:1053F000B5064C07E609E709E8091F0A042C01D1A4
:10540000012088E7284686E75CB9012024F02AFEBF
:10541000022017F007F814F071F9A5481BF08CF87A
:1054200029E0032C27D1A24800681BF04DF841F277
:105430008831884201D9012000E00020074614F09D
:105440003FF9012801D0012000E0002006460EB1FE
:10545000FFF736FD17B10EB102205CE794480068F3
:105460001BF032F89349884204D90F208E49086016
:105470003D2050E700BF28464DE78CB924F057FB8C
:105480008D481BF059F800201EF026FB064636B169
:10549000102000EB0620844908603D203BE70BE02C
:1054A000032C09D1844800681BF00EF840F6C411A3
:1054B000884201D903202EE728462CE764B910F072
:1054C00019FA0646012E06D0112000EB0620764977
:1054D00008603D201FE72DE0032C2BD10FF00CFBC3
:1054E00006460C2E01D1042015E70B2E08D10FF033
:1054F00063FA6D49086001207049087004200AE7CA
:10550000342E08D10FF058FA122101EB0020664921
:1055100008603D20FFE6664800681AF0D5FF68493C
:10552000884206D9132000EB06205F4908603D2021
:10553000F1E600BF2846EEE654B900206149087044
:1055400027F0FCFEFEF752FF64205F49087022E05E
:10555000032C20D15C480078401E5B49087014F091
:10556000AFF8022801D0012000E00020064656488E
:10557000007800280EDC2DF0EBFC01205349087068
:105580001EB95349087014F095F80120514908706C
:105590000620C0E600BF2846BDE61CB94E481AF0FA
:1055A000CBFF1AE0032C18D14CF250361AF044FC11
:1055B00008B90620AFE6484800681AF085FF4CF2AB
:1055C0005031884208D91AF00DFC142101EB00205B
:1055D000354908603D209EE600BF28469BE6BCB1E9
:1055E000032C15D1324800681AF06EFF46F2A8115C
:1055F00088420DD9FCF794F93048007808B10720AB
:1056000089E60FF0F7FD08B1092084E60A2082E65A
:10561000284680E624B92448006824F05AFD0EE0AC
:105620000E2C08D120480068152101EB00201E49EE
:1056300008603D206FE60D2C01D108206BE628465E
:1056400069E6D4B925481AF077FF10F0A5F90646A7
:10565000022E08D10FF050FA162101EB002012495A
:1056600008603D2057E6012E06D0172000EB0620EB
:105670000D4908603D204EE64FE0032C4DD10FF060
:105680003BFA06460C2E03D118F0F3F90A2042E645
:10569000342E25D10FF090F9182101EB002002499A
:1056A00008603D2037E600007413002080130020BE
:1056B0008C130020A086010094130020A01300206A
:1056C000400D0300A11300209C1300209E13002016
:1056D0009F1300209D130020A41300208813002096
:1056E0000B2E08D10FF068F9192101EB0020F849C1
:1056F00008603D200FE6F74800681AF0E5FE4CF21E
:105700005031884208D90FF0F7F91A2101EB002037
:10571000EF4908603D20FEE500BF2846FBE52CB9B7
:10572000EDA2F1A1F3A024F0C3FC0AE00F2C01D1FB
:105730000A20F0E5032C04D1FBF7D2FC08B10A20C3
:10574000E9E52846E7E534B9EC48007808B11820C7
:10575000E1E50B20DFE52846DDE574B927F0EEFD35
:105760000020E7490870DB481AF0E6FE032024F029
:1057700079FC022016F056FE0FE0032C0DD1D5481F
:1057800000681AF0A1FE064642F21070864203D964
:10579000192D01D10B20BEE500BF2846BBE534B969
:1057A0000EF094FD08B11220B5E51020B3E52846AF
:1057B000B1E500BFBCB9D3481AF0BEFE0C2D04D130
:1057C0000EF084FD30B91020A5E50EF07FFD08B184
:1057D0001220A0E50FF0E8FC08B30C2D01D10E203B
:1057E00099E50F2097E5032C19D10FF0DDFC28B1C6
:1057F0000C2D01D10E208EE50F208CE5C1480068EC
:105800001AF062FE44F62061884208D90FF074F95C
:105810003D2101EB0020AE4908603D207BE5284694
:1058200079E500BFDCB90F2D01D1012100E0002195
:1058300008460EF055FD0EF027FD0646012E0AD053
:10584000002033461722092100904FF48030FEF7E4
:1058500009FA0B205FE5AB481AF06EFE18E0032C46
:1058600016D10FF049F90C2801D10B2053E5A548BA
:1058700000681AF029FE44F62061884208D90FF02A
:105880003BF93E2101EB0020914908603D2042E5B3
:10589000284640E57CB9FEF7A9FD21F0BBFD0EF0DE
:1058A000E3FC064628F06CFF032024F0DBFB042019
:1058B00016F0B8FD64E0132C01D11A202BE5142C4E
:1058C00004D10020904908701F2024E5172C01D135
:1058D0000D2020E5262C01D10D201CE5032C33D111
:1058E00013F0EEFE052803D013F0EAFE062817D1C8
:1058F00021F09EFD10B121F079FD04E024F0AEFA14
:1059000008B124F012FC13F0DBFE052802D00628B3
:1059100004D101E01720FEE41820FCE400BF00BF22
:10592000FBF7CCFB60B321F083FD10B121F05EFDED
:1059300026E024F093FA10B124F0F7FB20E0FBF707
:105940003BFEE8B91120E6E4272C01D11120E2E466
:10595000122C01D12620DEE4212C01D12620DAE40C
:10596000242C01D14020D6E42B2C01D12A20D2E4D2
:105970002C2C01D12920CEE42D2C01D10120CAE408
:105980002846C8E474B921F03BFD52481AF0D4FD12
:1059900002224FF47A7141F2883024F044F916F073
:1059A0003BFD32E0032C30D141F27077494800686A
:1059B0001AF08AFD06463846864225D916F026FD9D
:1059C00020B10120514908701020A4E416F00EFD0A
:1059D0002E2808D116F004FD1B2101EB00203C49C4
:1059E00008603D2097E43B4800681AF06DFD4CF2DA
:1059F0005031884208D916F0F9FC1C2101EB002037
:105A0000334908603D2086E400BF284683E494B90A
:105A100000203F49087021F0FDFCFEF7E7FC0EF086
:105A200023FC064628F0ACFE032024F01BFB0420D8
:105A300016F0F8FC9BE0132C01D11A206BE4142C17
:105A400004D10020304908701F2064E4122C01D1D9
:105A5000262060E4212C01D126205CE4172C01D102
:105A60000C2058E4252C01D10C2054E4282C04D11E
:105A700000202849087013204DE4292C08D101206A
:105A8000244908702448008824490880132042E4EF
:105A90002B2C01D12A203EE42C2C01D129203AE4E0
:105AA000242C01D1402036E42D2C01D1012032E4F8
:105AB000032C5CD113F004FE052803D013F000FE84
:105AC000062840D121F0B4FC50B321F08FFC2DE02A
:105AD000741300208813002054415020544F204359
:105AE0004F4E54494E554500302E30312E30393509
:105AF0000000000056455253494F4E009F130020AE
:105B0000A1130020AC130020A91300209D13002036
:105B1000A8130020B4130020B0130020B2130020FB
:105B2000FFE724F09BF908B124F0FFFA13F0C8FD59
:105B3000052802D0062804D101E0172009E4182026
:105B400007E400BF00BFFBF7B9FA20B121F070FCF9
:105B500010B121F04BFC0AE024F080F910B124F0E0
:105B6000E4FA04E0FBF728FD08B9152049E42846CB
:105B700047E474B921F044FC032016F053FC0320E1
:105B800024F070FA0FF010FB08B1152039E414204E
:105B900037E4284635E41CB9F7481AF0CDFC17E085
:105BA000032C15D10FF000FB08B1152029E4F248B1
:105BB00000681AF089FC41F28831884208D90EF059
:105BC0009BFF3C2101EB0020EC4908603D2018E4DC
:105BD000284616E41CB9052016F024FC29E02A2CDE
:105BE00001D116200DE4032C23D113F069FD052803
:105BF00003D013F065FD062801D116202DE40FF027
:105C0000EDFA08B1162028E4DD48007838B10EF02E
:105C100045FFDC490988884201DB16201DE4FBF7BB
:105C2000CBFC08B1162018E4FBF748FA08B116209F
:105C300013E4284611E43CB9042016F0F3FB0120DC
:105C4000D1490870122008E4284606E444B9FEF75A
:105C5000C1FB032024F006FA012016F0E3FB0BE061
:105C6000032C09D113F02CFD062805D1002016F0D5
:105C7000D9FB0020FCF79FFA28460FE444B9FEF751
:105C8000A9FB0020FCF797FA002016F0CBFB11E0EF
:105C9000032C0FD1BD48007801280BD113F010FD63
:105CA000052807D127F04AFB0020B8490870FF20DB
:105CB000FCF781FA28460DE46CB921F0A1FB0EF047
:105CC000D3FA064629F00AFE012016F0ABFB0420A9
:105CD00024F0C8F923E0032C1DD113F0F1FC0328B4
:105CE0000AD013F0EDFC042806D114F063FE18B9B5
:105CF00024F01BFA1B200DE424F0BAF808B11C2094
:105D000008E4FBF7EDF950B124F09CF838B124F029
:105D10000CFA1B200CE4192C01D11C2008E42846A5
:105D200006E4032C04D124F0A3F808B11C2030E4CD
:105D300028462EE46CB929F041FA06460EF094FA92
:105D4000B04204D030460EF099FA1D2021E41E2006
:105D50001FE428461DE49CB90EF096FA0646012E73
:105D60000AD0002033461822092100904FF48030D9
:105D7000FDF778FF1E200CE47F481AF0DDFB18E0E9
:105D8000032C16D10EF0B8FE0C2801D11E2011E410
:105D9000794800681AF098FB44F62061884208D9D7
:105DA0000EF0AAFE1D2101EB0020744908603D2081
:105DB00011E428460FE40CB90B200CE428460AE451
:105DC00074B921F01DFB012016F02CFB0EF040FAF7
:105DD000064630462AF074FA052024F043F914E010
:105DE000032C0ED124F012F808B1212008E4FBF7AF
:105DF00077F950B123F0FEFF38B124F08AF9202062
:105E000005E41A2C01D1212014E4284612E4032CC5
:105E100004D123F0FBFF08B121200BE4284609E45C
:105E20006CB929F0DFFF06460EF012FAB04204D03A
:105E300030460EF013FA222014E4232012E4284600
:105E400010E49CB90EF020FA0646012E0AD000207C
:105E500033461922092100904FF48030FDF702FFEC
:105E6000232008E444481AF067FB18E0032C16D1FD
:105E70000EF042FE0C2801D1232008E43E480068C1
:105E80001AF022FB44F62061884208D90EF034FE55
:105E90001E2101EB0020394908603D202AE42846F4
:105EA00028E434B93A48007808B90B2022E42520C8
:105EB00020E428461EE46CB921F0A2FA01203349FF
:105EC000087027F041FA022016F0ACFA062024F000
:105ED000C9F819E0032C0DD1242D15D113F0F0FBD6
:105EE000052801D1172005E413F0EAFB06280BD1A1
:105EF000182010E41B2C07D124480078012801D178
:105F0000192008E40B2006E4284604E444B91E489E
:105F1000007818B916F07AFD17F0A4FD252008E4E2
:105F2000284606E4E4B91848007830B10020164944
:105F3000087016F06BFD17F09CFDFEF74BFA21F090
:105F400069FA072024F08EF824F084F80EF08CF91A
:105F500006462CF007FF022016F064FA27201AE408
:105F6000284618E41CB90B481AF0E6FA76E0152C1E
:105F700012D138200FE40000AC130020741300206D
:105F8000B4130020B21300209D130020A1130020A1
:105F9000A913002088130020162C04D10120FD49EC
:105FA00008701F2004E4222C01D139200CE41D2CA0
:105FB00001D1262008E4202C01D1282004E42B2C38
:105FC00001D12A2005E42C2C01D1292008E4032C3E
:105FD00044D127F003F900B3EF48007803280DDA25
:105FE000ED480078401CEC49087027F0A7F927F02D
:105FF00063F827F0E3F927F0A7F915E014F0D4FCD3
:106000000020E649087027F099F927F055F827F0A5
:10601000D5F90020E049087006E026F0DDFD0128F2
:1060200002D10020DC49087013F04AFB052801D199
:1060300017200FE413F044FB062801D1182009E4CF
:10604000FBF74EF850B121F0F3F910B121F0CEF981
:1060500004E023F0F9FD08B9282007E4284605E408
:106060004CB913F03FFCCD480078012801D119202C
:106070000DE40B200BE4284609E400BF8CB9012095
:1060800016F0D0F921F0BCF924F03BF8392D01D1FC
:1060900024F047F80FF088F808B13B200EE43B20CD
:1060A0000CE428460AE41CB9BD481AF045FA17E08A
:1060B000032C15D10FF078F808B13B2005E4B8485F
:1060C00000681AF001FA4EF66021884208D90EF0F5
:1060D00013FD332101EB0020B24908603D201AE492
:1060E000284618E4F4B3012C03D10020AE4908700F
:1060F0008DE0232C03D124F010F83C200BE4032C7A
:1061000061D123F09BFE08B1252004E4FAF7E8FFF3
:1061100030B123F087FE18B123F0FFFF3C2012E4DA
:10612000A24800681AF0D0F94CF25031884213D9D5
:106130009A48007880B99C48007868B913F0C0FA92
:10614000032809D123F06EFE30B101209649087072
:106150009249087027F0F8F827F040F8D0B18E483F
:10616000007800E053E003280DDA8B480078401CEB
:106170008949087027F0E2F826F09EFF27F01EF903
:1061800027F0E2F80DE023F04DFE50B123F0C5FFFB
:106190003C201AE426F020FD012802D100207E498F
:1061A000087013F08DFA032831D013F089FA04280F
:1061B0002DD114F0FFFB50BB23F034FE38B323F095
:1061C000ACFF3C200EE4062C01D129200AE4052C6A
:1061D00001D12A2006E4072C01D1332013E4082C36
:1061E00001D134200FE40A2C01D135200BE4092C15
:1061F00001D1362007E40C2C09D01C2C07D16748AC
:106200000078012801D1192018E40B2016E4284653
:1062100014E4032C07D123F011FE20B100206249C1
:10622000087025200AE4284608E400BF44BB21F09A
:10623000E7F821F081F8292D05D10EF023FC064660
:1062400021F0BEF804E00EF0B1FB064621F0B8F8EC
:1062500021F01AF8064621F011F80746314623F0DE
:10626000F1FE9FED530B23F03DFF012016F0DAF80D
:10627000292D02D121F06AF85AE021F079F857E08F
:10628000102C03D121F0A6F82D2004E4032C4FD1CB
:1062900013F016FA042803D121F09CF82D2006E40F
:1062A00013F00EFA052803D121F094F8172045E4E5
:1062B00013F006FA062803D121F08CF818203DE4EB
:1062C00021F020F80646022E01D12B2036E4032EC1
:1062D00001D12F2032E4052E01D131202EE4042EED
:1062E0000BD120F0C5FF34490880084600888C286F
:1062F00001D1302022E4322020E41F2E08D120F0EA
:10630000B7FF322101EB0020264908603D2015E44B
:1063100020F0C0FFB0EE408B23F0E4FE20F0B4FF8D
:10632000074620F0ABFF8046394623F08BFE00BFC6
:10633000284605E484B9B7EE000B23F0D3FE20F025
:10634000A3FF064620F09AFF0746314623F07AFE67
:1063500016481AF0F1F80BE0032C09D11348006835
:106360001AF0B2F842F21071884201D92C200DE4E3
:1063700028460BE41CBB0D481AF0DEF80DF012FFA6
:106380000646012E1AD0202000EB062005490860A1
:106390003D200BE4A9130020B5130020A113002019
:1063A000AC13002074130020A813002088130020D1
:1063B00000000000000000009013002025E0032CE6
:1063C00023D10EF099FB06460C2E01D12E2009E4B4
:1063D000342E08D10EF0F0FA212101EB0020FD4906
:1063E00008603D200AE4FC4800681AF06DF84EF69B
:1063F0006021884208D90EF07FFB222101EB0020AA
:10640000F44908603D2009E400BF284606E43CB991
:10641000AFF62412AFF64011F0A023F049FE0AE0D7
:10642000032C04D1FAF75CFE28B125200BE40F2CD5
:1064300001D1252007E4284605E444B9EB481AF0C9
:106440007BF8E9A2E8A1EAA023F032FE40E0032CA9
:106450003ED120F001FF074617B1E4481AF06CF86E
:1064600020F050FF0646022E01D0032E01D12F202E
:1064700021E4052E01D131201DE4042E0BD120F0A2
:10648000F7FEDE490880084600888C2801D13020BC
:1064900011E432200FE41F2E08D120F0E9FE232161
:1064A00001EB0020CB4908603D2004E4CF480068A0
:1064B0001AF00AF849F64041884208D920F022FF34
:1064C000242101EB0020C34908603D2013E400BFF4
:1064D000284610E464B913F0F3F8032801D026F03D
:1064E0002DFFC1A2AFF61021C5A023F0E1FD0AE007
:1064F000032C04D1FAF7F4FD28B125200AE40F2C6F
:1065000001D1252006E4284604E434B9AFF6382248
:10651000BFA1C2A023F0CCFD0AE0032C04D1FAF7FE
:10652000DFFD28B1252004E40F2C01D125200DE446
:1065300028460BE434B9ACA2AFF66421B9A023F02D
:10654000B7FD0AE0032C04D1FAF7CAFD28B12520D3
:1065500011E40F2C01D125200DE428460BE464B989
:10656000A6480288B2A101A82CF0EAFD9EA2AFF6CF
:106570009821B0A023F09CFD0AE0032C04D1FAF787
:10658000AFFD28B1252013E40F2C01D125200FE405
:1065900028460DE400BF74B923F060FD8E4819F061
:1065A000CBFF332D02D10DF0F1FD2DE0342D2BD199
:1065B0000DF0F8FD28E0032C26D10EF09DFA0646DA
:1065C0000C2E04D101209E49087025200EE4342EA3
:1065D00008D10EF0F1F9252101EB00207D4908607A
:1065E0003D200DE47C48006819F06EFF4EF66021F6
:1065F000884208D90EF080FA262101EB0020754967
:1066000008603D2009E400BF284606E48CB923F069
:1066100025FD714819F090FF0DF0D0FD0646012EC2
:1066200006D0272000EB06206A4908603D2005E4DB
:106630002DE0032C2BD16848006819F045FF44F683
:106640002061884223D90EF057FA06460C2E01D15C
:10665000372006E4342E08D10EF0AEF9282101EBE4
:1066600000205C4908603D2007E45B48006819F0A1
:106670002BFF4EF66021884208D90EF03DFA292101
:1066800001EB0020534908603D2007E400BF284685
:1066900004E48CB923F0E2FC4F4819F04DFF0DF0F3
:1066A00037FE0646012E06D02A2000EB0620494977
:1066B00008603D2017E42DE0032C2BD146480068EC
:1066C00019F002FF44F62061884223D90EF014FA33
:1066D00006460C2E01D1372005E4342E08D10EF0E9
:1066E0006BF92B2101EB00203A4908603D2008E4BA
:1066F0003948006819F0E8FE4EF66021884208D952
:106700000EF0FAF92C2101EB0020324908603D20FF
:1067100005E400BF284604E444B901204849087054
:1067200031A231A147A023F0C3FC0AE0032C04D11D
:10673000FAF7D6FC28B1252011E40F2C01D1252031
:106740000DE428460BE400BF00BF64B901203F49B7
:10675000087026F0F9FD00203D49088020F05AFE1F
:10676000FDF754FD26E0032C23D13948B0F9000091
:10677000002806DD36480088401E00B234490880F3
:106780000EE0322032490880FDF724FE012015F08A
:1067900049FE0D2023F066FC0E48006823F04CFCF7
:1067A000FAF78CFC30B120F043FE18B120F01EFE49
:1067B00000E000BF284605E454B920F021FE012086
:1067C00015F030FE08A208A122A023F071FC46E0DB
:1067D00044E000007413002088130020494D414715
:1067E00045532053415645440000000098130020B3
:1067F00053544F5050494E47000000009013002062
:10680000534156452043414E43454C4C45440000BE
:10681000415641494C41424C4500000055534220ED
:106820004E4F54005553422046554C4C000000003A
:106830002564000053415645204641494C454400DB
:106840009D1300205355434345535300A11300208B
:1068500092130020544553540000000000BF284606
:1068600006E4FE2000EB0520014908603D2015E408
:106870007413002001480068704700007413002062
:10688000014800787047000070130020014800782C
:10689000704700009E13002010B5002005490870C5
:1068A000054823F021FB05480EF0D8FF042000F036
:1068B0003DF810BD70130020D9A402081BA30208E4
:1068C0000C480078132801D101207047094800784E
:1068D000142801D10120F8E706480078152801D1D5
:1068E0000120F2E703480078162801D10120ECE7E7
:1068F0000020EAE77013002010B5212000F016F800
:1069000010BD10B5242000F011F810BD10B52320E3
:1069100000F00CF810BD10B5202000F007F810BDF5
:1069200010B5222000F002F810BD00002DE9F0475C
:1069300080462048077841463846FEF7B7FC0446B3
:106940004FF00009A74201D1012000E0002082465B
:1069500029E009F101000FFA80F9B9F1C80F0BDD48
:1069600040F2E730144908603E20124908700021C7
:10697000FEF79CFCBDE8F08701213846FEF796FC47
:106980000546BD4200D02C4600212046FEF78EFC75
:106990000646A64202D14FF0010A03E027463446DC
:1069A0004FF0000A00BFBAF1000FD2D001480470C6
:1069B00000BFDFE7701300207413002010B5012022
:1069C000024908701D20FFF7B1FF10BD9D13002084
:1069D00010B52D20FFF7AAFF10BD000010B5044828
:1069E0000068401C024908600320FFF79FFF10BDAC
:1069F0007C13002070B504461649204626F05CFE44
:106A000028B31548007805280BD1FBF711FC054683
:106A100010490888294619F065FB04200E490870C2
:106A20000AE0FBF709FC05460A490888294619F0DF
:106A300059FB0520084908700848048000EE104AF8
:106A4000B8EE400B064880ED000B012070BD002021
:106A5000FCE70000866A0120511500205215002035
:106A6000581500200C490988491E0C4A1288914289
:106A700002DC042101700EE00121094A117007496E
:106A80000988491C00EE101AB8EEC00B054981EDCB
:106A9000000B0021017070474A1500204C150020A2
:106AA00060150020681500200B490988002902DCC8
:106AB000032101700EE00121084A1170064909887E
:106AC000491E00EE101AB8EEC00B054981ED000B0F
:106AD00000210170704700004C1500206015002057
:106AE0006815002003B5ADF5097D8A9848BB8998E3
:106AF000032811D0252819D1F74880880090F6483E
:106B000040888790F4480088869002460420879B3E
:106B10008999FDF7A7F813E0002003460090EF489D
:106B2000027804208999FDF79DF809E000200346CA
:106B30000090EB48026804208999FDF793F800BFA4
:106B400000BF8998352881F0EB85DFE810F035002B
:106B500044004E00A000BB00BC00D6002501380157
:106B600078018F01AC0D050205065105CF0501071F
:106B70004A085308A308B908CF0833094A0970091D
:106B800079092808020D210D800D960D4107520745
:106B900074079807270528059D09A809100B240BE1
:106BA000490BBE0BD20BE90B030C760C8A0CE80CDC
:106BB000AA04B5040405D50D8A98042809D1C9484A
:106BC0001DF018FBC8481DF02DFB01200DF50B7DB5
:106BD00000BD8998FAE78A98052804D10120C349A5
:106BE00008700220F2E78998F0E78A9868B90020D7
:106BF000879087AB40F259720021BD4800681DF0B4
:106C0000A3FA1420BB4908803FE08A980A281ED1C5
:106C1000B74800680068B849884210D10020B749D9
:106C20000870B348006890F8000418B10020AB4920
:106C3000087002E00120A94908700320C6E701207E
:106C4000AE4908700220AE4908800420BEE78A9849
:106C50000B2808D10DF0B0FE662101EB0020A04901
:106C600008600B20B2E78A9802280ED1A14800885C
:106C7000002805DD9F480088401E9E49088004E0EA
:106C80006720974908600B20A0E789989EE78A98BB
:106C9000B0B9FAF7ABFE86A819F068FC9DF81802A7
:106CA00048B9BDF91A02BDF91C1200EB01208C494C
:106CB00008600B208AE70120914908800C2085E7B5
:106CC000899883E700BF8A98A8B90DF07BFE002859
:106CD00001DD012000E000208A490870899805281C
:106CE00004D100201BF074FE08206FE701201BF088
:106CF0006FFE06206AE7899868E78A9810BB824889
:106D000019F01AFC0020879087AB012211467848C1
:106D1000006800F500701DF08DFB86900020034692
:106D200000909DF81C2208214803FCF79BFF8698E1
:106D300038B13C21869801EB002069490860342075
:106D400044E727E08A98072800D13FE78A98082877
:106D500004D17820624908600B2037E78A98092817
:106D600004D179205E4908600B202FE78A98032818
:106D700010D16548006819F0A7FB44F620618842ED
:106D800008D90DF0B9FE7A2101EB002054490860C2
:106D90000B201BE7899819E78A9818B95A4819F007
:106DA000CBFB0AE08A98032807D15748006819F0FE
:106DB0008BFB642801D9082008E7899806E78A98A0
:106DC000E0B932204B4908804FF4EB6087900020F7
:106DD000869086AB02214648879A006800F580605D
:106DE0001DF028FB8590859838B17B21859801EBB3
:106DF00000203B4908600B20E8E61EE08A9807283F
:106E000001D10920E2E68A98082804D17C2034497F
:106E100008600B20DAE68A9802280ED135480088EF
:106E2000002805DD33480088401E3249088004E010
:106E30007D202B4908600B20C8E68998C6E68A9811
:106E400018B902202B4908800EE08A9802280BD13D
:106E500028480088002805DD26480088401E25496E
:106E6000088001E00A20B1E68998AFE68A98B8B9AF
:106E70000020879087AB012200211D4800681DF08B
:106E8000D9FA8690869838B17E21869801EB002049
:106E9000134908600B2099E632201649088059E012
:106EA0008A9807283CD10020184908801849088092
:106EB00018490880184908800021184801801148A5
:106EC000007830B100200F49087000210846FCF717
:106ED000D5FB0C207AE60000A459012039140020CB
:106EE0006C140020012502082925020872140020D4
:106EF0009814002070140020CDDBCDDB3814002066
:106F00007414002047140020901400203A1400202C
:106F10003C140020401400203E14002042140020A5
:106F20008A98082804D17F20F84908600B204DE694
:106F30008A9802280ED1F6480088002805DDF4481A
:106F40000088401EF249088004E08020EF49086074
:106F50000B203BE6899839E68A98002810D08A9859
:106F6000212804D10120EB49087031202EE68A98AF
:106F70001B282BD1E848007818B10420E549087097
:106F80008DE2E64800884EF66021884203DB05204A
:106F9000E049087083E206F0B1FC87909DF81C027E
:106FA00002468490DD48018885A807F059F8BDF8AD
:106FB0001402C0F3801018B90620D649087004E006
:106FC0000120D44908701A2000E668E28A981D283A
:106FD0000BD1D148007818B10420CE4908705EE288
:106FE0000120CC4908702320F0E58A981E280BD197
:106FF000C948007818B10420C64908704FE2012042
:10700000C44908702420E1E58A981C2835D1C2487B
:10701000007818B10420BF49087040E2BF480088DA
:107020004EF66021884203DB0520BA49087036E23B
:1070300006F064FC87909DF81C0202468490B748D5
:10704000018885A807F00CF8BDF81402C0F3801081
:1070500018B90620AF4908700EE0BDF81A024FF6C5
:10706000FF71884203D10720AA49087004E001207B
:10707000A84908701B20A9E511E28A980E280BD1B7
:10708000A548007820B90120A24908700E209DE58E
:107090000420A049087002E28A980F2852D19E4825
:1070A000007818B10E209B490870F8E101209A4938
:1070B000087000209A4908809A48006800F5C0606E
:1070C0009949097800EB412040894FF6FF718842C9
:1070D00028D19448006800F5C0609349097800EB16
:1070E000412000884EF6602188420FDA8D48006802
:1070F00000F5C0608C49097800EB412000883221FE
:1071000001EB00208149086034205FE58548006874
:1071100000F5C0608449097800EB4120408883492C
:1071200008800AE07F48006800F5C0607E49097861
:1071300000EB412040897D49088001207549087095
:107140000C2043E58A98102826D17348007820B98E
:107150000820704908700C2038E57148008841F219
:107160009411884204DB0F206A4908700C202DE539
:107170006E4800886E490880084600884EF66021F7
:10718000884204DB03206149086034201EE50120A9
:10719000604908700D2019E58A98112819D15E48B8
:1071A000007890B15E48008838B900205A490870CC
:1071B0000120584908700C2008E500205649087045
:1071C000012054490870102000E50820514908703A
:1071D00065E18A9812283BD14F48007818B1042005
:1071E0004C4908705BE10DF0CDFF18B1032049490F
:1071F000087054E106F082FB87909DF81C0202465D
:1072000084904648018885A806F02AFFBDF814023C
:10721000C0F3801018B906203E49087017E0BDF889
:107220001402C0F3401018B90A203A4908700EE061
:10723000BDF81A024FF6FF71884203D00C20354981
:10724000087004E00120334908701120BEE426E1F3
:107250008A98132834D13048007818B104202D4979
:1072600008701CE106F04AFB87909DF81C0202465C
:1072700084902A48018885A806F0F2FEBDF8140221
:10728000C0F3801018B906202249087017E0BDF835
:107290001402C0F3401018B90A201E4908700EE00D
:1072A000BDF81A024FF6FF71884203D10B2019492D
:1072B000087004E0012017490870182086E4EEE009
:1072C0008A9814280FD10DF07DFB002807DD0020DF
:1072D0001149087001200F490870042076E401204C
:1072E0000C490870DBE08A98152823D10DF06AFB61
:1072F000002807DD002008490870012005490870B2
:10730000052063E4012003490870C8E06C140020E4
:1073100070140020721400207C14002060140020DF
:107320007E140020981400203914002080140020BE
:10733000581400208A9816282BD1F848007818B1E4
:107340000420F7490870AAE006F0D8FA87909DF863
:107350001C0202468490F348018885A806F080FE4E
:10736000BDF81402C0F3801018B90620EC4908706B
:107370000EE0BDF81402C0F3401020B90120E84926
:1073800008701F2022E40120E549087021201DE437
:1073900085E08A98172821D1E048007818B10420A8
:1073A000DF4908707BE006F0A9FA87909DF81C027F
:1073B00002468490DB48018885A806F051FEBDF89E
:1073C0001402C0F3801018B90620D549087004E0F3
:1073D0000120D34908701F2004E460E08A9818282F
:1073E0002AD1CE48007818B10420CD49087056E063
:1073F00006F084FA87909DF81C0202468490C948E2
:10740000018885A806F02CFEBDF81402C0F3801098
:1074100018B90620C24908700DE0BDF81402C0F387
:10742000401018B90A20BE49087004E00120BC4988
:10743000087021200AE432E08A98192807D1012037
:10744000B74908700DF0B2FA48B322200AE48A98CE
:107450001A2801D11C2005E48A98202804D1012093
:10746000AF49087025200FE48A98062803D101202F
:10747000AB49087008E48A981F2810D10120A84958
:107480000870A9490870A9490870A94812F0BBFA08
:107490000FF00EFCA64811F0EDFD25200AE48998B6
:1074A00008E48A9830B9FAF7B1FA0A20A1490880AD
:1074B000322004E4899804E48A9810BB9E4819F0AD
:1074C0003BF80020879087AB012211469B4800685B
:1074D00000F500701CF0AEFF86900020034600907F
:1074E0009DF81C2208214803FCF7BCFB869838B1A4
:1074F0003C21869801EB00219148016034201FE473
:1075000027E08A98072805D100210320FCF7B6F868
:107510000C2015E48A98082805D101210420FCF7E5
:10752000ADF80C200CE48A98092801D1332007E437
:107530008A9803280DD18048006818F0C5FF44F6EA
:107540002061884205D902210420FCF797F80C201D
:107550000BE4899809E48A9818B97A4818F0ECFF86
:107560001AE08A98032817D17648006818F0ACFF13
:10757000B0F57A7F10D96F480088002806DD6D4885
:107580000088401E6B490880322004E40321042057
:10759000FCF774F80C200FE489980DE400BF8A987A
:1075A00020BB654818F0C8FF614812F002FA0FF0DE
:1075B0007FFB8998232801D1012000E000208790DB
:1075C00001225B49879811F077FD86908698012803
:1075D00007D03221869801EB002159480160342000
:1075E0000AE4534811F046FD252005E4899809E492
:1075F0008A9890BB32215448018001205349087079
:10760000494908704A4812F0D4F90FF051FB0DF0C7
:10761000B9FD78B10121464810F0FAFE88908898AB
:10762000012807D00421889801EB0021444801601B
:10763000342018E40020879001223D4987A80FF0EC
:107640000BF988908898012808D00521889801EBCB
:1076500000203B490860342005E422E0344811F062
:1076600009FDBDF81C0240F2D511484340F2627199
:1076700001EB400086900020859085AB40F2AA3255
:107680003348869900681CF0D5FE8490849838B100
:107690000621849801EB002029490860342019E470
:1076A00022E08A98072801D10F2013E48A9808283D
:1076B00004D107202249086034200BE48A9802286C
:1076C00012D121480088002805DD1F480088401E8F
:1076D0001D49088008E01BF06DFD082101EB00202A
:1076E00017490860342022E4899820E48A9818B960
:1076F000184818F021FF0EE08A9803280BD115488E
:10770000006818F0E1FE87908798B0F57A7F01D97C
:1077100025200CE400BF899809E400007C140020B7
:10772000721400206014002046140020451400202C
:10773000A459012050140020901400209814002017
:107740006C140020941400207014002044140020B5
:1077500054140020781400208A98B8BBF848008898
:1077600040F2D511484340F2627101EB400087902E
:107770000020869086AB40F2AA32F24887990068D2
:107780001CF058FE8590859808B3EF480088401C8F
:10779000ED490880084600880F2808DD9DF818028A
:1077A000092101EB0020E949086034200CE4E84994
:1077B00085980880E7480088401CE6490880E6482C
:1077C0000088401CE44908800C200DE406E00020FD
:1077D000DD4908803221E1480180B7E08A98072816
:1077E0007DD1DF480088401CDD49088008460088BC
:1077F000012803D1D2480088DA490880D04800889F
:10780000D9490880CE480088C117839000EB916069
:1078100080118790CA480088C117839000EB91605F
:1078200081118398A0EB811080B286900020859012
:1078300087987C90CD48006800F5C060CC490978F5
:1078400000EB412010304FF4F872014683906846F7
:10785000F8F7EEFCC548006800F5C060C449097837
:1078600000EB412083900FC8F9F7E8FA08B1012036
:10787000859040F2D51185984843BC49096801F5C7
:10788000206101EB8021879801EB4021869801EB74
:10789000C000408884904FF6FF71849888420BD1D5
:1078A000B248006800F5C060B149097800EB41209A
:1078B0004088B049088010E04EF6602184988842E4
:1078C00008DB0B21849801EB0021A04801603420E3
:1078D0001BE404E0A749849808800C2015E48A98EA
:1078E00009280BD19B480088401C9A4908809A4877
:1078F0000088401C984908800C2006E48A980828D3
:107900000BD194480088401C924908809248008816
:10791000401C914908800C2013E48A98022815D154
:107920008E480088002805DD8C480088401E8B4961
:1079300008800BE087480088401C864908808648FC
:107940000088401C844908800C2005E489980EE4D6
:107950008A98A8BB0120884908708849087088481F
:1079600012F027F80FF0A4F90DF08CF8B0F57A7F3B
:107970000FDB0121824810F04BFD88908898012888
:1079800007D00E21889801EB002170480160342057
:1079900012E47548008800907248038801227849F3
:1079A0006F4800880FF038F888908898012808D030
:1079B0000F21889801EB002164480160342045E4E0
:1079C00004E06F4811F056FB25203FE489983DE420
:1079D0008A9860B90120684908700CF0F3FF01280B
:1079E00003D168490870042030E420202EE48998EF
:1079F0002CE48A98F0B9012063490870604811F0BE
:107A0000D8FF0FF055F901225D49604800880FF05A
:107A1000CFFD87908798012807D01021879801EB28
:107A200000204A490860342010E4554811F022FB38
:107A300025200BE400BF8A9800BB01204E49087046
:107A4000514908704E4811F0B4FF0FF031F901228E
:107A50004B494E48008810F04DFD879087980128CB
:107A600007D01121879801EB0020384908603420A5
:107A700024E4434811F0FEFA25201FE400BF8A9851
:107A800008BB434818F058FD01203B4908703E49A7
:107A900008703B4811F08DFF0020034614220A2194
:107AA00000904FF48030FCF7DDF80FF001F9002072
:107AB000034615220A2100904FF48030FCF7D2F8DB
:107AC0000FF060FD69E08A98032866D101212C48F7
:107AD0000FF0A8FC8790879824280ED12C480068C6
:107AE00018F0F2FC2B49884256D94B21879801EBBC
:107AF000002116480160342044E48798012816D1FB
:107B00000020034616220A2100904FF48030FCF733
:107B1000A9F81B4811F0AEFA0020034617220A21EB
:107B200000904FF48030FCF79DF825202AE41221C4
:107B3000879801EB002005490860342022E42CE0FE
:107B400058140020541400204E1400206C140020FF
:107B50004C140020481400204A1400207014002007
:107B60007E14002064140020661400209814002065
:107B700039140020801400204614002044140020F2
:107B8000A459012072140020451400206014002024
:107B900090140020A086010000BF89981CE48A98F8
:107BA000E8B9FE4811F005FF0FF082F80123FB4A07
:107BB000FB480178FB48008811F08EFB879087987E
:107BC000012807D01321879801EB0020F6490860AF
:107BD00034202FE4F14811F04DFA25202AE4899849
:107BE00028E48A9820B90120F0490870122021E485
:107BF00089981FE48A9810BBEA48008840F2D511A2
:107C0000484340F2627101EB40008790002086906B
:107C100086AB40F2AA32E648879900681CF094FAD5
:107C20008590859838B11421859801EB0020DE49B4
:107C3000086034200AE43220DE49088028E08A986F
:107C40000A2801D1142006E48A980B2804D11520B3
:107C5000D5490860342006E48A980C2801D1132005
:107C600008E48A980D2801D1132017E48A98022885
:107C70000ED1D0480088002805DDCE480088401E7F
:107C8000CC49088004E01620C7490860342005E488
:107C9000899805E48A9818B9C74818F04DFC0DE09A
:107CA0008A9803280AD1C448006818F00DFC879010
:107CB0008798C82801D9122021E400BF89981EE4C2
:107CC0008A9818B9BC4818F037FC0DE08A98032848
:107CD0000AD1B948006818F0F7FB87908798C82840
:107CE00001D915200BE400BF899808E48A98D8BB15
:107CF000B248006800F5C060B149097800EB412046
:107D00004089B0490880084600884EF660218842C4
:107D100008DBAC480088172101EB0020A24908606D
:107D2000342004E40120A8490870A648008840F2E5
:107D3000D511484340F2627101EB4000879000206A
:107D4000869086AB40F2AA329948879900681CF069
:107D500071FB8590859840B11821859801EB002032
:107D600091490860342010E403E0322091490880F2
:107D70001EE08A98072801D1162006E48A98082870
:107D800004D1192088490860342004E48A98022824
:107D90000ED188480088002805DD86480088401EEE
:107DA0008449088004E01A207F490860342017E4E1
:107DB000899815E48A9818B97F4818F0BDFB0EE041
:107DC0008A9803280BD17C48006818F07DFB8790C7
:107DD0008798B0F57A7F01D9172006E400BF89980B
:107DE00005E48A9808BB01207849087008706B4840
:107DF00011F0DFFD0EF05CFF0123684A7148018835
:107E0000684800880EF0B8FF87908798012807D04F
:107E10001B21879801EB002063490860342008E4A7
:107E20005E4811F027F9252016E4899814E48A9811
:107E300020B901205D49087019200DE489980BE4F0
:107E40008A98F8B90120614908700870534811F008
:107E5000B0FD0EF02DFF01225049524800880FF06E
:107E6000AFFF87908798012807D01C21879801EBE6
:107E700000204D490860342011E4484811F0FAF818
:107E800025200CE489980AE48A9830B900205049EA
:107E9000088050490880262007E4899805E48A98DC
:107EA000C8BB3E48801C4A49098830F811008790B9
:107EB0000121494801800020869087987C903F48A6
:107EC000006800F5C0603E49097800EB41201030A1
:107ED0004FF4F872014680906846F8F7A9F93748E0
:107EE000006800F5C0603649097800EB41208090B9
:107EF0000FC8F8F7A3FF08B1012086908698C0F15B
:107F00000100C0B285908798849031480088401C59
:107F100080B2809084E0EAE000207F901F48801CBF
:107F2000809930F811007E908498401C7E9981429F
:107F300067D18698012821D17E987C901F480068DF
:107F400000F5C0601E49097800EB412010304FF465
:107F5000F87201467D906846F8F76AF9174800689C
:107F600000F5C0601649097800EB41207D900FC8EC
:107F7000F8F764FF90B301207F9042E07E987C90F8
:107F80000E48006800F5C0600D49097800EB4120FB
:107F900010304FF4F87201467D9020E0A459012082
:107FA00062140020601400206C140020461400208D
:107FB000541400207014002078140020981400201D
:107FC00039140020581400204414002045140020C7
:107FD000A014002082140020A214002011E06846A2
:107FE000F8F726F9F848006800F5C060F749097805
:107FF00000EB41207D900FC8F8F720FF08B9012061
:108000007F907F9838B1F2480088401CF049088082
:108010007E98849000E009E08098401C80B28090B7
:10802000EC480188809881423FF776AF00BF87987F
:10803000401D83908598012803D1839800F2AA30CF
:1080400083908398009000214FF48030879B859A1D
:10805000FBF708FE002003460090DD48028800215F
:108060004FF48030FBF7FEFD3220DB490880002012
:10807000829040F2D51185984843D349096801F5AB
:10808000206101EB8021879801EB402082AB80903A
:10809000CF480288839980981CF0CCF98190819810
:1080A00020B3CE48008803280FDACD4981980870A4
:1080B000CC480088401CCB490880C8480088401C38
:1080C00081B2C6480180272008E4002000909DF876
:1080D000083201210804819AFBF7C4FD1D21819813
:1080E00001EB0020C0490860342006E43DE08A9896
:1080F000072801D128200FE48A98082804D11E20DF
:10810000B9490860342007E48A98092817D1B34890
:10811000008803280EDA6320B1490870B14800884E
:10812000401CB0490880AD480088401CAB4908801D
:1081300027200AE41D20AC490860342005E48A9811
:10814000022812D1A4480088002805DDA248008832
:10815000401EA149088008E01BF02CF81F2101EB0C
:108160000020A1490860342012E4899810E48A981C
:1081700018B99E4818F0E0F90BE08A98032808D156
:108180009A48006818F0A0F9B0F5FA6F01D92620D6
:1081900015E4899813E48A9818B9954818F0CCF931
:1081A0001CE08A98032819D19148006818F08CF9CE
:1081B00087908798B0F57A7F0FD98E4801888448D8
:1081C000008808448B4908808248008809888842D2
:1081D00001DD262008E4292006E400BF899805E493
:1081E0008A98E8BB32207C49088078480078F8B942
:1081F0000020879087AB012204217348006800F5B6
:1082000000601CF017F986900020034600909DF84E
:108210001C220221C803FBF725FD869838B12021D6
:10822000869801EB002170480160342020E44AE088
:108230000020879087AB012203216348006800F586
:10824000C0601CF0F7F886900020034600909DF86F
:108250001C2203214FF48030FBF704FD869800E0D8
:1082600009E038B12121869801EB00205E490860C1
:10827000342041E427E08A98072801D12B203BE4F1
:108280008A98082804D1222057490860342033E412
:108290008A98092801D12A202EE48A98022812D12E
:1082A0004D480088002805DD4B480088401E4A499B
:1082B000088008E01AF07EFF232101EB00204A49E4
:1082C0000860342018E4899816E48A9818B94A4856
:1082D00018F032F90BE08A98032808D14648006864
:1082E00018F0F2F8B0F5FA6F01D9292004E4899862
:1082F0001CE48A9818B93E4818F01EF90EE08A98D6
:1083000003280BD13A48006818F0DEF88790879868
:10831000B0F57A7F01D92C2008E400BF899805E4E4
:108320008A98A8B92948007840B9002026490968E8
:1083300081F8000401202549087007E00120224946
:10834000096881F800040020204908702D2025E4E8
:10835000899823E48A9838BB32201F49088000207E
:10836000879087AB012202211748006800F58060E2
:108370001CF060F88690002000901348006890F888
:10838000000485909DF81C32024604218803FBF707
:1083900069FC869838B12421869801EB00201249A7
:1083A0000860342015E446E08A98072804D10020AC
:1083B000124908802F200CE48A98082820D1252013
:1083C00009490860342004E498140020391400207E
:1083D000A2140020A459012070140020821400204F
:1083E00086140020841400206C14002088140020BF
:1083F00078140020A0140020901400207E14002087
:108400008A98092801D12E2014E48A98022812D1D2
:10841000C7480088002805DDC5480088401EC449BB
:10842000088008E01AF0C6FE262101EB0020C149B1
:108430000860342007E4899805E48A9818B9BE4892
:1084400018F07AF80BE08A98032808D1BA48006837
:1084500018F03AF8B0F5FA6F01D92D2005E48998A3
:1084600015E48A98C0B9B54818F066F8B44818F011
:1084700063F8B448007870B3F8F7A6FEB248007805
:1084800003284AD1B148B0F900002D2101EB0020AA
:10849000A849086034200FE48A9803283DD1A948F0
:1084A000007840B9A548006818F00EF8B0F57A7F5A
:1084B00033D9302016E4F8F7AFFEA348007803283C
:1084C0000AD1A248B0F90000272101EB0020994908
:1084D0000860342006E420E09B48007802280BD195
:1084E0009648006817F0F0FFB0F57A7F15D90020A4
:1084F00094490870302014E49148006817F0E4FFB4
:108500004EF66021884208D98F480078282101EB77
:10851000002088490860342025E4899823E48A985B
:10852000A8B98B48007830B1002089490870002133
:108530000120FBF7A3F88748007830B10020854977
:10854000087000210220FBF799F80C200BE48998B1
:1085500009E48A98D0B9804811F02BFA0EF0A8FBF4
:108560007D497E48008810F0BBFF879087980128DE
:1085700007D02921879801EB00206E49086034203C
:1085800015E4754810F076FD252010E489980EE476
:108590008A9868BB7248008840F2D511484340F27F
:1085A000627101EB400087900020869086AB40F21C
:1085B000AA326C48879900681BF0C6FD85908598A3
:1085C00030B932205A4908800120674908700EE00E
:1085D000002000909DF818320B214FF48030859ACE
:1085E000FBF740FB2920604908700C2017E42CE0C1
:1085F0008A980A2801D11E2011E48A980B2804D1F8
:108600002B204C490860342009E48A980C2801D1B9
:108610001D2004E48A980D2801D11D2004E48A98C5
:10862000022812D142480088002805DD4048008811
:10863000401E3F49088008E01AF0BCFD2C2101EBE8
:1086400000203C490860342016E4899814E48A9894
:1086500018B93A4817F070FF0DE08A9803280AD13C
:108660003648006817F030FF87908798C82801D9EE
:108670001C2006E400BF899805E48A9818B92F48A1
:1086800017F05AFF0DE08A9803280AD12B4800689A
:1086900017F01AFF87908798C82801D90C2013E596
:1086A00000BF899810E58A9820B38A9805280BD1D5
:1086B00000202E49087026490870264908700120BC
:1086C000294908700220FFE48A98062803D1012076
:1086D00025490870F8E48A9814280BD10020234912
:1086E00008701B4908701B49087001201E4908705A
:1086F0000420E9E48998E7E48A9878B18A981428F4
:108700000BD10020194908701149087011490870EF
:108710000120154908700420D6E400BF8998D3E4ED
:10872000FE21899801EB0020024908603420CBE447
:10873000701400206C140020901400207814002085
:108740008C14002046140020BA140020BE1400200F
:108750004414002045140020A45901206014002076
:108760005A1400205C140020721400207C14002095
:108770002DE9F04780462048077841463846FEF705
:10878000B1F904464FF00009A74201D1012000E0F1
:108790000020824629E009F101000FFA80F9B9F1C1
:1087A000640F0BDD40F2E7301449086034201249B1
:1087B00008700021FEF796F9BDE8F08701213846E0
:1087C000FEF790F90546BD4200D02C460021204618
:1087D000FEF788F90646A64202D14FF0010A03E0EF
:1087E000274634464FF0000A00BFBAF1000FD2D03E
:1087F0000148047000BFDFE7681400206C140020FB
:108800000146092903DC01F13000C0B270470F298D
:1088100003DC01F13700C0B2F8E75F20F6E70000A3
:10882000B0F900100F4A12881144002904DA0D49EA
:108830000988494209B20180B0F90010094A12883A
:108840001144B1F5C87F05DD06490988C1F5C87135
:1088500009B201800188034A1288114409B2024A10
:1088600091807047D61C0020CC0C0220B0F900107B
:108870000E4A12881144002904DA0C490988494239
:1088800009B20180B0F90010084A12881144002989
:1088900004DD06490988494209B201800188034A7A
:1088A0001288114409B2024A11817047A01D0020AC
:1088B000700D022002461AB901F10800C0B27047DB
:1088C00001F11700C0B2FAE7B5EEC00BF1EE10FAF5
:1088D00003D29FED0E1BB0EE410B0E48008801EE57
:1088E000100AB8EE411BB4EEC10BF1EE10FA07DD31
:1088F0000848008801EE100AB8EE411BB0EE410BAB
:10890000BCEEC01B11EE100A80B2704700000000E0
:10891000000000004A15002010B5F8F71DFC10BD3E
:1089200070B505460E461446A4F120003A2822D21E
:10893000DFE800F0D1D2D2D2D2D2D2D2D2D2D2C2B9
:10894000D2C7BDCC1D22272C31363B40454AD2D25E
:10895000D2D2D2D2D24F54595E63686D7277D27C34
:1089600081868B9095D29A9FA4A9AEB3D2B8314696
:10897000284600F0F4F8AFE03146284600F04BF905
:10898000AAE03146284600F059F9A5E031462846CC
:1089900000F07EF9A0E03146284600F0A6F99BE001
:1089A0003146284600F0BBF996E03146284600F0F3
:1089B000E0F991E03146284600F00DFA8CE03146AE
:1089C000284600F01BFA87E03146284600F051FAAD
:1089D00082E03146284600F0A2FB7DE03146284681
:1089E00000F0FAFB78E03146284600F071FC73E0B5
:1089F0003146284600F0D2FC6EE03146284600F0B1
:108A00002BFD69E03146284600F047FD64E0314621
:108A1000284600F05BFD5FE03146284600F0E8FDA7
:108A20005AE03146284600F0FDFD55E03146284623
:108A300000F012FE50E03146284600F0B7FE4BE051
:108A40003146284600F0C4FE46E03146284600F094
:108A500003FF41E03146284600F054FF3CE0314638
:108A6000284600F0ABFF37E03146284600F0F1FF22
:108A700032E03146284601F061F82DE031462846C3
:108A800001F0D8F828E03146284601F0E5F823E067
:108A90003146284601F0FAF81EE03146284601F03A
:108AA0003AF919E03146284601F0C2F914E031469E
:108AB000284601F032FA0FE03146284601F03AFA32
:108AC0000AE03146284600F0F0FA05E03146284633
:108AD00000F0F7FA00E000BF00BF70BD70B50546BA
:108AE0000E4614460A2C38D2DFE804F0050A0F14AB
:108AF000191E23282D323146284600F030F870BD6B
:108B00003146284600F087F8F9E73146284600F05C
:108B100095F8F4E73146284600F0BAF8EFE7314619
:108B2000284600F0E2F8EAE73146284600F0F7F878
:108B3000E5E73146284600F01CF9E0E731462846D3
:108B400000F049F9DBE73146284600F057F9D6E74F
:108B50003146284600F08DF9D1E700BFCFE770B568
:108B600004460D46A9B2A21C90B20323082203F0CA
:108B7000E1FF05F10C0291B2A21C90B2032308227E
:108B800003F0D8FFAA1C91B2A0B20B23032203F07A
:108B9000D1FFAA1C91B204F1090290B20B23032267
:108BA00003F0C8FF6A1C91B2621C90B204F004F991
:108BB000EA1C91B2E21C90B204F0FEF86A1C91B279
:108BC00004F10A0290B204F0F7F8EA1C91B204F141
:108BD000080290B204F0F0F805F10D0291B2621CA7
:108BE00090B204F0E9F805F10B0291B2E21C90B2E8
:108BF00004F0E2F805F10B0291B204F1080290B220
:108C000004F0DAF805F10D0291B204F10A0290B213
:108C100004F0D2F870BD70B505460C46A1B2EA1C4E
:108C200090B20323062203F085FFE21C91B2AA1D35
:108C300090B20C23032203F07DFF70BD70B5044693
:108C40000D46A9B2A0B203230C2203F073FFAA1DA4
:108C500091B2A0B203230C2203F06CFF05F10C02C9
:108C600091B2A0B203230C2203F064FFEA1C91B27C
:108C700004F1090290B203231A4603F05BFF05F1E9
:108C8000090291B2A0B203231A4603F053FF70BD4C
:108C900070B504460D46A9B2A0B203230C2203F01E
:108CA00049FFAA1D91B2E21C90B20323092203F0EE
:108CB00041FF05F10C0291B2A0B203230C2203F094
:108CC00039FFEA1C91B204F1090290B203231A465B
:108CD00003F030FF05F1090291B204F1090290B2EC
:108CE00003231A4603F026FF70BD70B505460C46F7
:108CF000A1B2A8B20923032203F01CFFA21D91B266
:108D0000EA1C90B20323062203F014FFA1B205F17E
:108D1000090290B20F23032203F00CFF70BD70B55F
:108D200004460D46A9B2A0B203230C2203F002FFB1
:108D3000AA1D91B2A0B203230C2203F0FBFE05F1A1
:108D40000C0291B2A0B203230C2203F0F3FEEA1C42
:108D500091B2A0B203231A4603F0ECFE05F109021A
:108D600091B204F1090290B203231A4603F0E2FE25
:108D700070BD70B504460D46A9B2A0B203230C2203
:108D800003F0D8FEAA1D91B2A0B203230C2203F077
:108D9000D1FE05F10C0291B2A0B203230C2203F024
:108DA000C9FEEA1C91B2A0B203231A4603F0C2FE28
:108DB00005F1090291B2A0B203231A4603F0BAFEEC
:108DC00005F1090291B204F1090290B203231A4697
:108DD00003F0B0FE70BD70B504460D46A9B2A0B256
:108DE00003230C2203F0A6FEEA1C91B204F109024F
:108DF00090B20C23032203F09DFE70BD70B50446B3
:108E00000D46A9B2A0B203230C2203F093FEAA1DC3
:108E100091B2A0B203230C2203F08CFE05F10C02E8
:108E200091B2A0B203230C2203F084FEEA1C91B29B
:108E3000A0B203231A4603F07DFE05F1090291B2A8
:108E4000A0B203231A4603F075FEEA1C91B204F1A6
:108E5000090290B203231A4603F06CFE05F10902E1
:108E600091B204F1090290B203231A4603F062FEA4
:108E700070BD70B504460D46A9B2A0B20323092205
:108E800003F058FEAA1D91B2A0B20323092203F0F9
:108E900051FEEA1C91B2A0B203231A4603F04AFE27
:108EA000A9B204F1090290B20F23032203F042FE9B
:108EB00070BD00002DE9F04105460E461446002C19
:108EC00007DA3146284600F0F0F8644205F10F0059
:108ED00085B26048844210DD401C94FBF0F00A210A
:108EE00090FBF1F201FB1200C7B23A463146284628
:108EF000FFF7F4FD05F10F0085B25748844210DDFD
:108F0000401C94FBF0F00A2190FBF1F201FB1200EF
:108F1000C7B23A4631462846FFF7E0FD05F10F009B
:108F200085B24E48844210DD401C94FBF0F00A21CB
:108F300090FBF1F201FB1200C7B23A4631462846D7
:108F4000FFF7CCFD05F10F0085B24548844210DDE6
:108F5000401C94FBF0F00A2190FBF1F201FB12009F
:108F6000C7B23A4631462846FFF7B8FD05F10F0073
:108F700085B23C48844210DD401C94FBF0F00A218D
:108F800090FBF1F201FB1200C7B23A463146284687
:108F9000FFF7A4FD05F10F0085B242F20F70844285
:108FA00010DD401C94FBF0F00A2190FBF1F201FB74
:108FB0001200C7B23A4631462846FFF78FFD05F149
:108FC0000F0085B2B4F57A7F11DB4FF47A7094FB11
:108FD000F0F00A2190FBF1F201FB1200C7B23A4611
:108FE00031462846FFF77AFD05F10F0085B2632C64
:108FF00010DD642094FBF0F00A2190FBF1F201FBFC
:109000001200C7B23A4631462846FFF767FD05F120
:109010000F0085B2092C10DD0A2094FBF0F00A2124
:1090200090FBF1F201FB1200C7B23A4631462846E6
:10903000FFF754FD05F10F0085B20A2094FBF0F113
:1090400000FB1140C7B23A4631462846FFF746FDBD
:10905000BDE8F081FFC99A3BFFE0F5057F969800D7
:109060003F420F009F8601002DE9F04106460F4662
:1090700014462046F7F70CF91FFA80F8002510E097
:10908000625D39463046FFF74BFC605D202803D116
:1090900006F10C0086B202E006F10E0086B2681CF2
:1090A00085B24545ECDBBDE8F08170B504460D4660
:1090B000EA1D91B2A21C90B20323082203F03AFDEC
:1090C00070BD70B505460C4604F10C0291B26A1CE5
:1090D00090B203231A4603F02DFD04F1090291B268
:1090E000EA1C90B203231A4603F024FDA21D91B29C
:1090F0006A1D90B203231A4603F01CFDE21C91B2D4
:10910000EA1D90B203231A4603F014FDA1B205F143
:10911000090290B203231A4603F00CFD70BD70B52E
:1091200005460C46221D91B2A8B20B23032203F080
:1091300001FD221D91B205F1090290B20B23032219
:1091400003F0F8FC04F1090291B2EA1C90B2032387
:10915000062203F0EFFC221D91B2EA1C90B203F04C
:109160002BFE221D91B205F1080290B203F024FEFD
:10917000E01C03B2281D02B2E01C01B2681C00B260
:1091800001F01CFDE01C03B205F10A0002B2E01C74
:1091900001B2E81D00B201F011FDA01C03B205F1FF
:1091A000090002B2A01C01B2A81C00B201F006FD29
:1091B000601C03B205F1080002B2601C01B2E81C99
:1091C00000B201F0FBFC23B2E81D02B221B2281D5F
:1091D00000B201F0F3FC70BD70B505460C46A1B2BB
:1091E000A8B20F23032203F0A5FCA1B2EA1C90B29F
:1091F0000323062203F09EFCA21D91B2EA1C90B24A
:109200000323072203F096FC04F10C0291B2EA1C3E
:1092100090B20323062203F08DFCA21C91B205F14B
:10922000090290B20523022203F084FC04F1080233
:1092300091B205F1090290B20523022203F07AFCF3
:10924000601D03B205F10B0002B2E01C01B205F192
:109250000B0000B201F0B2FC04F10B0003B205F107
:109260000B0002B204F1090001B205F10B0000B2DB
:1092700001F0A4FC621C91B205F1090290B203F066
:109280009BFDE21C91B205F1080290B203F094FD3F
:10929000621D91B205F1080290B203F08DFD04F158
:1092A000090291B205F1080290B203F085FD04F1C4
:1092B0000B0291B205F1080290B203F07DFD04F1BA
:1092C0000D0291B205F1090290B203F075FD70BD77
:1092D00070B504460D46AA1C91B2A0B20B2303221E
:1092E00003F028FCA9B2A21C90B20323082203F0C9
:1092F00021FC05F10C0291B2A21C90B203230822BA
:1093000003F018FCAA1C91B204F1090290B20323E5
:109310001A4603F00FFC05F10A0291B204F10902AA
:1093200090B203231A4603F005FC6A1C91B2621C3A
:1093300090B203F041FDEA1C91B2E21C90B203F03E
:109340003BFD05F10D0291B2621C90B203F034FDB9
:1093500005F10B0291B2E21C90B203F02DFDEA1C64
:1093600091B204F1080290B203F026FD6A1C91B29A
:1093700004F10A0290B203F01FFD05F10B0291B255
:1093800004F1080290B203F017FD05F10D0291B24D
:1093900004F10A0290B203F00FFD70BD70B50446EF
:1093A0000D46EA1C91B2A0B20923032203F0C2FBCE
:1093B000A9B2A0B20323092203F0BCFB05F10C0201
:1093C00091B2A0B20323092203F0B4FBEA1C91B2CC
:1093D00004F1090290B20923032203F0ABFB6A1CDB
:1093E00091B204F1090290B203F0E6FCAA1C91B21A
:1093F00004F1090290B203F0DFFCAA1C91B204F15F
:109400000A0290B203F0D8FCEA1C91B204F10802FF
:1094100090B203F0D1FC05F10B0291B204F1080205
:1094200090B203F0C9FC05F10D0291B204F10902FA
:1094300090B203F0C1FC05F10C0291B204F10902F3
:1094400090B203F0B9FC05F10C0291B204F10A02EA
:1094500090B203F0B1FC70BD70B504460D46A9B2E0
:10946000A0B203230C2203F065FB05F10C0291B2BC
:10947000A0B203230C2203F05DFBAA1D91B2E21CF3
:1094800090B20323062203F055FBEA1C91B2A0B26E
:109490000923032203F04EFB70BD70B504460D4650
:1094A000A9B2A0B203230C2203F044FBAA1D91B27F
:1094B000E21C90B20323062203F03CFBEA1C91B2AB
:1094C000A0B20C23032203F035FB70BD70B5044637
:1094D0000D46EA1C91B2A0B20923032203F02AFB35
:1094E000EA1C91B2E21C90B203F066FCAA1C91B295
:1094F000621C90B203F060FC6A1C91B2A21C90B294
:1095000003F05AFCAA1C91B2A21C90B203F054FCC6
:10951000A9B2E21C90B20323062203F00BFB6A1CE3
:1095200091B204F1080290B203231A4603F002FB41
:1095300005F10B0291B2E21C90B203F03DFC05F183
:109540000C0291B2621C90B203F036FC05F10C02E1
:1095500091B2A21C90B203F02FFC05F10D0291B262
:10956000A21C90B203F028FC05F10C0291B2E21C9F
:1095700090B20323062203F0DDFA05F10B0291B24B
:1095800004F1080290B203F017FC05F10C0291B24D
:1095900004F1090290B203F00FFC05F10C0291B244
:1095A00004F1090290B203F007FC05F10C0291B23C
:1095B00004F10A0290B203F0FFFB05F10D0291B233
:1095C00004F1090290B203F0F7FB05F10A0291B22F
:1095D00004F1090290B20223032203F0ABFAEA1D60
:1095E00091B2A21D90B20323062203F0A3FA70BD2C
:1095F00070B505460C46A1B2A8B20F23032203F0B2
:1096000099FAA1B205F1090290B20F23032203F0E7
:1096100091FAA21D91B2EA1C90B20323062203F034
:1096200089FA70BD70B504460D46A9B2A0B20323F5
:109630000C2203F07FFA05F10C0291B2A0B20323D1
:109640000C2203F077FAEA1C91B2221D90B2092392
:10965000042203F06FFA70BD70B505460C46A1B246
:10966000A8B20F23032203F065FA621D91B2EA1C2F
:1096700090B20523032203F05DFA221D91B26A1D08
:1096800090B203F099FB04F10A0291B26A1D90B204
:1096900003F092FBA01D03B2A81D02B2E01C01B2B0
:1096A000A81D00B201F08AFA601D03B2E81D02B2E3
:1096B000A01C01B2E81D00B201F080FA201D03B227
:1096C00005F1080002B2601C01B205F1080000B209
:1096D00001F074FAE01C03B205F1090002B221B2F4
:1096E00000B201F06BFAA01C03B205F10A0002B24D
:1096F00021B200B201F062FA601C03B205F10B0066
:1097000002B221B200B201F059FA04F10B0003B227
:10971000A81D02B204F1080001B2A81D00B201F0B8
:109720004DFA04F10C0003B2E81D02B204F1090085
:1097300001B2E81D00B201F041FA04F10D0003B2DC
:1097400005F1080002B204F10A0001B205F10800B7
:1097500000B201F033FA04F10E0003B205F1090082
:1097600002B204F10B0001B205F1090000B201F0F0
:1097700025FA04F10E0003B205F10A0002B204F169
:109780000C0001B205F10A0000B201F017FA04F171
:109790000E0003B205F10B0002B204F10D0001B29C
:1097A00005F10B0000B201F009FA70BD70B5044676
:1097B0000D46A9B2A0B20F23032203F0BBF905F1B5
:1097C0000C0291B2A0B203230C2203F0B3F970BDD6
:1097D00070B505460C46A1B2A8B20F23032203F0D0
:1097E000A9F9A1B205F1090290B20F23032203F0F7
:1097F000A1F9601D03B2E81C02B2601C01B2E81CB2
:1098000000B201F0DBF9601D03B205F1080002B2FD
:10981000601C01B205F1080000B201F0CFF9A01DF3
:1098200003B2281D02B2A01C01B2281D00B201F033
:10983000C5F9A01D03B2E81D02B2A01C01B2E81DCB
:1098400000B201F0BBF9E21C91B26A1D90B205238F
:10985000022203F06FF970BD70B505460C46A1B247
:10986000A8B20F23032203F065F9A1B205F10902A2
:1098700090B20F23032203F05DF9601D03B2E81CD0
:1098800002B2601C01B2E81C00B201F097F9A01D01
:1098900003B2281D02B2A01C01B2281D00B201F0C3
:1098A0008DF904F1080003B2681D02B2201D01B257
:1098B000681D00B201F082F904F10A0003B2A81D8C
:1098C00002B2A01D01B2A81D00B201F077F904F1A7
:1098D0000C0003B2E81D02B204F1080001B2E81D59
:1098E00000B201F06BF904F10D0003B205F10800BC
:1098F00002B204F1090001B205F1080000B201F062
:109900005DF970BD70B504460D46A9B2A21C90B2B7
:109910000323082203F00EF905F10C0291B2A21CF8
:1099200090B20323082203F005F9AA1C91B2A0B259
:109930000B23032203F0FEF8AA1C91B204F10902E2
:1099400090B20B23032203F0F5F86A1C91B2621C5B
:1099500090B203F031FAEA1C91B2E21C90B203F02B
:109960002BFA6A1C91B204F10A0290B203F024FAB5
:10997000EA1C91B204F1080290B203F01DFA05F15D
:109980000B0291B2E21C90B203F016FA05F10D023F
:1099900091B2621C90B203F00FFA05F10B0291B282
:1099A00004F1080290B203F007FA05F10D0291B23A
:1099B00004F10A0290B203F0FFF970BD70B50546DC
:1099C0000C46A1B2A8B20F23032203F0B3F8A1B250
:1099D000EA1C90B20323062203F0ACF8E21D91B218
:1099E000EA1C90B20323062203F0A4F8E21C91B211
:1099F00005F1080290B203F0DFF9A21D91B205F162
:109A0000080290B203F0D8F904F1080003B205F19E
:109A1000090002B2601C01B205F1090000B201F0B8
:109A2000CDF8A21C91B205F10A0290B203F0C4F97C
:109A3000E21D91B205F10A0290B203F0BDF9E21CF9
:109A400091B205F10A0290B20423022203F072F8E7
:109A500070BD70B505460C46A1B2A8B20F23032213
:109A600003F068F8A1B2EA1C90B20323062203F0C7
:109A700061F8E21D91B2EA1C90B20323062203F0C2
:109A800059F8E21C91B205F1080290B203F094F982
:109A9000A21D91B205F1080290B203F08DF904F114
:109AA000080003B205F1090002B2601C01B205F121
:109AB000090000B201F082F8A21C91B205F10A027D
:109AC00090B203F079F9E21D91B205F10A0290B269
:109AD00003F072F9E21C91B205F10A0290B204237C
:109AE000022203F027F804F10A0291B2AA1D90B2F3
:109AF00003F062F904F10A0291B2EA1D90B2022366
:109B0000032203F017F804F10C0291B205F10802E8
:109B100090B203F051F904F10B0291B205F10A027F
:109B200090B203F049F904F10C0291B205F1090277
:109B300090B203231A4602F0FDFF70BD70B50446D3
:109B40000D46A9B2A21C90B20323082202F0F2FF34
:109B50006A1C91B204F1080290B203231A4602F083
:109B6000E9FF6A1C91B2621C90B203231A4602F00C
:109B7000E1FFAA1C91B204F10A0290B2032302226F
:109B800002F0D8FFAA1C91B2A0B20423032202F073
:109B9000D1FF6A1D91B2621C90B20223032202F02F
:109BA000C9FFAA1D91B2A21C90B20223072202F0A3
:109BB000C1FFEA1D91B2E21C90B20223072202F01B
:109BC000B9FF05F1080291B204F1080290B2022334
:109BD000032202F0AFFF05F1090291B204F109027C
:109BE00090B20423032202F0A5FF05F10B0291B20B
:109BF00004F1080290B203231A4602F09BFF05F11C
:109C00000C0291B2A21C90B20323082202F092FF30
:109C100005F10B0291B2621C90B203231A4602F0C6
:109C200089FF05F10A0291B2A0B20323022202F0D9
:109C300081FF70BD70B504460D46A9B2A0B20323E2
:109C40000C2202F077FFEA1C91B2221D90B20C2385
:109C5000032202F06FFF70BD70B504460D46A9B235
:109C6000A0B20F23032202F065FF05F10C0291B2AE
:109C7000A0B203230C2202F05DFFA9B204F1090295
:109C800090B20C23032202F055FF70BD70B505465B
:109C90000C46A1B2A8B203231A4602F04BFFA1B2B0
:109CA00005F1090290B203231A4602F043FFE21CB9
:109CB00091B26A1C90B203231A4602F03BFFE21CE9
:109CC00091B205F1080290B203231A4602F032FF66
:109CD000A21D91B2AA1C90B203231A4602F02AFFD9
:109CE000A21D91B2EA1D90B203231A4602F022FF90
:109CF00004F1090291B2EA1C90B20323062202F099
:109D000019FF04F10C0291B22A1D90B20323042220
:109D100002F010FF70BD70B505460C46A1B2A8B2A6
:109D200003231A4602F006FFA1B205F1090290B220
:109D300003231A4602F0FEFEE21C91B26A1C90B2A6
:109D400003231A4602F0F6FEE21C91B205F1080266
:109D500090B203231A4602F0EDFEA21D91B2AA1C96
:109D600090B203231A4602F0E5FEA21D91B2EA1D4D
:109D700090B203231A4602F0DDFE04F1090291B20B
:109D8000EA1C90B20323062202F0D4FE04F10C0276
:109D900091B22A1D90B20323042202F0CBFEA1B29D
:109DA00005F1090290B203231A4602F0C3FEA1B2E4
:109DB00005F1120290B203231A4602F0BBFEE21C28
:109DC00091B205F10A0290B203231A4602F0B2FEE4
:109DD000E21C91B205F1110290B203231A4602F07F
:109DE000A9FEA21D91B205F10B0290B203231A46FF
:109DF00002F0A0FEA21D91B205F1100290B2032361
:109E00001A4602F097FE04F1090291B205F10C0224
:109E100090B20323062202F08DFE04F10C0291B2EF
:109E200005F10D0290B20323042202F083FE70BDFF
:109E300070B505460C4604F1090291B22A1D90B294
:109E40000623042202F076FEA21D91B2EA1C90B213
:109E50000323062202F06EFEA1B2A8B203231A4623
:109E600002F068FEA1B2A8B203231A4602F062FE15
:109E7000A1B205F1090290B203231A4602F05AFE7C
:109E8000E21C91B26A1C90B20223032202F052FE3D
:109E9000E21C91B205F1080290B20223032202F003
:109EA00049FE601D03B2281D02B2601D01B2A81C4C
:109EB00000B200F083FE601D03B205F1090002B29A
:109EC000601D01B2E81D00B200F078FEA21C91B244
:109ED000EA1C90B202F070FFA21C91B205F10802D8
:109EE00090B202F069FF221D91B22A1D90B202F0D9
:109EF00063FF221D91B2EA1D90B202F05DFFA21D28
:109F000091B2AA1C90B202F057FFA21D91B205F1C6
:109F1000090290B202F050FF70BD70B504460D46C4
:109F200005F1090291B2E21C90B206231A4602F032
:109F300001FE70BD70B504460D46EA1D91B2A21C2B
:109F400090B20323082202F0F5FD2A1D91B2621D92
:109F500090B20823032202F0EDFD70BD2DE9F0431D
:109F600006460F4690460320A0EB480900244546CC
:109F70003EE07A1B91B2321990B202F01DFF7A1BBB
:109F800091B2321B90B202F017FF3A1B91B27219D4
:109F900090B202F011FF3A1B91B2721B90B202F024
:109FA0000BFF7A1991B2321990B202F005FF7A19BB
:109FB00091B2321B90B202F0FFFE3A1991B27219BF
:109FC00090B202F0F9FE3A1991B2721B90B202F00F
:109FD000F3FEB9F1000F04DA062000EB840081449F
:109FE00005E0601B0A2101EB800081446D1E641CAA
:109FF000AC42BED9BDE8F0832DE9F04F06460F46CE
:10A00000904699460024C9F100054FEA4800C0F186
:10A01000020A9FED560AB0EE403A9FED540AF0EE68
:10A02000403A9FED520AB0EE404A00EE108AB8EE78
:10A03000C00AF0EE403A00EE109AB8EEC00AB0EE58
:10A04000404A84EE230AB0EE403A00BF00EE104AC8
:10A05000B8EEC00AC0EE030ABCEEE00A10EE100A29
:10A0600080B2301A00EE100AB8EEC00BB0EE405BC2
:10A07000781900EE100AB8EEC00BB0EE401BB0EE3F
:10A08000450B02F007FF00EE104AB8EEC00AC0EE22
:10A09000030ABCEEE00A10EE100A80B2304400EE73
:10A0A000100AB8EEC00BB0EE405B781900EE100A53
:10A0B000B8EEC00BB0EE401BB0EE450B02F0EAFE6E
:10A0C00000EE104AB8EEC00AC0EE030ABCEEE00A89
:10A0D00010EE100A80B2304400EE100AB8EEC00B49
:10A0E000B0EE405B781B00EE100AB8EEC00BB0EE8D
:10A0F000401BB0EE450B02F0CDFE00EE104AB8EE6C
:10A10000C00AC0EE030ABCEEE00A10EE100A80B2EC
:10A11000301A00EE100AB8EEC00BB0EE405B781BB0
:10A1200000EE100AB8EEC00BB0EE401BB0EE450BCF
:10A1300002F0B0FED346A3450BDC601C04460121AF
:10A1400001EB40008244E54203D1AB4501DC4FF016
:10A15000000BAB4505DD681C0546012101EB400005
:10A160008244002D7FF772AFBDE8F08F0000000041
:10A170002DE9FF4F82B00F9CBDF80800BDF80A2002
:10A180006C4909688B4202D306B0BDE8F08F6A497A
:10A1900009688C4200D3F7E71918664D2D68A9426B
:10A1A00003D364490988C91A88B2A118624D2D6881
:10A1B000A94203D360490988091B8AB25F4909880B
:10A1C00061BB002127E0002521E0DFF874C1DCF845
:10A1D000006004EB010CDFF85C81D8F800800CFB18
:10A1E00008FC06EB8C0603EB050C06EB8C0601FB6A
:10A1F00000FC1FFA8CF707EB050C1FFA8CF7DDF853
:10A2000010C05CF827C0C6F800C06E1CB5B285420D
:10A21000DBDB4D1CA9B29142D5DB88E047490988B8
:10A22000012938D1002533E000262DE0DFF810B1F8
:10A23000DBF8001004EB050BDFF8F8E0DEF800E0D7
:10A240000BFB0EFB0BEB4B0B594403EB060B0BEB21
:10A250004B0B594405FB00FB1FFA8BFC0CEB060B68
:10A260001FFA8BFCDDF810B05BF82C70C7F30748C1
:10A27000C7F3072907F0FF0A81F800A081F80190D1
:10A2800081F80280711C8EB28642CFDB691C8DB2D0
:10A290009542C9DB4BE029490988042947D10025AB
:10A2A00043E000213DE0DFF898B0DBF8006004EB0C
:10A2B000050BDFF880E0DEF800E00BFB0EFB06EBA1
:10A2C0004B0603EB010B06EB4B0605FB00FB1FFAED
:10A2D0008BFC0CEB010B1FFA8BFCDDF810B05BF86C
:10A2E0002C70C7F30748C7F3072A07F0FF094FF0A0
:10A2F000F00B0BEB281B0BF0FF0BCDF804B00AF0B2
:10A30000F00B0BEB291B0BF0FF0BCDF800B0DDF8C9
:10A3100000B086F800B0DDF804B086F801B04E1C3D
:10A32000B1B28142BFDB691C8DB29542B9DB00BF7F
:10A330002AE70000DC130020E0130020E4130020D3
:10A34000D81300202DE9FF41BDF80050BDF8026090
:10A3500028480068824201D3BDE8FF812648006892
:10A36000834200D3F8E7501922490968884203D391
:10A3700020480088801A85B298191F4909688842C8
:10A3800003D31D480088C01A86B21C4800880428E0
:10A390002DD1002029E0002123E0DFF864C0DCF8A3
:10A3A000004003EB000CDFF84C80D8F800800CFB79
:10A3B00008FC04EB4C0402EB010C04EB4C04BDF86C
:10A3C00000C00CFB00FC1FFA8CF707EB010C1FFA16
:10A3D0008CF7DDF804C03CF817C0A4F800C04C1C92
:10A3E000A1B2A942D9DB411C88B2B042D3DB00BF85
:10A3F000B2E70000DC130020E0130020E41300208B
:10A40000D81300202DE9FF4FDDE90E8EDDF834C0B2
:10A41000BDF80070BDF80290314C2468A24201D30F
:10A42000BDE8FF8F2F4C2468A34200D3F8E7D4196E
:10A430002B4D2D68AC4203D3294C2488A41AA7B213
:10A4400003EB0904274D2D68AC4204D3254C248826
:10A45000E41A1FFA84F9244C2488042C3DD10024EA
:10A4600039E0002533E002EB050B1FFA8BF003EB1C
:10A47000040B1FFA8BF1604525DB704523DC414559
:10A4800021DBDDF840B059451DDCDFF860B0DBF8BA
:10A490000060DFF84CB0DBF800B001FB0BFB06EB13
:10A4A0004B0606EB4006BDF800B00BFB04FB1FFAA1
:10A4B0008BFA0AEB050B1FFA8BFADDF804B03BF8B8
:10A4C0001AB0A6F800B005F1010B1FFA8BF5BD42DA
:10A4D000C9DB651CACB24C45C3DB00BFA0E7000084
:10A4E000DC130020E0130020E4130020D813002028
:10A4F0002DE9FF41BDF80040BDF802602948006821
:10A50000824201D3BDE8FF8127480068834200D31F
:10A51000F8E7101923490968884203D321480088C5
:10A52000801A84B2981920490968884203D31E48CA
:10A530000088C01A86B21D480088042830D1002047
:10A540002CE0002126E0DFF868C0DCF8005003EBC7
:10A55000000CDFF85080D8F800800CFB08FC05EBFD
:10A560004C0502EB010C05EB4C05BDF800C00CFBE3
:10A5700000FC1FFA8CF7A4EB010CACF1010CBC44FD
:10A580001FFA8CF7DDF804C03CF817C0A5F800C02E
:10A590004D1CA9B2A142D6DB411C88B2B042D0DB2F
:10A5A00000BFAFE7DC130020E0130020E41300201D
:10A5B000D81300202DE9FF4FDDE90E8EDDF834C001
:10A5C000BDF80060BDF80290324C2468A24201D36D
:10A5D000BDE8FF8F304C2468A34200D3F8E79419FC
:10A5E0002C4D2D68AC4203D32A4C2488A41AA6B261
:10A5F00003EB0904284D2D68AC4204D3264C248873
:10A60000E41A1FFA84F9254C2488042C40D1002434
:10A610003CE0002536E002EB050B1FFA8BF003EB64
:10A62000040B1FFA8BF1604528DB704526DC4145A1
:10A6300024DBDDF840B0594520DCDFF864B0DBF8FE
:10A640000070DFF850B0DBF800B001FB0BFB07EB4C
:10A650004B0707EB4007BDF800B00BFB04FB1FFAEC
:10A660008BFAA6EB050BABF1010BD3441FFA8BFA67
:10A67000DDF804B03BF81AB0A7F800B005F1010B03
:10A680001FFA8BF5B542C6DB651CACB24C45C0DB8E
:10A6900000BF9DE7DC130020E0130020E41300203E
:10A6A000D81300202DE9FF4F86B01D46079E96F86F
:10A6B0000080079E76780596934E3668B24202D3A4
:10A6C0000AB0BDE8F08F914E3668B54200D3F7E787
:10A6D00002EB08068C4F3F68BE4204D38A4E368890
:10A6E000B61A1FFA86F8059E2E44884F3F68BE4270
:10A6F00004D3864E3688B61AB6B20596059E2E4409
:10A70000761E36B2049602EB0806761E34B2079E19
:10A7100096F80290032606EB490011462B46E6E028
:10A72000079E365CFF2E51D1BDF81870861CB742CB
:10A7300049DD471CDDF81CC01CF80760871CDDF8EC
:10A740001CC01CF807A04FF0030C0CEB460C079F35
:10A7500017F80C7003974FF0040C0CEB460C079F96
:10A7600017F80C700297019101EB0A077F1E0FFA90
:10A7700087FEA64500DDA646019F19E0DFF890B1EF
:10A78000DBF800C0DFF880B1DBF800B04FEA4B0B1C
:10A790000BFB03CC0CEB470CDDF80CB08CF801B0D4
:10A7A000DDF808B08CF800B007F1010C0FFA8CF757
:10A7B0007745E3DD01EB0A0739B2A14202DD11461C
:10A7C0005F1C3BB200BFC61CB0B290E0079E365C77
:10A7D000FE2E50D1471CDDF81CC01CF80760871CFA
:10A7E000DDF81CC01CF807E04FF0030C0CEB460C26
:10A7F000079F17F80C7003974FF0040C0CEB460CF6
:10A80000079F17F80C700297019303EB0E077F1E4A
:10A810003FB20097019B9A4623E0174619E0DFF804
:10A82000F0B0DBF800C0DFF8E0B0DBF800B04FEAD2
:10A830004B0B0BFB0ACC0CEB470CDDF80CB08CF887
:10A8400001B0DDF808B08CF800B007F1010C0FFA88
:10A850008CF702EB080CBC45E1DC0AF101070FFAAA
:10A8600087FA009FBA45D8DD114603EB0E073BB2CD
:10A87000C71CB8B23BE0DDF81CB01BF800604FF01D
:10A88000030E0EEB460EDDF81CB01BF80EC04FF0A9
:10A89000040E0EEB460EDDF81CB01BF80EA00AEB02
:10A8A0000C2B1FFA8BFBCDF80CB0DFF864B0DBF893
:10A8B0000070DFF854B0DBF800B003FB0BFB07EBD4
:10A8C0004B0707EB4107DDF80CB0A7F800B001F12A
:10A8D000010B0FFA8BF1A14204DD114603F1010BCC
:10A8E0000FFA8BF300F1010B1FFA8BF000BFBDF8DC
:10A8F0001860864205DDA1427FF712AF049EB34285
:10A90000FADD00BFDCE60000DC130020E0130020CD
:10A91000D81300202DE9FF4F87B014461E46DDF8FE
:10A9200050E0089D95F80090089D6D780695A04D23
:10A930002D68AC4202D30BB0BDE8F08F9D4D2D6861
:10A94000AE4200D3F7E704EB0905994F3F68BD42DB
:10A9500004D3974D2D882D1B1FFA85F9069D35448C
:10A96000944F3F68BD4204D3924D2D882D1BADB24C
:10A970000695069D35446D1E2DB2059504EB09051F
:10A980006D1E2BB2089D95F802A0032505EB4A0128
:10A9900022463046FFE0089D6D5CFF2D63D1BDF877
:10A9A0001C708D1CAF425BDD4D1CDDF820C01CF817
:10A9B00005708D1CDDF820C01CF805B04FF0030CAD
:10A9C0000CEB470C089D15F80C5004954FF0040C47
:10A9D0000CEB470C089D15F80C500395029202EB06
:10A9E0000B056D1E2DB20195019D9D4200DD019369
:10A9F000029D28E0754522DBDDF858C065451EDC68
:10AA0000DDF854C060451ADBDDF85CC0604516DC3B
:10AA1000DFF8A481D8F800C0DFF89481D8F800806E
:10AA20004FEA480808FB00CC0CEB450CDDF8108021
:10AA30008CF80180DDF80C808CF8008000BF05F1F7
:10AA4000010C0FFA8CF5DDF804C06545D2DD02EB90
:10AA50000B052AB29A4202DD2246451C28B200BFED
:10AA6000CD1CA9B297E0089D6D5CFE2D57D14D1C01
:10AA7000089F17F805C08D1C089F7D5D049503276E
:10AA800007EB4C07089DED5D0395042707EB4C078A
:10AA9000089DED5D02950190049D05446D1E2DB24B
:10AAA00000950198074630E0254628E0754522DBF1
:10AAB000DDF8588045451EDCDDF8548047451ADB3B
:10AAC000DDF85C80474516DCDFF8ECB0DBF8008091
:10AAD000DFF8DCB0DBF800B04FEA4B0B0BFB07886C
:10AAE00008EB4508DDF80CB088F801B0DDF808B0D7
:10AAF00088F800B000BF05F101080FFA88F504EBF3
:10AB00000908A845D2DC7D1C2FB2009DAF42CBDDE9
:10AB10002246049D054428B2CD1CA9B23BE0089F03
:10AB20007D5C4FF0030808EB4508089F17F808C044
:10AB30004FF0040808EB4508089F17F808B00BEB26
:10AB40000C27BFB2049772451BDB169FBA4218DC74
:10AB5000159FB84215DB179FB84212DCDFF858800A
:10AB6000D8F80070DFF84880D8F8008000FB08F8BB
:10AB700007EB480707EB4207DDF81080A7F80080D5
:10AB800000BF571C3AB29A4202DD2246471C38B237
:10AB90004F1CB9B200BFBDF81C508D4205DD9A4272
:10ABA0007FF7F9AE059DA842FADD00BFC3E60000BD
:10ABB000DC130020E0130020D81300202DE9F04F13
:10ABC0008AB004460D4691469A465A48007810B914
:10ABD0000AB0BDE8F08FA14503DACDF82490A14674
:10ABE000099CAA4503DACDF824A0AA46099D55453B
:10ABF0000ED151480068854209D2264605E0A9B227
:10AC0000B0B202F0D9F8701C06B24E45F7DD8EE006
:10AC10004C450ED1494800688442F8D2AEB205E0F6
:10AC2000A0B2314602F0C8F8701C86B25645F7DD76
:10AC30007DE000260027B34600200890079006908C
:10AC40000590049080460390029001900090A9EB3B
:10AC5000040006B2002E01DA704206B2AAEB05002B
:10AC600007B2002F01DA784207B2A3460895A14542
:10AC700003DB01200790069003E04FF0FF300790C0
:10AC80000690AA4503DB01200590049003E04FF0F5
:10AC9000FF3005900490BE420CDB0020079004902A
:10ACA000B046304606EBD071491009B203910297C5
:10ACB00001960BE0002006900590B846384607EB59
:10ACC000D071491009B203910296019700200090BB
:10ACD00028E0089A91B21FFA8BF002F06DF8DDE9D6
:10ACE0000210084400B20390039840450DDB03981E
:10ACF000A0EB080000B20390079858440FFA80FBBD
:10AD000005990898084400B20890069858440FFA2C
:10AD100080FB04990898084400B208900098401CF1
:10AD200000B20090DDE900018842D2DD00BF00BF23
:10AD30004EE70000D4130020E0130020DC130020B5
:10AD40002DE9F04304460D4616461F462B48007871
:10AD500008B9BDE8F083A019401E1FFA80F8E81971
:10AD6000401E1FFA80F926480068804504D3244815
:10AD70000088401E1FFA80F822480068814504D3ED
:10AD800020480088401E1FFA80F906B9E1E707B99C
:10AD9000DFE71B480068844200D3DAE719480068FF
:10ADA000854200D3D5E7A019401E02B22BB229B2CA
:10ADB00020B2FFF703FFE819401E03B222B229B206
:10ADC00020B2FFF7FBFEE819401E03B2A019401E97
:10ADD00002B2E819401E01B220B2FFF7EFFEE919F6
:10ADE000491E0BB2A119491E0AB2A119491E08B287
:10ADF00029B2FFF7E3FE00BF00BFAAE7D41300208B
:10AE0000DC130020E01300202DE9F04F2DED108B16
:10AE100087B0B0EE40ABB0EE41BBB0EE429BC7484E
:10AE2000007820B907B0BDEC108BBDE8F08FC448A6
:10AE3000008804287ED13AEE490BBDEEC00B10EE1F
:10AE4000100A07B23AEE090BB7EE001B30EE010B09
:10AE5000BDEEC00B10EE100A0FFA80F83BEE490B66
:10AE6000BDEEC00B10EE100A0FFA80F93BEE090B95
:10AE7000B7EE001B30EE010BBDEEC00B10EE100A5A
:10AE80000FFA80FAAF480068874200D3CAE7B8F1EA
:10AE9000000F00DAC6E7AC480068814500D3C1E77F
:10AEA000BAF1000F00DABDE7002F00DA0027A5484D
:10AEB0000068804504D3A3480088401E0FFA80F83C
:10AEC000B9F1000F01DA4FF000099F480068824590
:10AED00004D39D480088401E0FFA80FA3D4627E1C2
:10AEE0004E4620E100EE105AB8EEC00B30EE4AEBB1
:10AEF00000EE106AB8EEC00B30EE4BDB2EEE0E1BF0
:10AF00000DEE0D1BB0EE410B28F0FAFBB0EE40CB7E
:10AF1000B6EE000B39EE000BB4EECC0BF1EE10FAEE
:10AF20007DD9B6EE000B39EE400BB4EECC0BF1EE52
:10AF300010FA00E000E173D2B6EE003B39EE433B7D
:10AF40003CEE433BB7EE004B34EE438BDFF8FCB1F5
:10AF5000DBF80040DFF8ECB1DBF800B04FEA4B0B58
:10AF60000BFB064404EB450494F801B0CDF818B08F
:10AF700094F800C0DDF818B04FEA2B1B00EE10BAB1
:10AF8000DDF818B00BF00F0B00EE90BA4FEA2C1B57
:10AF900001EE10BA0CF00F0B01EE90BADFF8B0B171
:10AFA0009BF800B04FEA2B1B02EE10BADFF8A0B1FD
:10AFB0009BF800B00BF00F0B02EE90BADFF894B1E3
:10AFC0009BF800B04FEA2B1B06EE10BADFF884B1F5
:10AFD0009BF800B00BF00F0B06EE90BAB8EE423BB8
:10AFE00028EE033BB7EE004B34EE484BB8EE405B27
:10AFF00004EE053BB0EE437BB8EE623B28EE033B2C
:10B00000B7EE004B34EE484BB8EE605B04EE053B08
:10B01000B0EE43FBB8EE463B28EE033B01E080E098
:10B0200070E0B7EE004B34EE484BB8EE415B04EEF7
:10B03000053B8DED043BB8EE663B28EE033BB7EED7
:10B04000004B34EE484BB8EE615B04EE053B8DEDF2
:10B05000023BB0EE473BB6EE004B33EE043BBCEE9A
:10B06000C33B13EE10BA0BF0FF00B0EE4F3BB6EE51
:10B07000004B33EE043BBCEEC33B13EE10BA0BF0B7
:10B08000FF019DED043BB6EE004B33EE043BBCEEFE
:10B09000C33B13EE10BA0BF0FF029DED023BB6EE80
:10B0A000004B33EE043BBCEEC33B13EE10BA0BF087
:10B0B000FF03002800DA00200F2800DD0F20002900
:10B0C00000DA00210F2900DD0F21002A00DA00221A
:10B0D0000F2A00DD0F22002B00DA00230F2B00DDEA
:10B0E0000F2301EB001B0BF0FF0E03EB021B0BF019
:10B0F000FF0BCDF804B084F801E0DDF804B084F86B
:10B1000000B00EE0114804680E480068400000FBE3
:10B11000064404EB45040E48007860700D48007842
:10B120002070701C06B256457FF7DCAE681C05B275
:10B1300045457FF7D5AE00BF00BF73E6D4130020AE
:10B14000E4130020DC130020E0130020D8130020BB
:10B15000EA130020EB1300202DE9F04F2DED108BAA
:10B1600089B0B0EE40BBB0EE41CBB0EE428BB0EE5A
:10B1700043DBD948007820B909B0BDEC108BBDE89D
:10B18000F08FD648008804287ED13BEE480BBDEEF8
:10B19000C00B10EE100A07B23BEE080BB7EE001B17
:10B1A00030EE010BBDEEC00B10EE100A0FFA80F866
:10B1B0003CEE480BBDEEC00B10EE100A0FFA80F902
:10B1C0003CEE080BB7EE001B30EE010BBDEEC00BE2
:10B1D00010EE100A0FFA80FAC1480068874200D3C7
:10B1E000CAE7B8F1000F00DAC6E7BE48006881453B
:10B1F00000D3C1E7BAF1000F00DABDE7002F00DA93
:10B200000027B7480068804504D3B5480088401E31
:10B210000FFA80F8B9F1000F01DA4FF00009B148D8
:10B220000068824504D3AF480088401E0FFA80FAB8
:10B230003D464BE14E4644E100EE105AB8EEC00BDD
:10B2400030EE4BFB00EE106AB8EEC00B30EE4CEB6C
:10B250002FEE0F1B0EEE0E1BB0EE410B28F050FA36
:10B26000B0EE40AB00200890B6EE000B38EE000BBD
:10B27000B4EECA0BF1EE10FA45D9B6EE000B38EE7B
:10B28000400BB4EECA0B00E024E1F1EE10FA0ED24E
:10B2900001200890B6EE000B38EE400B3AEE400B62
:10B2A000B7EE001B31EE400BB0EE409B2BE0B6EE4C
:10B2B000000B3DEE000BB4EECA0BF1EE10FA0FD806
:10B2C0008948046886480068400000FB064404EB97
:10B2D000450486480078607085480078207012E048
:10B2E000B6EE000B3DEE400BB4EECA0BF1EE10FAD9
:10B2F00009D801200890B6EE000B3DEE400B3AEE67
:10B30000400BB0EE409B089800287CD0DFF8D8B105
:10B31000DBF80040DFF8C8B1DBF800B04FEA4B0BB8
:10B320000BFB064404EB450494F801C094F800E0DC
:10B330004FEA2C1B00EE10BA0CF00F0B00EE90BA87
:10B340004FEA2E1B02EE90BA0EF00F0B06EE10BA6B
:10B35000DFF898B19BF800B04FEA2B1B06EE90BACD
:10B36000DFF888B19BF800B00BF00F0B01EE10BABC
:10B37000DFF87CB19BF800B04FEA2B1B01EE90BACE
:10B38000DFF86CB19BF800B00BF00F0B02EE10BAB7
:10B39000B8EE663B29EE033BB7EE004B34EE494B6B
:10B3A000B8EE405B04EE053BB0EE437BB8EE413BAC
:10B3B00029EE033BB7EE004B34EE494BB8EE605B31
:10B3C00004EE053B8DED063BB8EE613B29EE033BF9
:10B3D000B7EE004B34EE494BB8EE625B04EE053B32
:10B3E0008DED043BB8EE423B29EE033BB7EE004B3C
:10B3F00034EE494BB8EE465B04EE053B8DED023B67
:10B40000B0EE473B00E05AE0B6EE004B33EE043BB3
:10B41000BCEEC33B13EE10BA0BF0FF009DED063BF4
:10B42000B6EE004B33EE043BBCEEC33B13EE10BA5A
:10B430000BF0FF019DED043BB6EE004B33EE043BF9
:10B44000BCEEC33B13EE10BA0BF0FF029DED023BC6
:10B45000B6EE004B33EE043BBCEEC33B13EE10BA2A
:10B460000BF0FF03002800DA00200F2800DD0F207A
:10B47000002900DA00210F2900DD0F21002A00DA5F
:10B4800000220F2A00DD0F22002B00DA00230F2BF1
:10B4900000DD0F2301EB001B0BF0FF0BCDF804B018
:10B4A00003EB021B0BF0FF0BCDF800B0DDF804B08E
:10B4B00084F801B0DDF800B084F800B000BF701C63
:10B4C00006B256457FF7B8AE681C05B245457FF712
:10B4D000B1AE00BF00BF4FE6D4130020E41300203C
:10B4E000DC130020E0130020D8130020EA13002012
:10B4F000EB1300202DE9F05F2DED0A0B2DED108BE5
:10B50000B8B0B0EE409BB0EE41ABB0EE43DBB0EE76
:10B5100044EBF948007828B938B0BDEC108B0AB07C
:10B52000BDE8F09FF548008804287DD1B0EE000BFF
:10B530008DEE001B8DED361BB0EE000B8EEE001B6A
:10B54000B0EE41FB9DED361B21EE011B0FEE0F1BF4
:10B55000B0EE410B28F0D4F88DED340B9DED340B9B
:10B5600039EE400BBDEEC00B10EE100A07B29DED98
:10B57000340B39EE000BB7EE001B30EE010BBDEEC5
:10B58000C00B10EE100A0FFA80F89DED340B3AEE66
:10B59000400BBDEEC00B10EE100A0FFA80F99DEDC6
:10B5A000340B3AEE000BB7EE001B30EE010BBDEE94
:10B5B000C00B10EE100A0FFA80FAD14800688742DB
:10B5C00000D3A9E7B8F1000F00DAA5E7CD4800687D
:10B5D000814500D3A0E7BAF1000F00DA9CE7002F05
:10B5E00000DA0027C6480068804504D3C4480088B4
:10B5F000401E0FFA80F8B9F1000F01DA4FF0000990
:10B60000C0480068824504D3BE480088401E0FFA37
:10B6100080FA9DED4C0B27F0C3FF8DED320B9DEDB5
:10B620004C0B28F015F800E01BE38DED300B9DED81
:10B63000320B20EE0D1BB0EE002B81EE020B39EE2B
:10B6400040BB9DED300B20EE0D1BB0EE002B81EECC
:10B65000020B3AEE400B8DED2E0B9DED320B20EEE2
:10B660000D1BB0EE000B81EE002B32EE090B8DEDC1
:10B670002C0B9DED300B20EE0D1BB0EE000B81EE80
:10B68000002B32EE0A0B8DED2A0B9DED300B20EED8
:10B690000E0BB0EE001B80EE012B32EE09CB9DEDC0
:10B6A000320B20EE0E1BB0EE000B81EE002B3AEEBB
:10B6B000420B8DED280B9DED300B20EE0E1BB0EEF6
:10B6C000000B81EE002B39EE420B8DED260B9DED2C
:10B6D000320B20EE0E0BB0EE001B80EE012B32EE93
:10B6E0000A0B8DED240B9FED880B8DED220B9FED4A
:10B6F000860B8DED200B3D46AFE24E46A8E20020C2
:10B700001590149013900F900E900D9000EE105A1B
:10B71000B8EEC00B8DED1A0B00EE106AB8EEC00B40
:10B720008DED180B9DED2A0B9DED2E1B30EE411B70
:10B730009DED1A0B21EE001B9DED2C0B30EE4B2BDB
:10B740009DED180B02EE401B9DED2C0B9DED2E2B5D
:10B7500000EE021B9DED2A0B00EE4B1B8DED1E1B18
:10B760009DED1E0BB5EEC00BF1EE10FA05D29DED6E
:10B770001E0BB1EE400B8DED1E0B9DED2A1B9DEDBA
:10B780002E2B31EE421B21EE011B9DED2C2B32EEB8
:10B790004B3B9DED2C2B32EE4B2B03EE021BB0EE00
:10B7A000410B27F0ADFF8DED1C0B9DED1E0B9DEDAC
:10B7B0001C1B80EE012B8DED222B9DED240B9DEDAE
:10B7C000281B30EE411B9DED1A0B21EE000B9DED69
:10B7D000261B31EE4C2B9DED181B02EE410B9DED0F
:10B7E000261B9DED282B01EE020B9DED241B01EE87
:10B7F0004C0B8DED1E0B9DED1E0BB5EEC00BF1EE4F
:10B8000010FA05D29DED1E0BB1EE400B8DED1E0B17
:10B810009DED241B9DED282B31EE421B21EE011BDB
:10B820009DED262B32EE4C3B9DED262B32EE4C2B24
:10B8300003EE021BB0EE410B27F062FF8DED1C0BF7
:10B840009DED1E0B9DED1C1B80EE012B8DED202B25
:10B850009DED360BB6EE001B30EE011B9DED200B6F
:10B86000B4EEC01BF1EE10FA02D2012015905FE099
:10B870009DED360BB6EE001B30EE411B9DED200B0F
:10B88000B4EEC01BF1EE10FA02DD012014904FE07F
:10B89000012013909DED1A0B30EE4C2B9DED240BE7
:10B8A0009DED281B30EE410B22EE000B9DED181B89
:10B8B0009DED282B31EE422B9DED261B31EE4C1BCE
:10B8C00002EE410B8DED160B9DED160BB5EEC00B88
:10B8D000F1EE10FA1CD29DED200B9DED361B30EEE3
:10B8E000410BB6EE001B30EE010BB7EE001B31EE44
:10B8F000400B8DED100B1BE0D4130020E41300204F
:10B90000DC130020E0130020000000000000000015
:10B910009DED360BB6EE001B30EE411B9DED200B6E
:10B9200030EE410BB7EE001B31EE400B8DED100BEE
:10B93000159810B101200F9057E0B6EE000B3FEEC6
:10B94000001B9DED220BB4EEC01BF1EE10FA02D2EB
:10B9500001200F9049E0B6EE000B3FEE401B9DED3D
:10B96000220BB4EEC01BF1EE10FA02DD01200E90A6
:10B970003BE001200D909DED1A0B30EE4B2B9DED21
:10B980002A0B9DED2E1B30EE410B22EE000B9DEDA0
:10B99000181B9DED2E2B31EE422B9DED2C1B31EE15
:10B9A0004B1B02EE410B8DED160B9DED160BB5EE0C
:10B9B000C00BF1EE10FA0EDDB6EE000B3FEE401BB1
:10B9C0009DED220B30EE410BB7EE001B31EE400B2C
:10B9D0008DED0A0B09E0B6EE000B3FEE401B9DED2E
:10B9E000220B30EE410B8DED0A0B002009908346AF
:10B9F0001FED3B8B159840BB0F9830BB149868B176
:10BA00000E9810B1012009901FE00D98E8B14FF099
:10BA1000010B9DED0A0BB0EE408B16E01398A0B120
:10BA20000E9830B14FF0010B9DED100BB0EE408B36
:10BA30000BE00D9848B14FF0010B9DED100B9DED03
:10BA40000A1B20EE010BB0EE408B099848B9BBF100
:10BA5000000F16D0B7EE000BB4EEC08BF1EE10FA6B
:10BA60000FDB8148046881480068400000FB064401
:10BA700004EB45047E48007860707E4800782070B2
:10BA8000E4E0BBF1000FFBD0B5EEC08BF1EE10FA95
:10BA9000F6DDDFF8D4C1DCF80040DFF8D0C1DCF817
:10BAA00000C04FEA4C0C0CFB064404EB450494F830
:10BAB00001E094F800C0CDF820C04FEA2E1C00EE43
:10BAC00010CA0EF00F0C00EE90CADDF820C04FEA4D
:10BAD0002C1C01EE10CADDF820C00CF00F0C01EE9A
:10BAE00090CADFF88CC19CF800C04FEA2C1C02EE13
:10BAF00010CADFF87CC19CF800C00CF00F0C02EEFD
:10BB000090CADFF870C19CF800C04FEA2C1C06EE0A
:10BB100010CADFF860C19CF800C00CF00F0C06EEF4
:10BB200090CAB8EE423B28EE033BB7EE004B34EE32
:10BB3000484BB8EE405B04EE053BB0EE437BB8EEFD
:10BB4000623B28EE033BB7EE004B34EE484BB8EEB9
:10BB5000605B04EE053B8DED063BB8EE463B28EE00
:10BB6000033BB7EE004B34EE484BB8EE415B04EEBE
:10BB7000053B8DED043BB8EE663B28EE033BB7EE8C
:10BB8000004B34EE484BB8EE615B04EE053B8DEDA7
:10BB9000023BB0EE473BB6EE004B33EE043BBCEE4F
:10BBA000C33B13EE10CA0CF0FF009DED063BB6EE52
:10BBB000004B33EE043BBCEEC33B13EE10CA0CF05B
:10BBC000FF019DED043BB6EE004B33EE043BBCEEB3
:10BBD000C33B13EE10CA0CF0FF029DED023BB6EE24
:10BBE000004B33EE043BBCEEC33B13EE10CA0CF02B
:10BBF000FF03002800DA00200F2800DD0F200029B5
:10BC000000DA00210F2900DD0F21002A00DA0022CE
:10BC10000F2A00DD0F22002B00DA00230F2B00DD9E
:10BC20000F2301EB001C0CF0FF0CCDF804C003EB5C
:10BC3000021C0CF0FF0CCDF800C0DDF804C084F845
:10BC400001C0DDF800C084F800C000BF701C06B25F
:10BC500056457FF754AD681C05B245457FF74DAD9D
:10BC600000BF00BF58E40000D8130020DC13002000
:10BC7000EA130020EB1300202DE9FF4F2DED028B7E
:10BC80008BB083460F46144694F8009094F801A0B8
:10BC9000E178A07801EB002080B2089061792079EA
:10BCA00001EB002080B20790E179A07901EB002040
:10BCB00080B20690617A207A01EB002080B2059074
:10BCC0000A25002002903EE00EF0ECF9029805EB08
:10BCD000400014F80080029805EB4000401C265CF0
:10BCE000F21911B208EB0B0210B2109AF7F7E2F852
:10BCF000B9F1000F0AD0C8EB4900401E584400B209
:10BD000004903146109A0498F7F7D4F8BAF1000F6E
:10BD10000AD0C6EB4A00401E384400B203904046A9
:10BD2000109A0399F7F7C6F8B9F1000F07D0BAF1E6
:10BD3000000F04D0109ADDE90310F7F7BBF8029862
:10BD4000401C80B20290089902988842BCDB022114
:10BD5000089801FB005085B2002002905CE00EF0D4
:10BD6000A1F9029800EB4000284414F800800298E2
:10BD700000EB40002844401C265C029800EB400089
:10BD80002844801C205C0A909DED0A0AB8EE400B06
:10BD9000B0EE408B9FED960B88EE001BB0EE418B12
:10BDA000F21911B208EB0B0210B2B0EE480B109A68
:10BDB000F7F78CF8B9F1000F0DD0C8EB4900401E21
:10BDC000584400B20490F01901B2B0EE480B109A3A
:10BDD0000498F7F77BF8BAF1000F0CD0C6EB4A00D5
:10BDE000401E384400B20390B0EE480B4046109A13
:10BDF0000399F7F76BF8B9F1000F09D0BAF1000F0A
:10BE000006D0B0EE480B109ADDE90310F7F75EF8A4
:10BE10000298401C80B202900799029888429EDBEB
:10BE2000079800EB4000284485B20020029059E0BA
:10BE30000EF038F9029800EB4000284414F8008016
:10BE4000029800EB40002844401C265C029800EB5E
:10BE500040002844801C205C09900020019039E0BB
:10BE6000F21911B2019A42445A4410B2109AF7F7EB
:10BE700021F8B9F1000F0DD0C8EB4900401E01991F
:10BE8000401A584400B20490F01901B2109A049874
:10BE9000F7F710F8BAF1000F0DD0C6EB4A00401EBC
:10BEA000384400B2039001994144594408B2109AB1
:10BEB0000399F6F7FFFFB9F1000F07D0BAF1000FB1
:10BEC00004D0109ADDE90310F6F7F4FF0198401C46
:10BED00080B20190099901988842C1DB0298401C08
:10BEE00080B20290069902988842A1DB069800EB86
:10BEF0004000284485B20020029070E00EF0D2F895
:10BF0000029805EB800014F80080029805EB800091
:10BF1000401C265C029805EB8000801C205C0A9087
:10BF20009DED0A0AB8EE400BB0EE408B9FED300B52
:10BF300088EE001BB0EE418B029805EB8000C01C20
:10BF4000205C09900020019041E0F21911B2019AA1
:10BF500042445A4410B2B0EE480B109AF6F7B6FFBE
:10BF6000B9F1000F0FD0C8EB4900401E0199401AEB
:10BF7000584400B20490F01901B2B0EE480B109A88
:10BF80000498F6F7A3FFBAF1000F0FD0C6EB4A00F2
:10BF9000401E384400B2039001994144594408B20C
:10BFA000B0EE480B109A0399F6F790FFB9F1000F25
:10BFB00009D0BAF1000F06D0B0EE480B109ADDE9B7
:10BFC0000310F6F783FF0198401C80B20190099995
:10BFD00001988842B9DB0298401C80B20290059912
:10BFE000029888428ADB0BB0BDEC028BBDE8FF8F64
:10BFF0000000000000E06F402DE9FF4104460D46BF
:10C0000016461F46102C71D2DFE804F008101820E5
:10C01000283038404850586068717981684601F08E
:10C0200063FDDDE90001CDE902017AE0684601F037
:10C0300067FDDDE90001CDE9020172E0684601F02B
:10C040006BFDDDE90001CDE902016AE0684601F01F
:10C050006FFDDDE90001CDE9020162E0684601F013
:10C0600073FDDDE90001CDE902015AE0684601F007
:10C0700077FDDDE90001CDE9020152E0684601F0FB
:10C080007BFDDDE90001CDE902014AE0684601F0EF
:10C090007FFDDDE90001CDE9020142E0684601F0E3
:10C0A00083FDDDE90001CDE902013AE0684601F0D7
:10C0B00087FDDDE90001CDE9020132E0684601F0CB
:10C0C0008BFDDDE90001CDE902012AE0684601F0BF
:10C0D0008FFDDDE90001CDE9020122E0684601F0B3
:10C0E00093FDDDE90001CDE902011AE017E06846A1
:10C0F00001F096FDDDE90001CDE9020111E068469D
:10C1000001F09AFDDDE90001CDE9020109E0684690
:10C1100001F09EFDDDE90001CDE9020101E0BDE88D
:10C12000FF8100BF9DF90D00304401B23B46284617
:10C13000029AFFF7A1FD00BFF1E72DE9FC47064693
:10C140000C46174698463046F4F7A2F81FFA80F9D5
:10C15000002513E0715D684601F0EAFB9DF90500DA
:10C16000384401B243462046009AFFF785FD9DF80A
:10C170000400401C204404B2681C85B24D45E9DB34
:10C18000BDE8FC872DE9FC4705460C4690469A46DB
:10C1900000262846F4F77CF81FFA80F9002709E00A
:10C1A000E95D684601F0C4FB9DF80400304486B2A6
:10C1B000781C87B24F45F3DB304606EBD071A4EB19
:10C1C00061010CB2002713E0E95D684601F0B0FBA5
:10C1D0009DF90500404401B253462046009AFFF7FE
:10C1E0004BFD9DF80400401C204404B2781C87B22B
:10C1F0004F45E9DBBDE8FC872DE9FF4F87B00546D9
:10C200000C469046DDE914AB00262846F4F740F8CA
:10C210001FFA80F9002709E0E95D05A801F088FB15
:10C220009DF81800304486B2781C87B24F45F3DB86
:10C23000304606EBD071A4EB61010CB2002719E087
:10C24000E95D05A801F074FBDDE91610CDE900AB4E
:10C25000CDE902109DF91900404401B220460A9B25
:10C26000059A00F00DF89DF81800401C204404B217
:10C27000781C87B24F45E3DB0BB0BDE8F08F0000C0
:10C280002DE9FF4F2DED028B8BB080460E461446F4
:10C2900094F800A094F801B0E178A07801EB0020B8
:10C2A00080B208906179207901EB002080B207907C
:10C2B000E179A07901EB002080B20690617A207AC2
:10C2C00001EB002080B205904FF00A090020029097
:10C2D0004FE00DF0E7FE029809EB4000275C029862
:10C2E00009EB4000401C255C07EB08011A988142CD
:10C2F0003BDB07EB08011C98814236DCA9191B982F
:10C30000814232DBA9191D9881422EDCAA1911B293
:10C3100007EB080210B2109AF6F7CCFDBAF1000F45
:10C320000AD0C7EB4A00401E404400B204902946A0
:10C33000109A0498F6F7BEFDBBF1000F0AD0C5EBCA
:10C340004B00401E304400B203903846109A0399C7
:10C35000F6F7B0FDBAF1000F07D0BBF1000F04D023
:10C36000109ADDE90310F6F7A5FD0298401C80B293
:10C370000290089902988842ABDB0221089801FBE1
:10C3800000901FFA80F9002002906DE00DF08AFE07
:10C39000029800EB40004844275C029800EB400004
:10C3A0004844401C255C029800EB40004844801C37
:10C3B000205C0A909DED0A0AB8EE400BB0EE408B6F
:10C3C0009FEDB20B88EE001BB0EE418B07EB08012E
:10C3D0001A98814244DB07EB08011C9881423FDC3C
:10C3E000A9191B9881423BDBA9191D98814237DCB2
:10C3F000AA1911B207EB080210B2B0EE480B109A5E
:10C40000F6F764FDBAF1000F0DD0C7EB4A00401EED
:10C41000404400B20490A81901B2B0EE480B109A43
:10C420000498F6F753FDBBF1000F0CD0C5EB4B00A1
:10C43000401E304400B20390B0EE480B3846109ACC
:10C440000399F6F743FDBAF1000F09D0BBF1000FD5
:10C4500006D0B0EE480B109ADDE90310F6F736FD72
:10C460000298401C80B202900799029888428DDBA6
:10C47000079800EB400048441FFA80F90020029022
:10C480006AE00DF00FFE029800EB40004844275C84
:10C49000029800EB40004844401C255C029800EBE9
:10C4A00040004844801C205C0990002001904BE033
:10C4B00007EB08011A98814242DB07EB08011C9840
:10C4C00081423DDCA9191B98814239DBA9191D98CD
:10C4D000814235DCAA1911B2019A3A44424410B2A1
:10C4E000109AF6F7E7FCBAF1000F0DD0C7EB4A003F
:10C4F000401E0199401A404400B20490A81901B2AC
:10C50000109A0498F6F7D6FCBBF1000F0DD0C5EBDE
:10C510004B00401E304400B203900199394441441D
:10C5200008B2109A0399F6F7C5FCBAF1000F07D0CC
:10C53000BBF1000F04D0109ADDE90310F6F7BAFC46
:10C540000198401C80B20190099901988842AFDBA4
:10C550000298401C80B2029006990298884290DBB3
:10C56000069800EB400048441FFA80F90020029032
:10C5700081E00DF097FD029809EB8000275C02989E
:10C5800009EB8000401C255C029809EB8000801CB0
:10C59000205C0A909DED0A0AB8EE400BB0EE408B8D
:10C5A0009FED3A0B88EE001BB0EE418B029809EB31
:10C5B0008000C01C205C09900020019053E007EB34
:10C5C00008011A9881424ADB07EB08011C98814256
:10C5D00045DCA9191B98814241DBA9191D988142AC
:10C5E0003DDCAA1911B2019A3A44424410B2B0EEAD
:10C5F000480B109AF6F76AFCBAF1000F0FD0C7EBA0
:10C600004A00401E0199401A404400B20490A81903
:10C6100001B2B0EE480B109A0498F6F757FCBBF144
:10C62000000F0FD0C5EB4B00401E304400B203900A
:10C6300001993944414408B2B0EE480B109A03996D
:10C64000F6F744FCBAF1000F09D0BBF1000F06D099
:10C65000B0EE480B109ADDE90310F6F737FC0198AD
:10C66000401C80B20190099901988842A7DB02988A
:10C67000401C80B20290059902988842FFF679AF7B
:10C680000BB0BDEC028BBDE8FF8F00000000000086
:10C6900000E06F402DE9F04F8BB082468B46144688
:10C6A00094F8008094F80190E178A07801EB0020E4
:10C6B00080B209906179207901EB002080B2089066
:10C6C000E179A07901EB002080B20790617A207AAD
:10C6D00001EB002080B206900A270020039052E070
:10C6E0000DF0E0FC039807EB4000255C039807EB96
:10C6F0004000401C265C0020009006EB0B0291B22B
:10C7000005EB0A02019090B200231A4600F0F8FBF4
:10C71000B8F1000F0FD0C5EB4800401E504402B2E4
:10C72000059200200090B1B20190059A90B20023CA
:10C730001A4600F0E5FBB9F1000F0FD0C6EB490037
:10C74000401E584402B20492002000900190049AC6
:10C7500091B2A8B200231A4600F0D2FBB8F1000F44
:10C760000DD0B9F1000F0AD0002000900190049A7A
:10C7700091B2059A90B200231A4600F0C1FB0398CB
:10C78000401C80B20390099903988842A8DB0221DB
:10C79000099801FB007087B20020039054E00DF06F
:10C7A00081FC039800EB40003844255C039800EBC3
:10C7B00040003844401C265C0020009006EB0B0231
:10C7C00091B205EB0A02019090B200231A4600F0E4
:10C7D00097FBB8F1000F0FD0C5EB4800401E504446
:10C7E00000B2059000200090B1B20190059A90B27D
:10C7F00000231A4600F084FBB9F1000F0FD0C6EBFE
:10C800004900401E584400B204900020009001905E
:10C81000049A91B2A8B200231A4600F071FBB8F155
:10C82000000F0DD0B9F1000F0AD000200090019048
:10C83000049A91B2059A90B200231A4600F060FB68
:10C840000398401C80B20390089903988842A6DBA5
:10C85000089800EB4000384487B2002003906EE057
:10C860000DF020FC039800EB40003844255C039851
:10C8700000EB40003844401C265C039800EB40006D
:10C880003844801C205C0A90002002904FE0002079
:10C89000009006EB0B0291B20190029A2A44524496
:10C8A00090B200231A4600F02BFBB8F1000F13D012
:10C8B000C5EB4800401E0299401A504400B2059052
:10C8C0000020009006EB0B0291B20190059A90B205
:10C8D00000231A4600F014FBB9F1000F12D0C6EB8A
:10C8E0004900401E584400B204900020009001907E
:10C8F000049A91B2029A2A44524490B200231A46F2
:10C9000000F0FEFAB8F1000F0DD0B9F1000F0AD017
:10C91000002000900190049A91B2059A90B20023F1
:10C920001A4600F0EDFA0298401C80B202900A9973
:10C9300002988842ABDB0398401C80B203900799B1
:10C94000039888428CDB079800EB4000384487B29C
:10C95000002003906BE00DF0A5FB039807EB80002F
:10C96000255C039807EB8000401C265C039807EBCE
:10C970008000C01C205C0A90002002904FE0002044
:10C98000009006EB0B0291B20190029A2A445244A5
:10C9900090B200231A4600F0B3FAB8F1000F13D09A
:10C9A000C5EB4800401E0299401A504400B2059061
:10C9B0000020009006EB0B0291B20190059A90B214
:10C9C00000231A4600F09CFAB9F1000F12D0C6EB12
:10C9D0004900401E584400B204900020009001908D
:10C9E000049A91B2029A2A44524490B200231A4601
:10C9F00000F086FAB8F1000F0DD0B9F1000F0AD09F
:10CA0000002000900190049A91B2059A90B2002300
:10CA10001A4600F075FA0298401C80B202900A99FA
:10CA200002988842ABDB0398401C80B203900699C1
:10CA3000039888428FDB0BB0BDE8F08F2DE9FF4FE4
:10CA400082B00E46174698460025C8F100047800CB
:10CA5000C0F10209DFED361AB0EE610ADFED341ADB
:10CA6000F0EE610ADFED321AB0EE611A01EE907A53
:10CA7000F8EE611AF0EE610A01EE908AF8EE611AA2
:10CA8000B0EE611AC1EE201AB0EE610A00BF01EEED
:10CA9000905AF8EEE11A81EE802AFCEEC21A11EEED
:10CAA000900A4000401C80B2019001EE905AF8EECE
:10CAB000E11A81EE802AFCEEC21A11EE900A029968
:10CAC000081A1FFA80FB01985844401E80B200905B
:10CAD000301903B2301901B2009802B20FFA8BF08C
:10CAE000FEF76CF8301B03B2301B01B2009802B2A3
:10CAF0000FFA8BF0FEF762F8CA46AA450BDC681CF9
:10CB00000546012101EB40008144EC4203D1A245DE
:10CB100001DC4FF0000AA24505DD601C044601213E
:10CB200001EB40008144002CB1DD06B0BDE8F08F80
:10CB3000000000002DE9F04F04460D4616461F4642
:10CB40002148007808B9BDE8F08FA019401E1FFAEF
:10CB500080FAE819401E1FFA80FB1C4800688245D5
:10CB600004D31A480088401E1FFA80FA184800684B
:10CB7000834504D316480088401E1FFA80FB06B97F
:10CB8000E1E707B9DFE711480068844200D3DAE73C
:10CB90000F480068854200D3D5E7A8460FE0A146BC
:10CBA00007E04146484600F007F909F101001FFA85
:10CBB00080F9D145F5DD08F101001FFA80F8D8456C
:10CBC000EDDD00BF00BFBEE7D4130020DC13002062
:10CBD000E01300202DE9F0431148007808B9BDE8C2
:10CBE000F083002600270F480088401E1FFA80F8B7
:10CBF0000D480088401E1FFA80F93C460BE0354680
:10CC000005E02146284600F0D7F8681C85B2454566
:10CC1000F7DD601C84B24C45F1DD00BF00BFDEE7EC
:10CC2000D4130020DC130020E013002070B503466D
:10CC30000C462C480078002852D02B4800688342CC
:10CC40004ED22A48006884424AD22948008890B9C6
:10CC50002848016824480068800000FB041101EBAB
:10CC60008301C87810708878507048789070087880
:10CC7000D070012070BD1E480088012814D11D48C5
:10CC800001681948006800EB400000FB041103EB49
:10CC900043000144FF2010708878507048789070ED
:10CCA0000878D0700120E5E711480088042816D1E3
:10CCB000104801680C480068400000FB041101EBBB
:10CCC00043014D780E782809107005F00F00507060
:10CCD0003009907006F00F00D0700120CAE700BF45
:10CCE0000020C7E7D4130020DC130020E01300204D
:10CCF000E4130020D81300200148008880B2704758
:10CD0000E01300200148008880B27047DC13002047
:10CD10000149086070470000EC13002030B50A4C50
:10CD200020700A4C21700A4C22700A4C237000F0CB
:10CD3000F00404EB2114084D2C7002F0F00404EB15
:10CD40002314064D2C7030BDE6130020E71300209D
:10CD5000E8130020E9130020EA130020EB13002061
:10CD600010B586B0044600200E490870214668467A
:10CD7000F5F786FA009808B1012000E00020094983
:10CD80000870094900980860BDF808000749086064
:10CD9000BDF80A000649086006490398088006B0F5
:10CDA00010BD0000D4130020D8130020DC13002095
:10CDB000E0130020E41300200A462B49097801B94A
:10CDC00070472A490968884200D3F9E72849096869
:10CDD0008A4200D3F4E727490988A9B9264B196884
:10CDE000224B1B689B0003FB021101EB8001234BCC
:10CDF0001B78CB70224B1B788B70224B1B784B70AF
:10CE0000214B1B780B702CE01A490988012914D199
:10CE1000194B1968154B1B6803EB430303FB021105
:10CE200000EB40031944164B1B788B70154B1B7895
:10CE30004B70154B1B780B7013E00E4909880429C1
:10CE40000FD10D4B1968094B1B685B0003FB0211E6
:10CE500001EB40010D4B1B784B700D4B1B780B7099
:10CE600000BF00BFACE70000D4130020DC1300209B
:10CE7000E0130020E4130020D8130020E613002064
:10CE8000E7130020E8130020E9130020EA13002034
:10CE9000EB13002000B5B5EEC01BF1EE10FA09DB74
:10CEA000B6EE002B31EE022BBDEEC22B12EE102A95
:10CEB00012B208E0B6EE002B31EE422BBDEEC22BD3
:10CEC00012EE102A12B291B2B5EEC00BF1EE10FACA
:10CED00009DBB6EE002B30EE022BBDEEC22B12EEBC
:10CEE000102A12B208E0B6EE002B30EE422BBDEE57
:10CEF000C22B12EE102A12B290B2FFF75DFF00BDF6
:10CF0000F0B50C46DDE905562549097801B9F0BDB3
:10CF100024490968884200D3F9E7234909688C420B
:10CF200000D3F4E72149098869B9214F39681D4FB9
:10CF30003F68BF0007FB041101EB8001CA708B70D2
:10CF40004D700E702AE01949098801290ED1184F39
:10CF50003968144F3F6807EB470707FB041100EBE4
:10CF6000400739448B704D700E7017E00F490988E7
:10CF7000042913D10E4F39680A4F3F687F0007FB21
:10CF8000041101EB400102F0F00707EB23174F708B
:10CF900005F0F00707EB26170F7000BF00BFB6E7DC
:10CFA000D4130020DC130020E0130020E413002041
:10CFB000D81300202DE9F0470D46DDE9087C0A9CD6
:10CFC000012600219CE006EA0508B8F1000F75D0A3
:10CFD000D0F800804FEA410A4FF0030909FA0AF934
:10CFE00028EA0908C0F8008002F003084FEA410966
:10CFF00008FA09F8D0F8009048EA0908C0F800805B
:10D00000D0F804804FF0010909FA01F928EA09086B
:10D01000C0F8048003F0010808FA01F8D0F8049081
:10D0200048EA0908C0F80480D0F808804FEA410AAD
:10D030004FF0030909FA0AF928EA0908C0F808803C
:10D0400007F003084FEA410908FA09F8D0F80890F8
:10D0500048EA0908C0F80880D0F80C804FEA410A75
:10D060004FF0030909FA0AF928EA0908C0F80C8008
:10D070000CF003084FEA410908FA09F8D0F80C90BF
:10D0800048EA0908C0F80C80082918DAD0F820808E
:10D090004FEA810A4FF00F0909FA0AF928EA09084C
:10D0A000C0F8208004F00F084FEA810908FA09F857
:10D0B000D0F8209048EA0908C0F820801BE0D0F89A
:10D0C0002480A1F108094FEA890A4FF00F0909FAF3
:10D0D0000AF928EA0908C0F8248004F00F08A1F131
:10D0E00008094FEA890908FA09F8D0F8249048EAB3
:10D0F0000908C0F82480760001F1010808F0FF015A
:10D100001029FFF660AFBDE8F08700002DE9F34F6E
:10D110002DED048BA1B025980F90BDF89800ADF8C7
:10D120004000FE48006813F0CFF90E90FC480078EC
:10D130008DF84200FB480088ADF844004FF0FF3006
:10D14000ADF84600ADF84800ADF84A000020139055
:10D15000401EADF8500000201590401EADF858005C
:10D160009FEDF10B8DED180BADF858009FEDEE0B18
:10D170008DED1C0BADF878009DF89800002837D095
:10D18000E748007838B90020E9490880E549088077
:10D19000E84813F0D1F9E748006813F095F9E6493B
:10D1A000E34A128841F83200BDF89400E04A128840
:10D1B00001EBC2018880BDF89600DF49DC4A128885
:10D1C00001EBC201C880DA480088401CD8490880B9
:10D1D000084600880A2801DB00200880D148008822
:10D1E0000A2804DACF480088401CCE4908808EE126
:10D1F00000200D90CB480088042874DB0120ADF896
:10D200004800CB48008804B2002007900120059018
:10D2100000207DE0059921B101B2ADF84610002152
:10D220000591611E0CB2002C00DA092498B9C2499C
:10D2300001EBC401B1F80490BF4951F834100991D1
:10D24000BD4901EBC401C9880C91BB4901EBC40184
:10D25000C9880B9156E0B84901EBC401CA880C9902
:10D260008A4204DDB44901EBC401C9880C91B2497A
:10D2700001EBC401CA880B998A4204DAAE4901EB7A
:10D28000C401C9880B91AC4901EBC401B1F8048019
:10D29000A94901EBC401C9880A91A74951F8341082
:10D2A0000891012814D1A44901EBC4018988B9422D
:10D2B00002DD0121069125E09F4901EBC401898827
:10D2C000B94202DA002106911CE00121079122E017
:10D2D000994901EBC4018988B94205DD069989B9EC
:10D2E0000121079117E0C4E0934901EBC40189884B
:10D2F000B94204DA069929B1012107910BE0012115
:10D30000079108E08C4901EBC4018F88411C88B269
:10D310000428FFF67FAF00BF079800287ED10120C8
:10D32000ADF84A00DDE90810461A1396002E76DDA6
:10D3300040F6C410864272DA0120ADF85000A8EB26
:10D34000090005B2002D01DA684205B20020ADF8EF
:10D3500050000A2D72DD0120ADF85800DDE90B10F8
:10D36000401A0FFA80FA00EE10AAB8EEC00B8DED4D
:10D37000180B554558DD0120ADF8680000EE105A35
:10D38000B8EEC00BB0EE408B00EE106AB8EEC00BEA
:10D3900088EE001BB0EE418B8DED1C8B9FED670B73
:10D3A000B4EEC08BF1EE10FA25DDADF87800C8457B
:10D3B00003DDB1EE480BB0EE408B02208DF800008B
:10D3C000ADF802800A98ADF804008DED028B9FED58
:10D3D0005D0B28EE009BBDEEC90B10EE10BA5A464D
:10D3E0000121072005F024FA01200D909DE80F008F
:10D3F000F6F738FA17E00020ADF878004FF47A7BA2
:10D4000000EE10BAB8EEC00B20EE080BBDEEC00B5C
:10D4100010EE10BA5A460221072001E020E016E083
:10D4200005F006FA00BF07E00020ADF86800002212
:10D430000621072005F0FCF908E0FFE70020ADF821
:10D4400058002A460321072005F0F2F907E00020E2
:10D45000ADF8500032460421072005F0E9F907E055
:10D460000020ADF84A0000220521072005F0E0F970
:10D4700002E00020ADF848000D98E0BB2948008884
:10D48000002843DD274800880A283FDA284800881A
:10D4900000283BDD284903C9CDE90B012448008859
:10D4A000401E254901EBC00103C9CDE90901BDF8C2
:10D4B0002800BDF83010401A04B2BDF82A00BDF8AB
:10D4C0003210401A05B2002C01DA604204B2002D7D
:10D4D00001DA684205B20A2C17DA0A2D15DA0120A2
:10D4E0008DF8100014488088ADF812001248C088EA
:10D4F000ADF8140000E009E09FED0B0B8DED060B7D
:10D5000004A80FC8F6F7AEF900BF00BF00BF9DF832
:10D510009800034908700D48007819E0C8130020EE
:10D52000BC130020B8130020000000000000000021
:10D53000BA130020C0130020D0060120B81E85EBCE
:10D5400051B89E3F0000000000408F40CC130020E7
:10D55000F0B91249098801EBC101114A02EBC1007F
:10D5600048220EA9F2F764FE0C480088401C0B49C3
:10D57000088008460088642801DB002008800948EC
:10D580000088642804DA07480088401C05490880A0
:10D5900021B0BDEC048BBDE8FC8F0000C41300205B
:10D5A00020070120C613002010B5024812F0C4FF66
:10D5B00010BD0000C813002010B503211DA01CF0F1
:10D5C00063FF1D48008800B21CF08CFF05211BA0E2
:10D5D0001CF05AFF1B48008800B21CF083FF5D203E
:10D5E0001CF03CFF002421E05B201CF037FF1649B3
:10D5F00031F8341008B21CF075FF2C201CF02EFFFF
:10D60000114901EBC401898808B21CF06BFF2C2082
:10D610001CF024FF0C4901EBC401C98808B21CF0BE
:10D6200061FF5D201CF01AFF601C84B20A2CDBDB5A
:10D6300010BD00005B633D00B81300202C696478C6
:10D640003D000000BA130020D00601200146094821
:10D65000007803280BDA0848064A127840F82210AE
:10D6600004480078401C034A1070012070470020D5
:10D67000FCE70000CD1300204023012000200349D7
:10D68000088003490880012070470000C61300206D
:10D69000C413002010B51548007828BB1448008832
:10D6A00000B2144908801248008800B2124908806C
:10D6B0000F480088642805DB1048008800B2104934
:10D6C000088002E000200E49088001200749087008
:10D6D0000948B0F900200BA10F4825F031FD0E4894
:10D6E0001DF002F8012010BD0020FCE7CC13002043
:10D6F000C6130020D0130020D2130020C413002032
:10D70000CE1300205B4C6F6744756D70537461726B
:10D7100074696E6725645D004C23012010B50648CE
:10D72000007838B100200449087004A01CF0DCFF28
:10D73000012010BD0020FCE7CC1300205B4C6F677C
:10D7400044756D70436F6D706C6574655D000000AD
:10D7500000B5A9B03848007800286AD03748B0F939
:10D760000000002802DCFFF7D9FF62E03448B0F97E
:10D77000000000EBC000334A02EBC001482216A8AB
:10D78000F2F756FDBDF9980014909DED240B8DED38
:10D79000120BBDF9880010909DED200B8DED0E0B46
:10D7A000BDF97800BDF970201B9B1D99CDE90932A8
:10D7B000CDE90B10BDF96A00BDF96810BDF966200E
:10D7C000BDF86430CDE90532CDE907109DF862005F
:10D7D00016A9CA88BDF85C1016AB1B7ACDE90131D9
:10D7E000CDE90320169800901748B0F900001349BE
:10D7F000B1F90010421A1448B0F900301349144826
:10D8000025F09EFC12481CF06FFF0D480088401C5C
:10D8100000B20B4908800846B0F90000642801DB1B
:10D820000020088005480088401E00B20349088097
:10D8300000BF29B000BD0000CC130020D21300208F
:10D84000CE13002020070120D013002060C40D0853
:10D850004C23012010B5FFF77BFF10BDC32070479C
:10D86000F0B5ADF5017D06460C461546ADF8F8411C
:10D870002046E11704EB9161C1F38F11ADF8FA1165
:10D880002046E11704EB91618911A4EB811189B263
:10D89000ADF8FC110020ADF8FE01BDF8FA017C9056
:10D8A0001548006800F5C06000EB452000F110014C
:10D8B0004FF4F8726846F2F7BBFC0F48006800F5B9
:10D8C000C06000EB452797E80F00F3F7B7FA10B1F7
:10D8D0000120ADF8FE01BDF8FE01C0F1010080B2EB
:10D8E000ADF800027E9830607F987060BDF800024D
:10D8F00030810DF5017DF0BD9814002008B50B486E
:10D90000006890F8000430B100208DF8000001207C
:10D910008DF8010005E001208DF8000000208DF851
:10D920000100BDF80010084608BD00009814002052
:10D930003CB504460D46A5F120003B286FD2DFE838
:10D9400000F0BBC7C7C7C7C3C7C7C7C7C7C7B7C725
:10D95000AFB31E22262A2E32363A3E42BFC7C7C771
:10D96000C7C7C7464A4E52565A5E62666A6F737799
:10D970007B7F83878B8F93979B9FA3A7AB002046CA
:10D9800000F0B2F83CBD204600F0BAF8FAE72046B5
:10D9900000F0C2F8F6E7204600F0CAF8F2E72046A9
:10D9A00000F0D2F8EEE7204600F0DAF8EAE7204689
:10D9B00000F0E2F8E6E7204600F0EAF8E2E7204669
:10D9C00000F0F2F8DEE7204600F0FAF8DAE7204649
:10D9D00000F002F9D6E7204600F00AF9D2E7204627
:10D9E00000F012F9CEE7204600F01AF9CAE7204607
:10D9F00000F022F9C6E7204600F02AF9C2E72046E7
:10DA000000F032F9BEE7204600F03AF9BAE72046C6
:10DA100000F042F9B6E7204600F04AF9B2E757E0D5
:10DA2000204600F051F9ADE7204600F059F9A9E78A
:10DA3000204600F061F9A5E7204600F069F9A1E76A
:10DA4000204600F071F99DE7204600F079F999E74A
:10DA5000204600F081F995E7204600F089F991E72A
:10DA6000204600F091F98DE7204600F099F989E70A
:10DA7000204600F0A1F985E7204600F0A9F981E7EA
:10DA8000204600F0B1F97DE7204600F0B9F979E7CA
:10DA9000204600F0C1F975E7204600F0C9F971E7AA
:10DAA000204600F001FA6DE7204600F0E5F969E74D
:10DAB000204600F0D5F965E7204600F001FA61E75D
:10DAC000204600F0C1F95DE7204600F0E1F959E792
:10DAD000044903C9CDE90001DDE90001C4E9000101
:10DAE00000BF4FE750C20D080CB5044A06CACDE985
:10DAF0000012DDE90012C0E900120CBD08C10D08DA
:10DB00000CB5044A06CACDE90012DDE90012C0E9ED
:10DB100000120CBD10C10D080CB5044A06CACDE9AF
:10DB20000012DDE90012C0E900120CBD18C10D0899
:10DB30000CB5044A06CACDE90012DDE90012C0E9BD
:10DB400000120CBD20C10D080CB5044A06CACDE96F
:10DB50000012DDE90012C0E900120CBD28C10D0859
:10DB60000CB5044A06CACDE90012DDE90012C0E98D
:10DB700000120CBD30C10D080CB5044A06CACDE92F
:10DB80000012DDE90012C0E900120CBD38C10D0819
:10DB90000CB5044A06CACDE90012DDE90012C0E95D
:10DBA00000120CBD40C10D080CB5044A06CACDE9EF
:10DBB0000012DDE90012C0E900120CBD48C10D08D9
:10DBC0000CB5044A06CACDE90012DDE90012C0E92D
:10DBD00000120CBD50C10D080CB5044A06CACDE9AF
:10DBE0000012DDE90012C0E900120CBD58C10D0899
:10DBF0000CB5044A06CACDE90012DDE90012C0E9FD
:10DC000000120CBD60C10D080CB5044A06CACDE96E
:10DC10000012DDE90012C0E900120CBD68C10D0858
:10DC20000CB5044A06CACDE90012DDE90012C0E9CC
:10DC300000120CBD70C10D080CB5044A06CACDE92E
:10DC40000012DDE90012C0E900120CBD78C10D0818
:10DC50000CB5044A06CACDE90012DDE90012C0E99C
:10DC600000120CBD80C10D080CB5044A06CACDE9EE
:10DC70000012DDE90012C0E900120CBD88C10D08D8
:10DC80000CB5044A06CACDE90012DDE90012C0E96C
:10DC900000120CBD90C10D080CB5044A06CACDE9AE
:10DCA0000012DDE90012C0E900120CBD98C10D0898
:10DCB0000CB5044A06CACDE90012DDE90012C0E93C
:10DCC00000120CBDA0C10D080CB5044A06CACDE96E
:10DCD0000012DDE90012C0E900120CBDA8C10D0858
:10DCE0000CB5044A06CACDE90012DDE90012C0E90C
:10DCF00000120CBDB0C10D080CB5044A06CACDE92E
:10DD00000012DDE90012C0E900120CBDB8C10D0817
:10DD10000CB5044A06CACDE90012DDE90012C0E9DB
:10DD200000120CBDC0C10D080CB5044A06CACDE9ED
:10DD30000012DDE90012C0E900120CBDC8C10D08D7
:10DD40000CB5044A06CACDE90012DDE90012C0E9AB
:10DD500000120CBDD0C10D080CB5044A06CACDE9AD
:10DD60000012DDE90012C0E900120CBDD8C10D0897
:10DD70000CB5044A06CACDE90012DDE90012C0E97B
:10DD800000120CBDE0C10D080CB5044A06CACDE96D
:10DD90000012DDE90012C0E900120CBDE8C10D0857
:10DDA0000CB5044A06CACDE90012DDE90012C0E94B
:10DDB00000120CBDF0C10D080CB5044A06CACDE92D
:10DDC0000012DDE90012C0E900120CBDF8C10D0817
:10DDD0000CB5044A06CACDE90012DDE90012C0E91B
:10DDE00000120CBD00C20D080CB5044A06CACDE9EC
:10DDF0000012DDE90012C0E900120CBD08C20D08D6
:10DE00000CB5044A06CACDE90012DDE90012C0E9EA
:10DE100000120CBD10C20D080CB5044A06CACDE9AB
:10DE20000012DDE90012C0E900120CBD18C20D0895
:10DE30000CB5044A06CACDE90012DDE90012C0E9BA
:10DE400000120CBD20C20D080CB5044A06CACDE96B
:10DE50000012DDE90012C0E900120CBD40C20D083D
:10DE60000CB5044A06CACDE90012DDE90012C0E98A
:10DE700000120CBD38C20D080CB5044A06CACDE923
:10DE80000012DDE90012C0E900120CBD30C20D081D
:10DE90000CB5044A06CACDE90012DDE90012C0E95A
:10DEA00000120CBD48C20D080CB5044A06CACDE9E3
:10DEB0000012DDE90012C0E900120CBD28C20D08F5
:10DEC000024A06CAC0E9001270470000881C002000
:10DED000004870479FF00C08004870477B870D088A
:10DEE0000048704706090D08004870475A020D089F
:10DEF00000487047CA0F0D08004870471A790D088E
:10DF000000487047E5FA0C080048704795720D0804
:10DF100000487047FA750D0800487047A35E0D0869
:10DF200000487047FF5F0D080048704748610D08C2
:10DF300000487047D7620D0800487047A3650D0878
:10DF400000487047A7660D0800487047463D0D0819
:10DF500000487047F3180D080048704705690D0820
:10DF60000048704784410D0800487047447D0D0803
:10DF700000487047FAE60C08004870473BEA0C0876
:10DF80000048704799460D0800487047DC460D0868
:10DF900000487047DDD90C080048704747DA0C0884
:10DFA0000048704787DA0C0800487047D3DA0C083D
:10DFB0000048704725DB0C080048704774DB0C08EC
:10DFC00000487047C3DB0C08004870471DDC0C0894
:10DFD000004870475DDC0C0800487047BEDC0C0848
:10DFE000004870475ED90C0800487047C5D90C0836
:10DFF00000487047FB000D080048704770F20C089D
:10E000000048704753E90C08004870478B1C0D0806
:10E0100000487047B9200D080048704762240D0879
:10E020000048704729270D080048704770290D08DF
:10E0300000487047D12A0D0800487047AC2C0D08E5
:10E0400000487047222F0D08004870474E320D08D7
:10E05000004870475D360D0800487047786C0D0821
:10E06000F0B5ADF5037D05460E4614462246314611
:10E0700080A8FFF7F5FB0027BDF802027C901A4844
:10E08000006800F5C06000EB442000F110014FF47F
:10E09000F8726846F2F7CCF81348006800F5C060E3
:10E0A00000EB442C9CE80F00F2F7C8FE00B10127FA
:10E0B00040F2D51078430C49096801F5206101EB65
:10E0C0008020BDF8021200EB4120BDF8041200EBE5
:10E0D000C10001687E9140687F907E9828607F989B
:10E0E00068600DF5037DF0BD9814002018B5024658
:10E0F0000020009000BF92F83C00012801D10220CE
:10E1000018BD012082F83C0000BF0868092822D908
:10E110001068C0680B780A3B03EB43040723A34055
:10E1200098431368D8604F4B0868984207D110682D
:10E13000C0680B7A40EA03601368D8601FE00B7870
:10E140000A3B03EB4303886898401368DB68184375
:10E150001368D86013E0106800690B7803EB430480
:10E160000723A3409843136818610B7803EB43031C
:10E170008868984013681B691843136818614868D9
:10E18000072817D21068406B0B795B1E03EB8304E2
:10E190001F23A340984313685863088880B20B7903
:10E1A0005B1E03EB8303984013685B6B1843136893
:10E1B000586331E048680D2817D21068006B0B795E
:10E1C000DB1F03EB83041F23A340984313681863EA
:10E1D000088880B20B79DB1F03EB83039840136838
:10E1E0001B6B18431368186316E01068C06A0B793C
:10E1F0000D3B03EB83041F23A34098431368D862AD
:10E20000088880B20B790D3B03EB830398401368B9
:10E21000DB6A18431368D862134B1068984208D120
:10E220000868122805D11148006840F48000C3F83E
:10E2300004030D4B106898420DD10A4B08689842B0
:10E2400002D00868112806D10848006840F4000090
:10E25000054BC3F8040300BF002082F83C0000BF58
:10E2600000BF4DE7120000100020014004230140D0
:10E270002DE9FE4F04460026206C00283ED1606444
:10E2800084F83C002D492068084450B3B0F5007F65
:10E2900032D12B48006840F4806029490860084664
:10E2A000006800F4806526481438006840F02000BB
:10E2B0002349143908600846006800F02005032748
:10E2C0004FF000084FF003094FF0000A4FF0000B29
:10E2D00043463A4609151B488DE8000EFEF76AFED4
:10E2E0000BE01748006840F4807015490860084644
:10E2F000006800F4807500E000BF00BF206C00F0F3
:10E30000100088B9206C20F4885040F0020020648E
:10E310002046F2F78BFB00206064206C20F00200A6
:10E3200040F00100206400E0012600BF002084F8D6
:10E330003C0000BF3046BDE8FE8F000000E0FEBF9D
:10E340004438024000140240014600BF91F83C00EE
:10E35000012801D102207047012081F83C0000BF54
:10E360000868806800F0010028B90868806840F0FB
:10E3700001000A68906000BF002081F83C0000BFE7
:10E380006FF022000A6810600020E4E7014691F86F
:10E390003500022803D08020486501207047052001
:10E3A00081F835000868006820F001000A681060F4
:10E3B0000020F3E770B504460CB9012070BD94F855
:10E3C0003500022800D1F9E72068006820F001003C
:10E3D0002168086000202168086021684860216881
:10E3E00088602168C860216808612120216848612F
:10E3F0002046F3F733FE054694F85C103F20884032
:10E40000A8600020606584F8350000BF84F83400FF
:10E4100000BF00BFD2E7000070B5044600250CB96C
:10E42000012070BD00BF002084F8340000BF02202E
:10E4300084F835002068006820F001002168086039
:10E4400000BF2068006800F001000028F9D12068B2
:10E45000056822480540D4E901010843E168084302
:10E460002169084361690843A1690843E1690843D8
:10E47000216A08430543606A042803D1D4E90B01EB
:10E4800008430543206805602068456925F00705B5
:10E49000606A0543606A04280DD1A06A0543E06AFA
:10E4A00048B12046F3F7F4FD28B140206065012013
:10E4B00084F83500B5E7206845612046F3F7CEFDC6
:10E4C000064694F85C103F208840B06000206065EC
:10E4D000012084F835000020A3E700003F8010E011
:10E4E00010B50446D4F894021CF0A7FD10BD10B579
:10E4F00004460CB9012010BD032084F89102204687
:10E5000000F011FB20681EF05BFA002084F89102F5
:10E5100000BFF0E710B50446D4F894021CF0ACFD3F
:10E5200010BD10B5044620681EF05CFB10BD10B590
:10E53000044620681EF05CFB10BD024601EB81031F
:10E5400002F1380000EBC30090F824007047024647
:10E5500001EB810302F1380000EBC3004069704712
:10E5600070B504460D46002600BF94F890020128BD
:10E5700001D1022070BD012084F8900200BF29461D
:10E5800020681EF043FB00BF002084F8900200BF0B
:10E590003046EFE72DE9FE4F04460D4616461F466E
:10E5A000DDE90D9ADDF830804FF0000B00BF94F8E4
:10E5B0009002012802D10220BDE8FE8F012084F8DC
:10E5C000900200BF05EB850104F1380000F83170BE
:10E5D00005EB850100EBC100A0F808A005EB850163
:10E5E00004F1380000EBC100457005EB850104F132
:10E5F000380000EBC10080F8079006F07F0105EBC2
:10E60000850204F1380000EBC2008170C6F3C0112E
:10E6100005EB850204F1380000EBC200C17005EB88
:10E62000850104F1380000EBC10080F804808DE81A
:10E6300000073B463246294620681EF0A4FB83466D
:10E6400000BF002084F8900200BF5846B4E770472E
:10E650002DE9F05F04460D4616461F46DDE90BB96D
:10E66000DDF834A0DDF8288005EB850104F13800E1
:10E6700000EBC100C67005EB850104F1380000EB2A
:10E68000C100C771B8F1000F08D1032105EB850265
:10E6900004F1380000EBC200817207E0022105EBB3
:10E6A000850204F1380000EBC200817237B1012FFE
:10E6B0007DD0022F3DD0032F3AD182E0B8F1010F77
:10E6C00036D1AEBBB9F1000F07D1012105EB8502B0
:10E6D00004F1380000EBC200417605EB850104F13E
:10E6E000380000EBC100407E40B9002105EB8502F7
:10E6F00004F1380000EBC200817207E0022105EB53
:10E70000850204F1380000EBC200817205EB85013F
:10E7100004F1380000EBC10090F82400022807D073
:10E7200005EB850104F1380000EBC10080F805A07D
:10E7300085E05EBB05EB850104F1380000EBC1000C
:10E74000407E40B9002105EB850204F1380000EB62
:10E75000C200817207E0022105EB850204F1380056
:10E7600000EBC200817205EB850104F1380000EB7B
:10E77000C10090F82400022822D005EB850104F1A5
:10E78000380000EBC10080F805A019E005EB850119
:10E7900004F1380000EBC100007E48B9002105EB10
:10E7A000850204F1380000EBC200817208E03DE010
:10E7B000022105EB850204F1380000EBC2008172F2
:10E7C0003DE0CEB905EB850104F1380000EBC10056
:10E7D000407E40B9002105EB850204F1380000EBD2
:10E7E000C200817221E0022105EB850204F13800AC
:10E7F00000EBC200817218E005EB850104F13800DE
:10E8000000EBC100007E40B9002105EB850204F158
:10E81000380000EBC200817207E0022105EB85029F
:10E8200004F1380000EBC200817208E0002105EB22
:10E83000850204F1380000EBC200817200BF00BF06
:10E8400005EB850104F1380000EBC100C0F80CB005
:10E8500005EB850104F1380000EBC100C0F8109011
:10E86000002105EB850204F1380000EBC20080F8BE
:10E87000241005EB850204F1380000EBC200416171
:10E8800005EB850104F1380000EBC1004570002163
:10E8900005EB850204F1380000EBC20080F825107A
:10E8A000227C05EB850C04F1380303EBCC012068D6
:10E8B0001EF034FBBDE8F09F2DE9F04104462668C8
:10E8C0000025002720681EF09CF901287ED172489F
:10E8D0000088401C7049088020681EF03DFD08B982
:10E8E000BDE8F0816D4840696D49884202D06320DF
:10E8F0006C49088020681EF02FFD00F40010B0F570
:10E90000001F08D168480088401C674908804FF400
:10E9100000102168486120681EF01EFD00F4801080
:10E92000B0F5801F08D161480088401C5F4908800D
:10E930004FF480102168486120681EF00DFD00F042
:10E940008060B0F1806F08D159480088401C584958
:10E9500008804FF080602168486120681EF0FCFC50
:10E9600000F00200022807D152480088401C51499B
:10E97000088002202168486120681EF0EDFC00F04C
:10E980000050B0F1005F15D14B480088401C4A4947
:10E990000880D6F8400420F02E00C6F84004204637
:10E9A000FFF7B8FD012120681EF025FC4FF0005054
:10E9B0002168486120681EF0CFFC00F08070B0F143
:10E9C000807F09D13D480088401C00E061E03B4960
:10E9D0000880204601F04AF820681EF0BDFC00F0D7
:10E9E000080008280AD136480088401C34490880AD
:10E9F000204600F0D3F808202168486120681EF006
:10EA0000ABFC00F00070B0F1007F27D12D480088EA
:10EA1000401C2C49088020681EF079FA0746002522
:10EA200015E00120A840384080B106F5A06000EB59
:10EA30004510006800F4004020B1E9B2204600F023
:10EA400022FB03E0E9B2204600F097FD6D1CA068B0
:10EA5000A842E6D84FF000702168486120681EF097
:10EA60007BFC00F01000102813D117480088401CD0
:10EA7000154908802068806920F0100021688861AD
:10EA8000204601F0A3F82068806940F0100021685A
:10EA9000886100BF24E70000C41700200000044084
:10EAA00033000004DA170020C8170020CA1700201E
:10EAB000CC170020CE170020D0170020D21700203E
:10EAC000D4170020D6170020D817002010B58AB020
:10EAD000044614B901200AB010BD032084F8910245
:10EAE000204600F021F820681DF06AFF282204F17A
:10EAF00010016846F1F79CFB94E80F001DF002FF3F
:10EB0000012120681EF079FC282204F110016846DA
:10EB1000F1F78EFB94E80F001EF0F2FA012084F862
:10EB200091020020D7E770472DE9FE4F82464FF053
:10EB300000091448006840F00200124908600846C5
:10EB4000006800F0020902240025032600274FF088
:10EB50000C082B4622464FF470410B488DE8C0014B
:10EB6000FEF728FA0748006840F0005005490860A1
:10EB70000846006800F00059200304490860BDE819
:10EB8000FE8F0000303802400004024008E100E03F
:10EB900010B5044620681EF015FC10BD10B50446E3
:10EBA000D4F894021CF0D3FA10BD10B5044600BF8F
:10EBB00094F89002012801D1022010BD012084F8B0
:10EBC000900200BF20681DF057FF012120681DF052
:10EBD00031FF00BF002084F8900200BF00BFECE7C7
:10EBE00010B5044600BF94F89002012801D102201C
:10EBF00010BD012084F8900200BF20681EF015FCB3
:10EC000000BF002084F8900200BF00BFF0E701467B
:10EC10000846002809DB00F01F0301229A4043093F
:10EC20009B0003F1E023C3F8002100BF7047000000
:10EC30002DE9F04F05460E461746002000BF244937
:10EC40000968C1F30221084629460346B446B8467E
:10EC50001C46C4F1070BBBF1040F02D94FF0040BA3
:10EC600001E0C4F1070BDA4604F1040BBBF1070F16
:10EC700002D24FF0000B01E0A4F1030BD9464FF094
:10EC8000010B0BFA0AFBABF1010B0BEA0C0B0BFAB5
:10EC900009FB4FF0010E0EFA09FEAEF1010E0EEA6D
:10ECA000080E4BEA0E0200BF002904DB13071C0EFE
:10ECB000084B5C5409E013074FEA136C044B0C3308
:10ECC00001F00F04241F03F804C000BFBDE8F08F5B
:10ECD0000CED00E000E400E000BFFEE7816B014ABC
:10ECE00011607047E0160020F8B504460D46042771
:10ECF0000026002000902A466946204617F0A2FB15
:10ED0000064616B1A06B3043A0630098C0F34327BA
:10ED10003846F8BD2DE9F04190B006460D469046C4
:10ED20000024002742466946304617F001FB07469B
:10ED300067B140F2FF502C490860B06B3843B063B4
:10ED4000012086F8340010B0BDE8F0810098C0F3CF
:10ED500081142C700098C0F340146C700098C0F3BC
:10ED600007444FF6FF7000EA042068800098040E04
:10ED70006888204368800198C4B2200668600198C2
:10ED8000C0F30724686840EA044068600198C0F353
:10ED90000744686840EA042068600198040E6868C7
:10EDA000204368600298C4B22C720298C0F3072412
:10EDB0006C720298C0F30354AC720298040E4FF6C2
:10EDC000FF7000EA0420A8810398C4B2A8892043F8
:10EDD000A8810398C0F38524AC730398C0F3012481
:10EDE000EC730020AFE70000381C01402DE9F04330
:10EDF00087B00446884616461D46DDF83890002741
:10EE0000B8F1000F07D1A06B40F00060A0630120B3
:10EE100007B0BDE8F08394F83400012865D10020E4
:10EE2000A0637119E06D814205D9A06B40F00070BC
:10EE3000A0630120ECE7032084F83400002021685F
:10EE4000C862C4F828806802E0622068C06B48F29B
:10EE50002A1108432168C863606C012800D076023B
:10EE60004FF0FF3001906802029090200390022042
:10EE70000490002005900120069001A9206816F05A
:10EE80009BFE4A464FF40071206816F0E9FC0746E5
:10EE900057B140F2FF5021688863A06B3843A063EC
:10EEA000012084F83400B3E7012D08D90A2020633B
:10EEB0004A463146206816F011FD074607E0092052
:10EEC00020634A463146206816F027FD074657B1B1
:10EED00040F2FF5021688863A06B3843A063012093
:10EEE00084F8340094E7002092E7022090E70000C5
:10EEF00038B504460C4800780A2814D10B4800782D
:10EF000030B10F20084908700020084908700AE055
:10EF1000002003460246042100908020F4F7A2FE60
:10EF200010200149087038BDD816002001170020B4
:10EF300038B504460C480078032814D10B480078F3
:10EF400030B10420084908700020084908700AE020
:10EF5000002003460322092100908020F4F782FE5E
:10EF600005200149087038BDD81600200017002080
:10EF70002DE9F04387B00446894616461D460E9F8C
:10EF80004FF00008B9F1000F08D1A06B40F000600D
:10EF9000A0630120387007B0BDE8F08394F8340016
:10EFA00001286CD10020A0637119E06D814207D95E
:10EFB000A06B40F00070A063072038700120EAE7E2
:10EFC000032084F8340000202168C862C4F820902F
:10EFD000680260622068C06B44F21A11084321681D
:10EFE000C863606C012800D076023A464FF4007185
:10EFF000206816F035FC8046B8F1000F0BD040F2C7
:10F00000FF5021688863A06B40EA0800A0630120DC
:10F0100084F83400BFE7012D08D9282020633A4640
:10F020003146206816F08AFD804607E018202063EC
:10F030003A463146206816F0A0FD8046B8F1000F30
:10F040000BD040F2FF5021688863A06B40EA0800B3
:10F05000A063012084F834009DE74FF0FF30019059
:10F0600068020290902003900020049005900120F7
:10F07000069001A9206816F09FFD00208BE7022072
:10F08000387000BF87E72DE9F04106460C46356829
:10F09000002705F5A06000EB4410806800F0040034
:10F0A00090B1042105F5A06000EB4410816005F5E6
:10F0B000A06000EB4410C06840F0020105F5A060BC
:10F0C00000EB4410C16069E005F5A06000EB44105E
:10F0D000806800F0200030B1202105F5A06000EB31
:10F0E000441081605AE005F5A06000EB4410806890
:10F0F00000F0080028B305F5A06000EB4410C068DC
:10F1000040F0020105F5A06000EB4410C16005214C
:10F1100004EB840206F1380000EBC20080F82510F1
:10F12000102105F5A06000EB44108160082105F571
:10F13000A06000EB44108160214630681DF066FD40
:10F140002CE005F5A06000EB4410806800F48060BE
:10F1500020B305F5A06000EB4410C06840F0020148
:10F1600005F5A06000EB4410C160214630681DF039
:10F170004DFD102105F5A06000EB441081600821D1
:10F1800004EB840206F1380000EBC20080F8251081
:10F19000C90105F5A06000EB4410816005F5A06091
:10F1A00000EB4410806800F40070B8B105F5A06071
:10F1B00000EB4410C06840F0020105F5A06000EBD0
:10F1C0004410C160214630681DF020FD4FF40071ED
:10F1D00005F5A06000EB44108160CCE105F5A0606E
:10F1E00000EB4410806800F0010000287DD03069F9
:10F1F000A8B104EB840106F1380000EBC1000169FD
:10F2000005F5A06000EB44100069C0F31200091A74
:10F2100004EB840206F1380000EBC20041610121D9
:10F2200004EB840206F1380000EBC20080F82510E0
:10F23000002104EB840206F1380000EBC2000162F9
:10F24000012105F5A06000EB4410816004EB84010E
:10F2500006F1380000EBC100C07940B104EB840135
:10F2600006F1380000EBC100C079022816D105F57F
:10F27000A06000EB4410C06840F0020105F5A060FA
:10F2800000EB4410C160214630681DF0BFFC102126
:10F2900005F5A06000EB441081602BE004EB8401D5
:10F2A00006F1380000EBC100C079032822D105F532
:10F2B000A06000EB4410006840F0005105F5A0602C
:10F2C00000EB44100160012104EB840206F13800D8
:10F2D00000EBC20080F8241004EB840106F1380032
:10F2E00000EBC10090F8242000E014E021463046F5
:10F2F000FFF7ADF904EB840106F1380000EBC10023
:10F30000007E80F0010104EB840206F1380000EB7E
:10F31000C20001762FE105F5A06000EB4410806883
:10F3200000F00200002871D005F5A06000EB441049
:10F33000C06820F0020105F5A06000EB4410C16038
:10F3400004EB840106F1380000EBC10090F82500C1
:10F35000012809D1012104EB840206F1380000EBF9
:10F36000C20080F8241069E004EB840106F1380043
:10F3700000EBC10090F82500052809D1052104EB18
:10F38000840206F1380000EBC20080F8241055E03A
:10F3900004EB840106F1380000EBC10090F8250071
:10F3A000062809D004EB840106F1380000EBC10007
:10F3B00090F82500082841D104EB840106F13800BB
:10F3C00000EBC10004EB8401026A06F1380000EB97
:10F3D000C100006A401C04EB840306F1380101EB14
:10F3E000C3010862032A12D9002104EB840206F14A
:10F3F000380000EBC2000162042104EB840206F134
:10F40000380000EBC20080F8241009E029E0022156
:10F4100004EB840206F1380000EBC20080F82410EF
:10F4200005F5A06000EB4410076827F0804747F01F
:10F43000004705F5A06000EB44100760022105F5C8
:10F44000A06000EB4410816004EB840106F13800F9
:10F4500000EBC10090F8242021463046FFF7F7F872
:10F4600089E005F5A06000EB4410806800F08000A2
:10F4700070B305F5A06000EB4410C06840F00201D5
:10F4800005F5A06000EB4410C16004EB840106F1B7
:10F49000380000EBC100006A401C04EB840206F156
:10F4A000380101EBC2010862062104EB840206F177
:10F4B000380000EBC20080F82510214630681DF0AE
:10F4C000A5FB802105F5A06000EB4410816052E0AF
:10F4D000FFE705F5A06000EB4410806800F0100025
:10F4E000E0B304EB840106F1380000EBC100C07901
:10F4F000032810D105F5A06000EB4410C06840F06F
:10F50000020105F5A06000EB4410C160214630689F
:10F510001DF07CFB1EE004EB840106F1380000EBDB
:10F52000C100C07940B104EB840106F1380000EB62
:10F53000C100C07902280DD105F5A06000EB441090
:10F54000076827F0804747F0004705F5A06000EB0B
:10F5500044100760032104EB840200E00BE006F195
:10F56000380000EBC20080F82510102105F5A060DE
:10F5700000EB44108160BDE8F0812DE9F0410546C3
:10F580000C462E68002706F5A06000EB441080684A
:10F5900000F0040090B1042106F5A06000EB4410D7
:10F5A000816006F5A06000EB4410C06840F00201E5
:10F5B00006F5A06000EB4410C16054E206F5A060BF
:10F5C00000EB4410806800F0200088B3202106F58D
:10F5D000A06000EB4410816004EB840105F1380069
:10F5E00000EBC10040790128E7D1042104EB84023B
:10F5F00005F1380000EBC20080F8251006F5A06088
:10F6000000EB4410C06840F0020106F5A06000EB7A
:10F610004410C160214628681DF0F8FA022104EB6D
:10F62000840205F1380000EBC20080F824101AE2D1
:10F63000FFE706F5A06000EB4410806800F0400092
:10F6400038B3042104EB840205F1380000EBC2005A
:10F6500080F82510002104EB840205F1380000EB4E
:10F66000C200016206F5A06000EB4410C06840F0E3
:10F67000020106F5A06000EB4410C1602146286835
:10F680001DF0C4FA402106F5A06000EB4410816033
:10F69000E9E106F5A06000EB4410806800F400701A
:10F6A000B8B106F5A06000EB4410C06840F002015C
:10F6B00006F5A06000EB4410C160214628681DF0EB
:10F6C000A5FA4FF4007106F5A06000EB44108160CC
:10F6D000C9E106F5A06000EB4410806800F001006D
:10F6E00030B3002104EB840205F1380000EBC200C6
:10F6F000016206F5A06000EB4410C06840F0020112
:10F7000006F5A06000EB4410C160214628681DF09A
:10F710007DFA012106F5A06000EB4410816004EB46
:10F72000840205F1380000EBC20080F825109AE150
:10F7300006F5A06000EB4410806800F00800F8B106
:10F74000082106F5A06000EB4410816006F5A0607A
:10F7500000EB4410C06840F0020106F5A06000EB29
:10F760004410C160214628681DF050FA052104EBC1
:10F77000840205F1380000EBC20080F8251072E128
:10F7800006F5A06000EB4410806800F0100038B36C
:10F79000002104EB840205F1380000EBC200016295
:10F7A00006F5A06000EB4410C06840F0020106F5C9
:10F7B000A06000EB4410C160214628681DF026FAC5
:10F7C000032104EB840205F1380000EBC20080F84D
:10F7D0002510102106F5A06000EB4410816042E185
:10F7E00006F5A06000EB4410806800F08000F8B1DE
:10F7F00006F5A06000EB4410C06840F0020106F579
:10F80000A06000EB4410C160214628681DF0FEF99D
:10F81000062104EB840205F1380000EBC20080F8F9
:10F820002510802106F5A06000EB441081601AE1EC
:10F8300006F5A06000EB4410806800F4806028B3F7
:10F8400006F5A06000EB4410C06840F0020106F528
:10F85000A06000EB4410C160214628681DF0D6F975
:10F86000102106F5A06000EB44108160890106F5C7
:10F87000A06000EB44108160082104EB840205F1D4
:10F88000380000EBC20080F82510ECE006F5A0601F
:10F8900000EB4410806800F0020000289FD006F5BD
:10F8A000A06000EB4410C06820F0020106F5A060E3
:10F8B00000EB4410C16004EB840105F1380000EB5B
:10F8C000C10090F82500012822D1012104EB840217
:10F8D00005F1380000EBC20080F8241004EB84012D
:10F8E00005F1380000EBC100C07902280FD104EB0C
:10F8F000840105F1380000EBC100407E80F0010179
:10F9000004EB840205F1380000EBC200417698E078
:10F9100004EB840105F1380000EBC10090F82500EC
:10F92000032809D1022104EB840205F1380000EB21
:10F93000C20080F8241084E004EB840105F1380053
:10F9400000EBC10090F82500042811D1022104EB3E
:10F95000840205F1380000EBC20080F82410002179
:10F9600004EB840205F1380000EBC200417168E04D
:10F9700004EB840105F1380000EBC10090F825008C
:10F98000052809D1052104EB840205F1380000EBBC
:10F99000C20080F8241054E004EB840105F1380023
:10F9A00000EBC10090F82500062809D004EB840183
:10F9B00005F1380000EBC10090F82500082840D17F
:10F9C00004EB840105F1380000EBC10004EB840175
:10F9D000026A05F1380000EBC100006A401C04EB2C
:10F9E000840305F1380101EBC3010862032A11D930
:10F9F000002104EB840205F1380000EBC200016233
:10FA0000042104EB840205F1380000EBC20080F809
:10FA1000241008E0022104EB840205F1380000EB19
:10FA2000C20080F8241006F5A06000EB44100768BF
:10FA300027F0804747F0004706F5A06000EB441030
:10FA40000760022106F5A06000EB4410816004EB22
:10FA5000840105F1380000EBC10090F82420214614
:10FA60002846FEF7F4FDBDE8F08100007CB50446B1
:10FA70004C480088401C4B4908802568D5F8400454
:10FA80000190D5F840040090009820F02E000090DE
:10FA9000019800F0020002281AD143480088401C57
:10FAA00041490880019800F0010068B13F48008892
:10FAB000401C3E4908802068806920F00050216881
:10FAC00088612046FEF70CFD009840F0020000908F
:10FAD000019800F00800082851D135480088401CE2
:10FAE00033490880009840F008000090019800F029
:10FAF0000400042837D12F480088401C2D49088075
:10FB0000A06902281ED12C480088401C2A49088080
:10FB1000019800F4C020B0F5802F09D12748008853
:10FB2000401C26490880022120681DF064FB16E075
:10FB300023480088401C22490880012120681DF0CC
:10FB40005AFB0CE0E068032809D11E480088401CDD
:10FB50001C4908804EF6602140F204404151204685
:10FB6000FEF7BEFC0BE0D5F8400420F02E00C5F8EF
:10FB700040042068806940F0005021688861019845
:10FB800000F02000202808D10F480088401C0E49B2
:10FB90000880009840F0200000900098C5F84004CC
:10FBA0007CBD0000DC170020DE170020E0170020DD
:10FBB000E2170020E4170020E6170020E8170020D5
:10FBC000EA170020EC170020EE1700202DE9F0477F
:10FBD00005462F680024A046A1462868D0F820805A
:10FBE00008F00F04C8F3434AC8F30A16BAF1020F2B
:10FBF00009D0BAF1030F66D0BAF1050F61D0BAF19E
:10FC0000070F5FD160E0002E5AD004EB840105F1AC
:10FC1000380000EBC100C068E8B3B2B204EB840C5A
:10FC200005F1380303EBCC03D96828681DF09AFB73
:10FC300004EB840105F1380000EBC100C0688119B4
:10FC400004EB840205F1380000EBC200C16004EB54
:10FC5000840105F1380000EBC1004069811904EB13
:10FC6000840205F1380000EBC200416107F5A06095
:10FC700000EB441000691649084060B107F5A06028
:10FC800000EB4410D0F8009029F0804949F0004979
:10FC900007F5A06000E013E000EB4410C0F800900E
:10FCA00004EB840105F1380000EBC100007E80F018
:10FCB000010104EB840205F1380000EBC20001767B
:10FCC00003E002E000BF00BF00BF00BFBDE8F08757
:10FCD0000000F81F10B50DF0B1FC04461CB918F077
:10FCE00035FA012010BD0020FCE7000010B51049D6
:10FCF00091F822000DF0C2FD28B90D4991F82200BB
:10FD00000DF0ADFD10B10DF0C1FE10E0084991F805
:10FD100022000DF0BDFD50B10548408E4FF6FF7139
:10FD2000884202D10CF078FE01E00DF093FC10BD8A
:10FD3000000D022000B58BB000200A900521EEA036
:10FD400009F098FE38B102F069FD12F0E5FD0120DE
:10FD50000A9002F073BB0921E9A009F08BFE30B1D3
:10FD600018F01EFC12F0C2FD01200A90F1E70B21F1
:10FD7000E6A009F07FFE30B1F1F70EFE12F096FD1D
:10FD800001200A90E5E70D21E3A009F073FE20B100
:10FD900012F08CFD01200A90DBE70C21E2A009F0B3
:10FDA00069FE30B1F1F704FE12F0C2FD01200A90A5
:10FDB000CFE70E21E0A009F05DFE20B112F0B8FD02
:10FDC00001200A90C5E70C21DFA009F053FE30B1F5
:10FDD00012F0E2FD12F032FD01200A90B9E70B218A
:10FDE000DCA009F047FE20B112F03EFD01200A9090
:10FDF000AFE70421DAA009F021FE98B104200190B8
:10FE0000002209A901A809F09BFF0028A1D0BDF894
:10FE10002400C0B2009002F01FFC002899D00120FD
:10FE20000A9096E70821D0A009F008FED0B108207A
:10FE30000190002209A901A809F082FF002888D0BA
:10FE4000BDF92400002884DBBDF924000E288DDADA
:10FE50000020C849BDF92420885412F047FD012034
:10FE60000A9076E70721C4A009F0E8FD70B30720E7
:10FE70000190012209A901A809F062FF00288BD096
:10FE8000BDF92400002887DBBDF924000E288FDA95
:10FE9000002208A901A809F053FF002888D00120FA
:10FEA000B449BDF9242088540020B549BDF9242067
:10FEB00021F81200BDF82000B249BDF9242021F834
:10FEC000120012F013FD01200A9042E70921AEA0B2
:10FED00009F0B4FDA8B30020009009200190012290
:10FEE00009A901A809F02CFF50B3BDF9240010B1F5
:10FEF00001281AD10CE00022694601A809F020FF70
:10FF000028B1BDF90000A349088001200A900DE046
:10FF10000022694601A809F013FF28B1BDF90000CD
:10FF20009D49088001200A9000E000BF00BF0A98A8
:10FF300030B101209949BDF92420885412F0B6FC53
:10FF400007E7FFE70A2196A009F078FDD0B10A2063
:10FF50000190002209A901A809F0F2FE0028B4D0FE
:10FF6000BDF924000028B0DBBDF924000228ACDA7A
:10FF700000208A49BDF92420885412F097FC012002
:10FF80000A90E6E6092189A009F058FDD0B10920C0
:10FF90000190002209A901A809F0D2FE002894D0FE
:10FFA000BDF92400002890DBBDF924000B288CDA71
:10FFB00001208149BDF92420885412F0B9FC0120A8
:10FFC0000A90C6E60A217DA009F038FDD0B10A20CA
:10FFD0000190002209A901A809F0B2FE0028AFD0C3
:10FFE000BDF924000028ABDBBDF924000B28A7DAFB
:10FFF00000207149BDF92420885412F099FC012099
:020000040802F0
:100000000A90A6E6082170A009F018FDD0B10820DA
:100010000190002209A901A809F092FE00288FD0C2
:10002000BDF9240000288BDBBDF924000D2887DAF8
:1000300001206849BDF92420885412F0FFFB0120FB
:100040000A9086E6092164A009F0F8FCD0B10920E5
:100050000190002209A901A809F072FE002890D0A1
:10006000BDF9240000288CDBBDF924000D2888DAB6
:1000700000205849BDF92420885412F0DFFB0120EC
:100080000A9066E6092157A009F0D8FCC8B10920FA
:100090000190002209A901A809F052FE002890D081
:1000A000BDF9240000288CDBBDF924000D2888DA76
:1000B000BDF8240080B2009012F086FB01200A9067
:1000C00047E604214AA009F0B9FC002899D0042091
:1000D0000190022209A901A809F032FE002890D05F
:1000E000BDF92400AB2801F0B28203DCAB2882F01A
:1000F000A48181E0DCE1000052455345540000003A
:10010000504F4C4C535F4F4646000000494E4A4505
:100110004354535F4F464600494E4A454354535F4C
:1001200051554552590000005357495443484553CF
:100130005F4F46460000000053574954434845531B
:100140005F515545525900004556454E54535F4F37
:100150004646000046494E4745525052494E5400CB
:100160005245414400000000504F4C4C5F4F464602
:1001700000000000B6270120504F4C4C5F4F4E004E
:100180007E2701209A270120494E4A4543545F4F5C
:100190004E0000000214002004140020001400206F
:1001A000494E4A4543545F4F464600005357495411
:1001B00043485F4F4E000000C42701205357495465
:1001C00043485F4F464600004556454E545F4F4EEC
:1001D000000000006C2801204556454E545F4F46F4
:1001E000460000004556454E545F47455400000008
:1001F00043414C4C00000000810000BF7944496835
:100200008F440000680500007E0500009205000094
:10021000A6050000B6050000C6050000D6050000D2
:10022000E6050000F60500000606000016060000C0
:10023000260600003606000046060000660600009E
:10024000760600008606000096060000A60600005E
:10025000B6060000CA060000EE0600000207000015
:10026000260700003A0700005E0700007207000042
:10027000860700009A070000AA070000CE070000CA
:10028000E2070000F607000006080000160800005C
:100290003A0800007008000090080000A008000064
:1002A000D2080000E6080000180900002C09000030
:1002B00040090000500900006409000078090000AE
:1002C0009C090000B0090000C4090000D409000026
:1002D000E4090000F4090000040A0000180A000004
:1002E000280A0000380A0000480A0000660A0000D8
:1002F0007A0A00008E0A0000A20A0000B60A000076
:10030000CA0A0000DE0A0000F20A0000060B000024
:100310001A0B00002E0B0000420B0000520B0000D5
:10032000660B00007A0B00008E0B00009E0B000095
:10033000AE0B0000C20B0000D60B0000EA0B000061
:100340000E0C0000220C0000520C0000820C000079
:10035000960C0000AA0C0000BE0C0000D20C00009D
:10036000E60C0000FA0C00000A0D00002E0D000043
:10037000620D0000760D00008A0D00009E0D000049
:10038000B20D0000C60D0000DA0D0000EE0D0000F9
:10039000020E0000160E00002A0E00003E0E0000A5
:1003A000520E0000660E00007A0E00008E0E000055
:1003B000A20E0000B60E0000CA0E0000DE0E000005
:1003C000F20E0000060F00001A0F00002E0F0000B2
:1003D000520F0000760F00009A0F0000BE0F0000C1
:1003E000F20F0000061000001A1000002E1000008E
:1003F00042100000561000006A1000007E1000003D
:1004000092100000A6100000BA100000CE100000EC
:10041000E2100000F61000000A1100004E1100006A
:100420007E11000092110000A6110000BA11000018
:10043000CE110000E2110000F61100000A120000C7
:100440001E12000032120000461200005A12000074
:100450006E1200008212000096120000AA12000024
:10046000BE120000D2120000E6120000FA120000D4
:100470000E13000022130000361300004613000084
:100480005A1300007A1300008E130000A21300001C
:10049000B6130000C6130000D6130000E6130000D8
:1004A000FA1300000E14000022140000361400009D
:1004B000AC38AA2881F0C187810000BF794449681F
:1004C0008F4400009E110000B2110000C611000010
:1004D000DA110000EE1100000212000016120000F6
:1004E0002A1200003E1200005212000066120000A4
:1004F0007A1200008E120000A2120000B612000054
:10050000CA120000DE120000F21200000613000002
:100510001A1300002E1300004213000056130000AF
:100520006A1300007E13000092130000A61300005F
:10053000BA130000CE130000E2130000F61300000F
:100540000A1400001E1400003214000046140000BB
:100550005A1400006E14000082140000961400006B
:10056000AA140000BE140000D2140000E61400001B
:10057000FA1400000E1500002215000036150000C8
:100580004A1500005E150000721500008615000077
:100590009A150000AE150000C2150000D615000027
:1005A000EA150000FE1500001216000026160000D5
:1005B0003A1600004E160000621600007616000083
:1005C0008A1600009E160000B2160000C616000033
:1005D000DA160000EE1600000217000016170000E1
:1005E0002A1700003E17000052170000661700008F
:1005F0007A1700008E170000A2170000B61700003F
:10060000CA170000DE170000EE170000FE170000FA
:1006100012180000261800003C1800004E180000B8
:100620006418000076180000881800009A1800006E
:10063000AC180000C2180000D8180000EA1800002A
:1006400000190000161900002C19000042190000C2
:10065000581900006E190000841900009A19000052
:10066000B0190000C6190000DC190000F2190000E2
:10067000081A00001E1A0000341A00004A1A00006E
:10068000601A0000761A00008C1A0000A21A0000FE
:10069000B81A0000CE1A0000E41A0000FA1A00008E
:1006A0000C1B00001E1B0000341B00004A1B000036
:1006B0007C1B00009E1B0000B01B0000C21B000042
:1006C000D41B0000EA1B0000001C0000161C0000E8
:1006D0002C1C00003E1C0000501C0000661C00008A
:1006E0007C1C0000921C0000A81C0000BE1C000026
:1006F000D01C0000E61C0000FC1C0000121D0000C5
:10070000281D00003E1D0000541D00006A1D000051
:10071000801D0000961D0000AC1D0000C21D0000E1
:10072000D81D0000EE1D0000041E00001A1E00006F
:100730002C1E0000421E0000581E00006E1E00000D
:10074000841E00009A1E0000B01E0000C61E00009D
:10075000DC1E0000F21E0000081F00001E1F00002B
:10076000341F00004A1F0000601F0000FDF776F8EC
:1007700001460090002011F0EBFF01200A9001F0EB
:100780005CBEF6F77DF801460090012011F086FF6F
:1007900001200A90F3E7F6F76DF801460090022079
:1007A00011F0D6FF01200A90E9E7F6F707F90320D8
:1007B00011F060FF01200A90E1E7F6F7ACF80420A1
:1007C00011F058FF01200A90D9E7F6F795F80520B7
:1007D00011F050FF01200A90D1E7F6F7A1F80620AA
:1007E00011F048FF01200A90C9E7F6F78FF80720BB
:1007F00011F040FF01200A90C1E7F6F782F80820C7
:1008000011F038FF01200A90B9E7F4F730FD092014
:1008100011F030FF01200A90B1E7F4F72DFD0A2016
:1008200011F028FF01200A90A9E7F4F739FD0B2009
:1008300011F020FF01200A90A1E7F4F722FD0C201F
:1008400011F018FF01200A9099E7002206A901A8DB
:1008500009F01EFB40B1BDF81800F4F717FD0D209C
:1008600011F008FF01200A9089E7F4F7F1FC0E204F
:1008700011F000FF01200A9081E7F4F7F3FC0F204C
:1008800011F0F8FE01200A9079E7F4F7E6FC102059
:1008900011F0F0FE01200A9071E7F6F799F81120A7
:1008A00011F0E8FE01200A9069E703F003FD122031
:1008B00011F0E0FE01200A9061E703F0D5FC01464B
:1008C0000090132011F0EAFE01200A9057E7002261
:1008D00004A901A809F034FA50B1BDF81000C0B263
:1008E000009003F0CBFC142011F0C4FE01200A900C
:1008F00045E703F06FFC01460090152011F0CEFE95
:1009000001200A903BE7002204A901A809F018FA87
:1009100050B1BDF81000C0B2009003F065FC162085
:1009200011F0A8FE01200A9029E703F0CFFC014650
:100930000090172011F0B2FE01200A901FE700225C
:1009400004A901A809F0FCF950B1BDF81000C0B22B
:10095000009003F0C5FC182011F08CFE01200A90D5
:100960000DE703F047FC01460090192011F096FEB8
:1009700001200A9003E703F087FC014600901A204B
:1009800011F08CFE01200A90F9E603F089FC014683
:1009900000901B2011F082FE01200A90EFE61FF06C
:1009A000A3FC1C2011F066FE01200A90E7E600225D
:1009B00004A901A809F0C4F950B1BDF81000C0B2F3
:1009C00000901FF07DFC1D2011F054FE01200A90C4
:1009D000D5E61FF0D3F9014600901E2011F0D6FE97
:1009E00001200A90CBE61FF0E3F9014600901F209A
:1009F00011F0CCFE01200A90C1E620F06BFB202014
:100A000011F038FE01200A90B9E618F02FFB2120E2
:100A100011F030FE01200A90B1E6002204A901A8DD
:100A200009F08EF950B1BDF81000C0B2009018F076
:100A300075FB222011F01EFE01200A909FE6012284
:100A400006A901A809F024FA98B1002204A901A876
:100A500009F076F968B1BDF81000C0B20146009007
:100A6000BDF8180018F068FB232011F003FE0120E8
:100A70000A9084E6002206A901A809F009FA40B10B
:100A8000BDF8180018F008FB242011F0F3FD012038
:100A90000A9074E618F0FCFA252011F0EBFD012015
:100AA0000A906CE6012207A901A809F077FA88B13B
:100AB000002206A901A809F0EBF958B1BDF81810F9
:100AC000079818F055FB01460090262011F0E6FD2E
:100AD00001200A9053E618F045FB014600902720BC
:100AE00011F0DCFD01200A9049E6012207A901A8C6
:100AF00009F054FA88B1002206A901A809F0C8F942
:100B000058B1BDF81810079818F0F6FA0146009091
:100B1000282011F0C3FD01200A9030E618F0E6FA13
:100B200001460090292011F0B9FD01200A9026E627
:100B300018F0AAFA014600902A2011F0AFFD01201A
:100B40000A901CE60FF0C4F92B2011F093FD012050
:100B50000A9014E60FF0BEF8014600902C2011F028
:100B6000D9FD01200A900AE60FF010F90146009025
:100B70002D2011F0B1FD01200A9000E6002202A90B
:100B800001A808F095FF50B19DED020B0FF080F920
:100B9000014600902E2011F0BDFD01200A90EEE5E7
:100BA000FCF778FD014600902F2011F0EFFD0120A9
:100BB0000A90E4E5FCF7B2FD01460090302011F008
:100BC000E5FD01200A90DAE5FCF758FD312011F02F
:100BD00051FD01200A90D2E5FCF7EEFC322011F025
:100BE00049FD01200A90CAE50CF02CFE332011F0DB
:100BF00041FD01200A90C2E50CF07EFF342011F087
:100C000039FD01200A90BAE5F3F7BAF801460090E1
:100C1000352011F07FFD01200A90B0E5F3F7F0FADE
:100C2000362011F027FD01200A90A8E5F3F7EEFA2F
:100C3000372011F01FFD01200A90A0E5F3F780F89E
:100C4000382011F017FD01200A9098E5002207A92D
:100C500001A809F0A3F938B10798F3F7CBFA3920C6
:100C600011F008FD01200A9089E5F3F7B5F9014676
:100C700000903A2011F08AFD01200A907FE5F3F7F9
:100C8000B3F9014600903B2011F080FD01200A904D
:100C900075E5F3F7AEF9014600903C2011F076FDC2
:100CA00001200A906BE5F3F749F8014600903D20DA
:100CB00011F06CFD01200A9061E5F3F711FA01468D
:100CC00000903E2011F062FD01200A9057E5EFF7F9
:100CD00055FE014600903F2011F03AFD01200A9098
:100CE0004DE5EFF777FE01460090402011F030FD12
:100CF00001200A9043E51BF06FFF01460090412060
:100D000011F0CCFC01200A9039E51BF0E7FE01460A
:100D10000090422011F0C2FC01200A902FE51BF048
:100D2000E7FE01460090432011F0B8FC01200A9034
:100D300025E51BF0C1FE01460090442011F0AEFCF9
:100D400001200A901BE51BF0A5FE452011F092FC46
:100D500001200A9013E51BF097FE01460090462003
:100D600011F09CFC01200A9009E51CF0CFFA014625
:100D70000090472011F092FC01200A90FFE41CF043
:100D8000D1FA01460090482011F088FC01200A9019
:100D9000F5E41CF0D9FA492011F06CFC01200A900E
:100DA000EDE41CF0CBFA4A2011F064FC01200A901B
:100DB000E5E416F0A7FA014600904B2011F06EFC16
:100DC00001200A90DBE416F053FA014600904C2013
:100DD00011F0BEFC01200A90D1E416F07FFA014622
:100DE00000904D2011F096FC01200A90C7E40022EB
:100DF00006A901A809F04CF850B1BDF8180016F08A
:100E0000C9FA014600904E2011F048FC01200A90DA
:100E1000B5E418F013FF014600904F2011F03EFC9E
:100E200001200A90ABE4012206A901A809F030F8DC
:100E300080B1002205A901A809F02AF850B1BDF837
:100E40001410BDF8180019F01FF8502011F012FC12
:100E500001200A9093E4012206A901A809F018F8DC
:100E600080B1002205A901A809F012F850B1BDF81F
:100E70001410BDF8180019F01DF8512011F0FAFBFC
:100E800001200A907BE40BF0B1FA01460090522059
:100E900011F004FC01200A9071E40BF0A1FA014664
:100EA0000090532011F054FC01200A9067E417F0E1
:100EB000F5FE01460090542011F0F0FB01200A904D
:100EC0005DE417F0DFFE01460090552011F0E6FBCF
:100ED00001200A9053E417F0DBFE014600905620F3
:100EE00011F0DCFB01200A9049E417F0B5FD014642
:100EF0000090572011F04AFC01200A903FE417F0BF
:100F000083FF582011F0B6FB01200A9037E400223D
:100F100006A901A808F0BCFF50B1BDF8180017F0F1
:100F200029FD01460090592011F030FC01200A9063
:100F300025E4012206A901A808F0AAFF90B1002229
:100F400005A901A808F0A4FF60B1BDF81410BDF810
:100F5000180017F037FD014600905A2011F016FCDA
:100F600001200A900BE417F0C5FD014600905B20BC
:100F700011F00CFC01200A900CE417F0C3FD0146AF
:100F800000905C2011F002FC01200A900CE417F0A4
:100F9000A9FD014600905D2011F0F8FB01200A90A8
:100FA0000AE417F0B7FD014600905E2011F0EEFB59
:100FB00001200A9008E417F0B5FD014600905F207B
:100FC00011F0E4FB01200A9006E417F0DFFD014672
:100FD0000090602011F0DAFB01200A9004E417F081
:100FE000BBFD01460090612011F0D0FB01200A906A
:100FF0000AE417F0E5FD01460090622011F0C6FBFF
:1010000001200A9008E417F04FFE0146009063208B
:1010100011F080FB01200A9006E417F0C3FE0146A0
:101020000090642011F0B2FB01200A9004E417F054
:10103000C3FE01460090652011F0A8FB01200A9034
:1010400012E417F003FF01460090662011F026FB22
:1010500001200A9008E417F0EBFE0146009067209B
:1010600011F01CFB01200A9006E417F053FE014624
:101070000090682011F08AFB01200A9004E417F028
:1010800029FE01460090692011F080FB01200A90A2
:101090000AE417F077FE014600906A2011F076FB13
:1010A00001200A9008E417F05DFE014600906B20D5
:1010B00011F06CFB01200A9008E417F01BFE0146BA
:1010C00000906C2011F062FB01200A9010E417F0F0
:1010D00031FE014600906D2011F058FB01200A906E
:1010E00006E417F09FFF014600906E2011F04EFBC2
:1010F00001200A9006E417F0CDFC014600906F2015
:1011000011F0CCFA01200A900EE417F073FD0146AD
:101110000090702011F0C2FA01200A9004E417F048
:101120008DFD01460090712011F0B8FA01200A905F
:1011300004E4002206A901A808F0AAFE50B1BDF8F7
:10114000180017F0F7FC01460090722011F01EFB0A
:1011500001200A9004E4002206A901A808F098FEE4
:1011600050B1BDF8180017F019FD0146009073202A
:1011700011F00CFB01200A9006E4002206A901A848
:1011800008F086FE50B1BDF8180017F0EDFC0146DE
:101190000090742011F0FAFA01200A9006E400226F
:1011A00006A901A808F074FE50B1BDF8180017F0A8
:1011B0000FFD01460090752011F0E8FA01200A9019
:1011C00006E4012206A901A808F062FE90B10022FF
:1011D00005A901A808F05CFE60B1BDF81410BDF8C7
:1011E000180017F095FB01460090762011F0CEFA1A
:1011F00001200A9008E418F089F801460090772051
:1012000011F04CFA01200A9006E418F067F8014644
:101210000090782011F042FA01200A900EE418F0B4
:1012200063F801460090792011F038FA01200A9005
:1012300004E418F05FF8014600907A2011F02EFACD
:1012400001200A9015E418F05BF8014600907B201D
:1012500011F024FA01200A900BE417F0C9FF0146AF
:1012600000907C2011F01AFA01200A9011E418F085
:101270000DF8014600907D2011F010FA01200A902F
:1012800007E417F0F5FF014600907E2011F006FA02
:1012900001200A9005E417F0B8FF014600907F2076
:1012A00011F0FCF901200A9014E417F0BAFF01468E
:1012B0000090802011F0F2F901200A900AE417F062
:1012C000CAFF01460090812011F0E8F901200A9040
:1012D0000AE417F0B3FF01460090822011F0DEF916
:1012E00001200A9019E417F0DDFF014600908320E9
:1012F00011F0D4F901200A900FE417F0E1FF014644
:101300000090842011F0CAF901200A9005E401221E
:1013100004A901A808F014FDD0B1012206A901A872
:1013200008F0B6FDA0B1002205A901A808F0B0FDA3
:1013300070B1BDF81000C0B20090BDF81420BDF827
:10134000181018F0D3F8852011F094F901200A90B4
:1013500009E4012206A901A808F09AFD80B1002243
:1013600005A901A808F094FD50B1BDF81410BDF80E
:10137000180018F0CEF8862011F07CF901200A90B0
:101380000DE403F0B9FB01460090872011F086F9C7
:1013900001200A900DE403F007FF01460090882029
:1013A00011F0F4F901200A900DE403F005FB014669
:1013B0000090892011F0CCF901200A900BE403F091
:1013C00019FF014600908A2011F0E0F901200A90EF
:1013D00009E404F0FFFC014600908B2011F0D6F9DF
:1013E00001200A9007E404F0E3FA014600908C2003
:1013F00011F0CCF901200A9005E404F005FB014648
:1014000000908D2011F0C2F901200A9005E403F04C
:1014100033FB014600908E2011F040F901200A9024
:101420000BE403F0CFFA014600908F2011F072F91F
:1014300001200A9009E403F02BFB01460090902064
:1014400011F068F901200A900EE403F02DFB01462B
:101450000090912011F05EF901200A9004E403F05D
:1014600011FB01460090922011F054F901200A90DE
:1014700004E403F087FE01460090932011F086F902
:1014800001200A9004E403F009FB01460090942037
:1014900011F040F901200A9004E403F00BFB01462F
:1014A0000090952011F036F901200A9004E402F032
:1014B0004DFF01460090962011F02CF901200A9072
:1014C00004E402F07BFE01460090972011F022F91F
:1014D00001200A9004E404F05FFA0146009098208D
:1014E00011F018F901200A9004E402F04FFE0146C1
:1014F0000090992011F00EF901200A9004E402F006
:1015000051FE014600909A2011F004F901200A9042
:1015100004E403F045FA014600909B2011F0FAF82C
:1015200001200A9004E403F041FA014600909C2057
:1015300011F0F0F801200A9004E404F095F89D20E1
:1015400011F098F801200A9004E403F0E5FA01464E
:1015500000909E2011F0A2F801200A9004E40022DD
:1015600006A901A808F094FC40B1BDF8180004F0E9
:101570003BFC9F2011F07EF801200A9008E404F063
:10158000B9F901460090A02011F088F801200A90D6
:1015900006E404F0F5F901460090A12011F07EF870
:1015A00001200A9004E415F043FF01460090A220B8
:1015B00011F0B0F801200A9004E415F02BFFA320ED
:1015C00011F058F801200A9006E415F019FFA42044
:1015D00011F050F801200A9008E415F007FFA5204B
:1015E00011F048F801200A9012E411F0E3FD0146E1
:1015F0000090A62011F08EF801200A9008E411F066
:1016000043FD01460090A72011F048F801200A9000
:1016100008E411F04BFD01460090A82011F07AF883
:1016200001200A9016E411F047FD01460090A92020
:1016300011F070F801200A900CE411F0A9FD0146A8
:101640000090AA2011F066F801200A901AE411F027
:1016500093FD01460090AB2011F05CF801200A9048
:1016600010E411F09BFD01460090AC2011F052F8FF
:1016700001200A9006E411F097FD01460090AD208C
:1016800011F048F801200A9006E411F07BFD0146B4
:101690000090AE2011F03EF801200A9006E411F00F
:1016A00065FD01460090AF2011F034F801200A904A
:1016B00006E411F007FD01460090B02011F02AF871
:1016C00001200A9006E411F01BFD01460090B120B4
:1016D00011F020F801200A9006E411F0FFFC014609
:1016E0000090B22011F016F801200A9006E411F0E3
:1016F000EFFC01460090B32011F00CF801200A9095
:1017000004E411F0F1FC01460090B42011F002F85D
:1017100001200A900CE411F0EDFC01460090B52088
:1017200010F0F8FF01200A901CE411F0EFFC0146D4
:101730000090B62010F0EEFF01200A9012E411F0A4
:10174000EBFC01460090B72010F0E4FF01200A9066
:1017500008E411F0FFFC01460090B82010F0DAFF19
:1017600001200A9008E411F0E3FC01460090B92042
:1017700010F0D0FF01200A9008E411F0D3FC0146DC
:101780000090BA2010F0C6FF01200A9008E411F082
:10179000D5FC01460090BB2010F0BCFF01200A9050
:1017A00008E411F0D1FC01460090BC2010F0B2FF1B
:1017B00001200A9008E411F0D3FC01460090BD20FE
:1017C00010F0A8FF01200A9008E411F063FC014624
:1017D0000090BE2010F09EFF01200A9008E411F056
:1017E0005FFC01460090BF2010F0B2FF01200A907C
:1017F00008E412F02FFD01460090C02010F04EFFCB
:1018000001200A9008E411F00FFC01460090C1206D
:1018100010F0BCFF01200A9008E411F029FC0146F9
:101820000090C22010F0B2FF01200A9008E411F0ED
:10183000F5FB01460090C32010F06CFF01200A90D8
:1018400008E411F00FFC01460090C42010F080FF66
:1018500001200A9008E411F011FC01460090C52017
:1018600010F094FF01200A9008E411F0F5FB014606
:101870000090C62010F08AFF01200A9008E411F0C1
:10188000C7FB01460090C72010F080FF01200A909E
:1018900008E411F0D5FB01460090C82010F03AFF93
:1018A00001200A9008E411F0D1FB01460090C92004
:1018B00010F06CFF01200A9008E411F0BBFB014618
:1018C0000090CA2010F062FF01200A9008E411F095
:1018D0009DFA01460090CB2010F058FF01200A909D
:1018E00008E411F029FB01460090CC2010F04EFFD7
:1018F00001200A9008E411F025FB01460090CD205C
:1019000010F044FF01200A9008E411F0F7FA0146B4
:101910000090CE2010F03AFF01200A9008E411F068
:10192000C9FA01460090CF2010F030FF01200A9044
:1019300010E411F077FA01460090D02010F0EAFE92
:1019400001200A9006E411F0EBFA01460090D12044
:1019500010F01CFF01200A900EE411F0D5FA0146A8
:101960000090D22010F012FF01200A9004E411F040
:10197000F5FA01460090D32010F008FF01200A90EC
:101980000CE411F0D3FA01460090D42010F0FEFED2
:1019900001200A9014E411F057FA01460090D52076
:1019A00010F0F4FE01200A900AE411F053FA014607
:1019B0000090D62010F0CCFE01200A901AE411F01D
:1019C00085FA01460090D72010F0E0FE01200A9031
:1019D00010E411F075FA01460090D82010F0D6FE00
:1019E00001200A9006E411F083FA01460090D92004
:1019F00010F0CCFE01200A9006E411F073FA0146C3
:101A00000090DA2010F0C2FE01200A9006E411F0E6
:101A100027FA01460090DB2010F0B8FE01200A9062
:101A200006E411F02FFA01460090DC2010F0AEFE23
:101A300001200A9006E411F01FFA01460090DD2013
:101A400010F0A4FE01200A9006E411F093FA01467A
:101A50000090DE2010F09AFE01200A9006E411F0BA
:101A600083FA01460090DF2010F090FE01200A90DA
:101A700006E411F019FA01460090E02010F086FE0D
:101A800001200A9006E411F07BFA01460090E12063
:101A900010F07CFE01200A9006E411F01DFA0146C8
:101AA0000090E22010F072FE01200A9006E411F08E
:101AB0006DFA01460090E32010F068FE01200A90C4
:101AC00006E411F0B5F901460090E42010F05EFE46
:101AD00001200A9006E411F0E1F901460090E520AA
:101AE00010F054FE01200A9006E411F0A7F9014617
:101AF0000090E62010F04AFE01200A9006E411F062
:101B000009FA01460090E72010F040FE01200A90FB
:101B10001EE411F01DFA01460090E82010F036FE98
:101B200001200A9014E411F0B3F901460090E92075
:101B300010F02CFE01200A900AE411F097F90146FA
:101B40000090EA2010F022FE01200A9018E411F023
:101B500063F901460090EB2010F018FE01200A9076
:101B60000EE411F025FA01460090EC2010F0F0FD93
:101B700001200A9001E211F021FA01460090ED20C7
:101B800010F0E6FD01200A90F7E111F01DFA014680
:101B90000090EE2010F0DCFD01200A90EDE111F044
:101BA00025FA01460090EF2010F0D2FD01200A90A6
:101BB000E3E111F0F1F901460090F02010F0C8FDCA
:101BC00001200A90D9E111F0EDF901460090F120D1
:101BD00010F0BEFD01200A90CFE111F0FBF90146A3
:101BE0000090F22010F0B4FD01200A90C5E111F040
:101BF000F7F901460090F32010F0AAFD01200A90A9
:101C0000BBE111F0DFF801460090F42010F0BEFDBA
